
SPI_Temp_Control.elf:     file format elf32-littlearm

Sections:
Idx Name          Size      VMA       LMA       File off  Algn
  0 .isr_vector   000001ac  08000000  08000000  00010000  2**0
                  CONTENTS, ALLOC, LOAD, READONLY, DATA
  1 .text         00006bac  080001b0  080001b0  000101b0  2**4
                  CONTENTS, ALLOC, LOAD, READONLY, CODE
  2 .rodata       000004cc  08006d60  08006d60  00016d60  2**3
                  CONTENTS, ALLOC, LOAD, READONLY, DATA
  3 .ARM.extab    00000000  0800722c  0800722c  000201dc  2**0
                  CONTENTS
  4 .ARM          00000008  0800722c  0800722c  0001722c  2**2
                  CONTENTS, ALLOC, LOAD, READONLY, DATA
  5 .preinit_array 00000000  08007234  08007234  000201dc  2**0
                  CONTENTS, ALLOC, LOAD, DATA
  6 .init_array   00000004  08007234  08007234  00017234  2**2
                  CONTENTS, ALLOC, LOAD, DATA
  7 .fini_array   00000004  08007238  08007238  00017238  2**2
                  CONTENTS, ALLOC, LOAD, DATA
  8 .data         000001dc  20000000  0800723c  00020000  2**2
                  CONTENTS, ALLOC, LOAD, DATA
  9 .ccmram       00000000  10000000  10000000  000201dc  2**0
                  CONTENTS
 10 .bss          000000d0  200001dc  200001dc  000201dc  2**2
                  ALLOC
 11 ._user_heap_stack 00000604  200002ac  200002ac  000201dc  2**0
                  ALLOC
 12 .ARM.attributes 00000030  00000000  00000000  000201dc  2**0
                  CONTENTS, READONLY
 13 .debug_info   0000a0c1  00000000  00000000  0002020c  2**0
                  CONTENTS, READONLY, DEBUGGING, OCTETS
 14 .debug_abbrev 00001739  00000000  00000000  0002a2cd  2**0
                  CONTENTS, READONLY, DEBUGGING, OCTETS
 15 .debug_aranges 000008c8  00000000  00000000  0002ba08  2**3
                  CONTENTS, READONLY, DEBUGGING, OCTETS
 16 .debug_ranges 00000830  00000000  00000000  0002c2d0  2**3
                  CONTENTS, READONLY, DEBUGGING, OCTETS
 17 .debug_macro  000235b9  00000000  00000000  0002cb00  2**0
                  CONTENTS, READONLY, DEBUGGING, OCTETS
 18 .debug_line   0000a090  00000000  00000000  000500b9  2**0
                  CONTENTS, READONLY, DEBUGGING, OCTETS
 19 .debug_str    000d49c4  00000000  00000000  0005a149  2**0
                  CONTENTS, READONLY, DEBUGGING, OCTETS
 20 .comment      00000050  00000000  00000000  0012eb0d  2**0
                  CONTENTS, READONLY
 21 .debug_frame  00003550  00000000  00000000  0012eb60  2**2
                  CONTENTS, READONLY, DEBUGGING, OCTETS

Disassembly of section .text:

080001b0 <__do_global_dtors_aux>:
 80001b0:	b510      	push	{r4, lr}
 80001b2:	4c05      	ldr	r4, [pc, #20]	; (80001c8 <__do_global_dtors_aux+0x18>)
 80001b4:	7823      	ldrb	r3, [r4, #0]
 80001b6:	b933      	cbnz	r3, 80001c6 <__do_global_dtors_aux+0x16>
 80001b8:	4b04      	ldr	r3, [pc, #16]	; (80001cc <__do_global_dtors_aux+0x1c>)
 80001ba:	b113      	cbz	r3, 80001c2 <__do_global_dtors_aux+0x12>
 80001bc:	4804      	ldr	r0, [pc, #16]	; (80001d0 <__do_global_dtors_aux+0x20>)
 80001be:	f3af 8000 	nop.w
 80001c2:	2301      	movs	r3, #1
 80001c4:	7023      	strb	r3, [r4, #0]
 80001c6:	bd10      	pop	{r4, pc}
 80001c8:	200001dc 	.word	0x200001dc
 80001cc:	00000000 	.word	0x00000000
 80001d0:	08006d44 	.word	0x08006d44

080001d4 <frame_dummy>:
 80001d4:	b508      	push	{r3, lr}
 80001d6:	4b03      	ldr	r3, [pc, #12]	; (80001e4 <frame_dummy+0x10>)
 80001d8:	b11b      	cbz	r3, 80001e2 <frame_dummy+0xe>
 80001da:	4903      	ldr	r1, [pc, #12]	; (80001e8 <frame_dummy+0x14>)
 80001dc:	4803      	ldr	r0, [pc, #12]	; (80001ec <frame_dummy+0x18>)
 80001de:	f3af 8000 	nop.w
 80001e2:	bd08      	pop	{r3, pc}
 80001e4:	00000000 	.word	0x00000000
 80001e8:	200001e0 	.word	0x200001e0
 80001ec:	08006d44 	.word	0x08006d44

080001f0 <strlen>:
 80001f0:	4603      	mov	r3, r0
 80001f2:	f813 2b01 	ldrb.w	r2, [r3], #1
 80001f6:	2a00      	cmp	r2, #0
 80001f8:	d1fb      	bne.n	80001f2 <strlen+0x2>
 80001fa:	1a18      	subs	r0, r3, r0
 80001fc:	3801      	subs	r0, #1
 80001fe:	4770      	bx	lr

08000200 <memchr>:
 8000200:	f001 01ff 	and.w	r1, r1, #255	; 0xff
 8000204:	2a10      	cmp	r2, #16
 8000206:	db2b      	blt.n	8000260 <memchr+0x60>
 8000208:	f010 0f07 	tst.w	r0, #7
 800020c:	d008      	beq.n	8000220 <memchr+0x20>
 800020e:	f810 3b01 	ldrb.w	r3, [r0], #1
 8000212:	3a01      	subs	r2, #1
 8000214:	428b      	cmp	r3, r1
 8000216:	d02d      	beq.n	8000274 <memchr+0x74>
 8000218:	f010 0f07 	tst.w	r0, #7
 800021c:	b342      	cbz	r2, 8000270 <memchr+0x70>
 800021e:	d1f6      	bne.n	800020e <memchr+0xe>
 8000220:	b4f0      	push	{r4, r5, r6, r7}
 8000222:	ea41 2101 	orr.w	r1, r1, r1, lsl #8
 8000226:	ea41 4101 	orr.w	r1, r1, r1, lsl #16
 800022a:	f022 0407 	bic.w	r4, r2, #7
 800022e:	f07f 0700 	mvns.w	r7, #0
 8000232:	2300      	movs	r3, #0
 8000234:	e8f0 5602 	ldrd	r5, r6, [r0], #8
 8000238:	3c08      	subs	r4, #8
 800023a:	ea85 0501 	eor.w	r5, r5, r1
 800023e:	ea86 0601 	eor.w	r6, r6, r1
 8000242:	fa85 f547 	uadd8	r5, r5, r7
 8000246:	faa3 f587 	sel	r5, r3, r7
 800024a:	fa86 f647 	uadd8	r6, r6, r7
 800024e:	faa5 f687 	sel	r6, r5, r7
 8000252:	b98e      	cbnz	r6, 8000278 <memchr+0x78>
 8000254:	d1ee      	bne.n	8000234 <memchr+0x34>
 8000256:	bcf0      	pop	{r4, r5, r6, r7}
 8000258:	f001 01ff 	and.w	r1, r1, #255	; 0xff
 800025c:	f002 0207 	and.w	r2, r2, #7
 8000260:	b132      	cbz	r2, 8000270 <memchr+0x70>
 8000262:	f810 3b01 	ldrb.w	r3, [r0], #1
 8000266:	3a01      	subs	r2, #1
 8000268:	ea83 0301 	eor.w	r3, r3, r1
 800026c:	b113      	cbz	r3, 8000274 <memchr+0x74>
 800026e:	d1f8      	bne.n	8000262 <memchr+0x62>
 8000270:	2000      	movs	r0, #0
 8000272:	4770      	bx	lr
 8000274:	3801      	subs	r0, #1
 8000276:	4770      	bx	lr
 8000278:	2d00      	cmp	r5, #0
 800027a:	bf06      	itte	eq
 800027c:	4635      	moveq	r5, r6
 800027e:	3803      	subeq	r0, #3
 8000280:	3807      	subne	r0, #7
 8000282:	f015 0f01 	tst.w	r5, #1
 8000286:	d107      	bne.n	8000298 <memchr+0x98>
 8000288:	3001      	adds	r0, #1
 800028a:	f415 7f80 	tst.w	r5, #256	; 0x100
 800028e:	bf02      	ittt	eq
 8000290:	3001      	addeq	r0, #1
 8000292:	f415 3fc0 	tsteq.w	r5, #98304	; 0x18000
 8000296:	3001      	addeq	r0, #1
 8000298:	bcf0      	pop	{r4, r5, r6, r7}
 800029a:	3801      	subs	r0, #1
 800029c:	4770      	bx	lr
 800029e:	bf00      	nop

080002a0 <__aeabi_drsub>:
 80002a0:	f081 4100 	eor.w	r1, r1, #2147483648	; 0x80000000
 80002a4:	e002      	b.n	80002ac <__adddf3>
 80002a6:	bf00      	nop

080002a8 <__aeabi_dsub>:
 80002a8:	f083 4300 	eor.w	r3, r3, #2147483648	; 0x80000000

080002ac <__adddf3>:
 80002ac:	b530      	push	{r4, r5, lr}
 80002ae:	ea4f 0441 	mov.w	r4, r1, lsl #1
 80002b2:	ea4f 0543 	mov.w	r5, r3, lsl #1
 80002b6:	ea94 0f05 	teq	r4, r5
 80002ba:	bf08      	it	eq
 80002bc:	ea90 0f02 	teqeq	r0, r2
 80002c0:	bf1f      	itttt	ne
 80002c2:	ea54 0c00 	orrsne.w	ip, r4, r0
 80002c6:	ea55 0c02 	orrsne.w	ip, r5, r2
 80002ca:	ea7f 5c64 	mvnsne.w	ip, r4, asr #21
 80002ce:	ea7f 5c65 	mvnsne.w	ip, r5, asr #21
 80002d2:	f000 80e2 	beq.w	800049a <__adddf3+0x1ee>
 80002d6:	ea4f 5454 	mov.w	r4, r4, lsr #21
 80002da:	ebd4 5555 	rsbs	r5, r4, r5, lsr #21
 80002de:	bfb8      	it	lt
 80002e0:	426d      	neglt	r5, r5
 80002e2:	dd0c      	ble.n	80002fe <__adddf3+0x52>
 80002e4:	442c      	add	r4, r5
 80002e6:	ea80 0202 	eor.w	r2, r0, r2
 80002ea:	ea81 0303 	eor.w	r3, r1, r3
 80002ee:	ea82 0000 	eor.w	r0, r2, r0
 80002f2:	ea83 0101 	eor.w	r1, r3, r1
 80002f6:	ea80 0202 	eor.w	r2, r0, r2
 80002fa:	ea81 0303 	eor.w	r3, r1, r3
 80002fe:	2d36      	cmp	r5, #54	; 0x36
 8000300:	bf88      	it	hi
 8000302:	bd30      	pophi	{r4, r5, pc}
 8000304:	f011 4f00 	tst.w	r1, #2147483648	; 0x80000000
 8000308:	ea4f 3101 	mov.w	r1, r1, lsl #12
 800030c:	f44f 1c80 	mov.w	ip, #1048576	; 0x100000
 8000310:	ea4c 3111 	orr.w	r1, ip, r1, lsr #12
 8000314:	d002      	beq.n	800031c <__adddf3+0x70>
 8000316:	4240      	negs	r0, r0
 8000318:	eb61 0141 	sbc.w	r1, r1, r1, lsl #1
 800031c:	f013 4f00 	tst.w	r3, #2147483648	; 0x80000000
 8000320:	ea4f 3303 	mov.w	r3, r3, lsl #12
 8000324:	ea4c 3313 	orr.w	r3, ip, r3, lsr #12
 8000328:	d002      	beq.n	8000330 <__adddf3+0x84>
 800032a:	4252      	negs	r2, r2
 800032c:	eb63 0343 	sbc.w	r3, r3, r3, lsl #1
 8000330:	ea94 0f05 	teq	r4, r5
 8000334:	f000 80a7 	beq.w	8000486 <__adddf3+0x1da>
 8000338:	f1a4 0401 	sub.w	r4, r4, #1
 800033c:	f1d5 0e20 	rsbs	lr, r5, #32
 8000340:	db0d      	blt.n	800035e <__adddf3+0xb2>
 8000342:	fa02 fc0e 	lsl.w	ip, r2, lr
 8000346:	fa22 f205 	lsr.w	r2, r2, r5
 800034a:	1880      	adds	r0, r0, r2
 800034c:	f141 0100 	adc.w	r1, r1, #0
 8000350:	fa03 f20e 	lsl.w	r2, r3, lr
 8000354:	1880      	adds	r0, r0, r2
 8000356:	fa43 f305 	asr.w	r3, r3, r5
 800035a:	4159      	adcs	r1, r3
 800035c:	e00e      	b.n	800037c <__adddf3+0xd0>
 800035e:	f1a5 0520 	sub.w	r5, r5, #32
 8000362:	f10e 0e20 	add.w	lr, lr, #32
 8000366:	2a01      	cmp	r2, #1
 8000368:	fa03 fc0e 	lsl.w	ip, r3, lr
 800036c:	bf28      	it	cs
 800036e:	f04c 0c02 	orrcs.w	ip, ip, #2
 8000372:	fa43 f305 	asr.w	r3, r3, r5
 8000376:	18c0      	adds	r0, r0, r3
 8000378:	eb51 71e3 	adcs.w	r1, r1, r3, asr #31
 800037c:	f001 4500 	and.w	r5, r1, #2147483648	; 0x80000000
 8000380:	d507      	bpl.n	8000392 <__adddf3+0xe6>
 8000382:	f04f 0e00 	mov.w	lr, #0
 8000386:	f1dc 0c00 	rsbs	ip, ip, #0
 800038a:	eb7e 0000 	sbcs.w	r0, lr, r0
 800038e:	eb6e 0101 	sbc.w	r1, lr, r1
 8000392:	f5b1 1f80 	cmp.w	r1, #1048576	; 0x100000
 8000396:	d31b      	bcc.n	80003d0 <__adddf3+0x124>
 8000398:	f5b1 1f00 	cmp.w	r1, #2097152	; 0x200000
 800039c:	d30c      	bcc.n	80003b8 <__adddf3+0x10c>
 800039e:	0849      	lsrs	r1, r1, #1
 80003a0:	ea5f 0030 	movs.w	r0, r0, rrx
 80003a4:	ea4f 0c3c 	mov.w	ip, ip, rrx
 80003a8:	f104 0401 	add.w	r4, r4, #1
 80003ac:	ea4f 5244 	mov.w	r2, r4, lsl #21
 80003b0:	f512 0f80 	cmn.w	r2, #4194304	; 0x400000
 80003b4:	f080 809a 	bcs.w	80004ec <__adddf3+0x240>
 80003b8:	f1bc 4f00 	cmp.w	ip, #2147483648	; 0x80000000
 80003bc:	bf08      	it	eq
 80003be:	ea5f 0c50 	movseq.w	ip, r0, lsr #1
 80003c2:	f150 0000 	adcs.w	r0, r0, #0
 80003c6:	eb41 5104 	adc.w	r1, r1, r4, lsl #20
 80003ca:	ea41 0105 	orr.w	r1, r1, r5
 80003ce:	bd30      	pop	{r4, r5, pc}
 80003d0:	ea5f 0c4c 	movs.w	ip, ip, lsl #1
 80003d4:	4140      	adcs	r0, r0
 80003d6:	eb41 0101 	adc.w	r1, r1, r1
 80003da:	3c01      	subs	r4, #1
 80003dc:	bf28      	it	cs
 80003de:	f5b1 1f80 	cmpcs.w	r1, #1048576	; 0x100000
 80003e2:	d2e9      	bcs.n	80003b8 <__adddf3+0x10c>
 80003e4:	f091 0f00 	teq	r1, #0
 80003e8:	bf04      	itt	eq
 80003ea:	4601      	moveq	r1, r0
 80003ec:	2000      	moveq	r0, #0
 80003ee:	fab1 f381 	clz	r3, r1
 80003f2:	bf08      	it	eq
 80003f4:	3320      	addeq	r3, #32
 80003f6:	f1a3 030b 	sub.w	r3, r3, #11
 80003fa:	f1b3 0220 	subs.w	r2, r3, #32
 80003fe:	da0c      	bge.n	800041a <__adddf3+0x16e>
 8000400:	320c      	adds	r2, #12
 8000402:	dd08      	ble.n	8000416 <__adddf3+0x16a>
 8000404:	f102 0c14 	add.w	ip, r2, #20
 8000408:	f1c2 020c 	rsb	r2, r2, #12
 800040c:	fa01 f00c 	lsl.w	r0, r1, ip
 8000410:	fa21 f102 	lsr.w	r1, r1, r2
 8000414:	e00c      	b.n	8000430 <__adddf3+0x184>
 8000416:	f102 0214 	add.w	r2, r2, #20
 800041a:	bfd8      	it	le
 800041c:	f1c2 0c20 	rsble	ip, r2, #32
 8000420:	fa01 f102 	lsl.w	r1, r1, r2
 8000424:	fa20 fc0c 	lsr.w	ip, r0, ip
 8000428:	bfdc      	itt	le
 800042a:	ea41 010c 	orrle.w	r1, r1, ip
 800042e:	4090      	lslle	r0, r2
 8000430:	1ae4      	subs	r4, r4, r3
 8000432:	bfa2      	ittt	ge
 8000434:	eb01 5104 	addge.w	r1, r1, r4, lsl #20
 8000438:	4329      	orrge	r1, r5
 800043a:	bd30      	popge	{r4, r5, pc}
 800043c:	ea6f 0404 	mvn.w	r4, r4
 8000440:	3c1f      	subs	r4, #31
 8000442:	da1c      	bge.n	800047e <__adddf3+0x1d2>
 8000444:	340c      	adds	r4, #12
 8000446:	dc0e      	bgt.n	8000466 <__adddf3+0x1ba>
 8000448:	f104 0414 	add.w	r4, r4, #20
 800044c:	f1c4 0220 	rsb	r2, r4, #32
 8000450:	fa20 f004 	lsr.w	r0, r0, r4
 8000454:	fa01 f302 	lsl.w	r3, r1, r2
 8000458:	ea40 0003 	orr.w	r0, r0, r3
 800045c:	fa21 f304 	lsr.w	r3, r1, r4
 8000460:	ea45 0103 	orr.w	r1, r5, r3
 8000464:	bd30      	pop	{r4, r5, pc}
 8000466:	f1c4 040c 	rsb	r4, r4, #12
 800046a:	f1c4 0220 	rsb	r2, r4, #32
 800046e:	fa20 f002 	lsr.w	r0, r0, r2
 8000472:	fa01 f304 	lsl.w	r3, r1, r4
 8000476:	ea40 0003 	orr.w	r0, r0, r3
 800047a:	4629      	mov	r1, r5
 800047c:	bd30      	pop	{r4, r5, pc}
 800047e:	fa21 f004 	lsr.w	r0, r1, r4
 8000482:	4629      	mov	r1, r5
 8000484:	bd30      	pop	{r4, r5, pc}
 8000486:	f094 0f00 	teq	r4, #0
 800048a:	f483 1380 	eor.w	r3, r3, #1048576	; 0x100000
 800048e:	bf06      	itte	eq
 8000490:	f481 1180 	eoreq.w	r1, r1, #1048576	; 0x100000
 8000494:	3401      	addeq	r4, #1
 8000496:	3d01      	subne	r5, #1
 8000498:	e74e      	b.n	8000338 <__adddf3+0x8c>
 800049a:	ea7f 5c64 	mvns.w	ip, r4, asr #21
 800049e:	bf18      	it	ne
 80004a0:	ea7f 5c65 	mvnsne.w	ip, r5, asr #21
 80004a4:	d029      	beq.n	80004fa <__adddf3+0x24e>
 80004a6:	ea94 0f05 	teq	r4, r5
 80004aa:	bf08      	it	eq
 80004ac:	ea90 0f02 	teqeq	r0, r2
 80004b0:	d005      	beq.n	80004be <__adddf3+0x212>
 80004b2:	ea54 0c00 	orrs.w	ip, r4, r0
 80004b6:	bf04      	itt	eq
 80004b8:	4619      	moveq	r1, r3
 80004ba:	4610      	moveq	r0, r2
 80004bc:	bd30      	pop	{r4, r5, pc}
 80004be:	ea91 0f03 	teq	r1, r3
 80004c2:	bf1e      	ittt	ne
 80004c4:	2100      	movne	r1, #0
 80004c6:	2000      	movne	r0, #0
 80004c8:	bd30      	popne	{r4, r5, pc}
 80004ca:	ea5f 5c54 	movs.w	ip, r4, lsr #21
 80004ce:	d105      	bne.n	80004dc <__adddf3+0x230>
 80004d0:	0040      	lsls	r0, r0, #1
 80004d2:	4149      	adcs	r1, r1
 80004d4:	bf28      	it	cs
 80004d6:	f041 4100 	orrcs.w	r1, r1, #2147483648	; 0x80000000
 80004da:	bd30      	pop	{r4, r5, pc}
 80004dc:	f514 0480 	adds.w	r4, r4, #4194304	; 0x400000
 80004e0:	bf3c      	itt	cc
 80004e2:	f501 1180 	addcc.w	r1, r1, #1048576	; 0x100000
 80004e6:	bd30      	popcc	{r4, r5, pc}
 80004e8:	f001 4500 	and.w	r5, r1, #2147483648	; 0x80000000
 80004ec:	f045 41fe 	orr.w	r1, r5, #2130706432	; 0x7f000000
 80004f0:	f441 0170 	orr.w	r1, r1, #15728640	; 0xf00000
 80004f4:	f04f 0000 	mov.w	r0, #0
 80004f8:	bd30      	pop	{r4, r5, pc}
 80004fa:	ea7f 5c64 	mvns.w	ip, r4, asr #21
 80004fe:	bf1a      	itte	ne
 8000500:	4619      	movne	r1, r3
 8000502:	4610      	movne	r0, r2
 8000504:	ea7f 5c65 	mvnseq.w	ip, r5, asr #21
 8000508:	bf1c      	itt	ne
 800050a:	460b      	movne	r3, r1
 800050c:	4602      	movne	r2, r0
 800050e:	ea50 3401 	orrs.w	r4, r0, r1, lsl #12
 8000512:	bf06      	itte	eq
 8000514:	ea52 3503 	orrseq.w	r5, r2, r3, lsl #12
 8000518:	ea91 0f03 	teqeq	r1, r3
 800051c:	f441 2100 	orrne.w	r1, r1, #524288	; 0x80000
 8000520:	bd30      	pop	{r4, r5, pc}
 8000522:	bf00      	nop

08000524 <__aeabi_ui2d>:
 8000524:	f090 0f00 	teq	r0, #0
 8000528:	bf04      	itt	eq
 800052a:	2100      	moveq	r1, #0
 800052c:	4770      	bxeq	lr
 800052e:	b530      	push	{r4, r5, lr}
 8000530:	f44f 6480 	mov.w	r4, #1024	; 0x400
 8000534:	f104 0432 	add.w	r4, r4, #50	; 0x32
 8000538:	f04f 0500 	mov.w	r5, #0
 800053c:	f04f 0100 	mov.w	r1, #0
 8000540:	e750      	b.n	80003e4 <__adddf3+0x138>
 8000542:	bf00      	nop

08000544 <__aeabi_i2d>:
 8000544:	f090 0f00 	teq	r0, #0
 8000548:	bf04      	itt	eq
 800054a:	2100      	moveq	r1, #0
 800054c:	4770      	bxeq	lr
 800054e:	b530      	push	{r4, r5, lr}
 8000550:	f44f 6480 	mov.w	r4, #1024	; 0x400
 8000554:	f104 0432 	add.w	r4, r4, #50	; 0x32
 8000558:	f010 4500 	ands.w	r5, r0, #2147483648	; 0x80000000
 800055c:	bf48      	it	mi
 800055e:	4240      	negmi	r0, r0
 8000560:	f04f 0100 	mov.w	r1, #0
 8000564:	e73e      	b.n	80003e4 <__adddf3+0x138>
 8000566:	bf00      	nop

08000568 <__aeabi_f2d>:
 8000568:	0042      	lsls	r2, r0, #1
 800056a:	ea4f 01e2 	mov.w	r1, r2, asr #3
 800056e:	ea4f 0131 	mov.w	r1, r1, rrx
 8000572:	ea4f 7002 	mov.w	r0, r2, lsl #28
 8000576:	bf1f      	itttt	ne
 8000578:	f012 437f 	andsne.w	r3, r2, #4278190080	; 0xff000000
 800057c:	f093 4f7f 	teqne	r3, #4278190080	; 0xff000000
 8000580:	f081 5160 	eorne.w	r1, r1, #939524096	; 0x38000000
 8000584:	4770      	bxne	lr
 8000586:	f032 427f 	bics.w	r2, r2, #4278190080	; 0xff000000
 800058a:	bf08      	it	eq
 800058c:	4770      	bxeq	lr
 800058e:	f093 4f7f 	teq	r3, #4278190080	; 0xff000000
 8000592:	bf04      	itt	eq
 8000594:	f441 2100 	orreq.w	r1, r1, #524288	; 0x80000
 8000598:	4770      	bxeq	lr
 800059a:	b530      	push	{r4, r5, lr}
 800059c:	f44f 7460 	mov.w	r4, #896	; 0x380
 80005a0:	f001 4500 	and.w	r5, r1, #2147483648	; 0x80000000
 80005a4:	f021 4100 	bic.w	r1, r1, #2147483648	; 0x80000000
 80005a8:	e71c      	b.n	80003e4 <__adddf3+0x138>
 80005aa:	bf00      	nop

080005ac <__aeabi_ul2d>:
 80005ac:	ea50 0201 	orrs.w	r2, r0, r1
 80005b0:	bf08      	it	eq
 80005b2:	4770      	bxeq	lr
 80005b4:	b530      	push	{r4, r5, lr}
 80005b6:	f04f 0500 	mov.w	r5, #0
 80005ba:	e00a      	b.n	80005d2 <__aeabi_l2d+0x16>

080005bc <__aeabi_l2d>:
 80005bc:	ea50 0201 	orrs.w	r2, r0, r1
 80005c0:	bf08      	it	eq
 80005c2:	4770      	bxeq	lr
 80005c4:	b530      	push	{r4, r5, lr}
 80005c6:	f011 4500 	ands.w	r5, r1, #2147483648	; 0x80000000
 80005ca:	d502      	bpl.n	80005d2 <__aeabi_l2d+0x16>
 80005cc:	4240      	negs	r0, r0
 80005ce:	eb61 0141 	sbc.w	r1, r1, r1, lsl #1
 80005d2:	f44f 6480 	mov.w	r4, #1024	; 0x400
 80005d6:	f104 0432 	add.w	r4, r4, #50	; 0x32
 80005da:	ea5f 5c91 	movs.w	ip, r1, lsr #22
 80005de:	f43f aed8 	beq.w	8000392 <__adddf3+0xe6>
 80005e2:	f04f 0203 	mov.w	r2, #3
 80005e6:	ea5f 0cdc 	movs.w	ip, ip, lsr #3
 80005ea:	bf18      	it	ne
 80005ec:	3203      	addne	r2, #3
 80005ee:	ea5f 0cdc 	movs.w	ip, ip, lsr #3
 80005f2:	bf18      	it	ne
 80005f4:	3203      	addne	r2, #3
 80005f6:	eb02 02dc 	add.w	r2, r2, ip, lsr #3
 80005fa:	f1c2 0320 	rsb	r3, r2, #32
 80005fe:	fa00 fc03 	lsl.w	ip, r0, r3
 8000602:	fa20 f002 	lsr.w	r0, r0, r2
 8000606:	fa01 fe03 	lsl.w	lr, r1, r3
 800060a:	ea40 000e 	orr.w	r0, r0, lr
 800060e:	fa21 f102 	lsr.w	r1, r1, r2
 8000612:	4414      	add	r4, r2
 8000614:	e6bd      	b.n	8000392 <__adddf3+0xe6>
 8000616:	bf00      	nop

08000618 <__aeabi_dmul>:
 8000618:	b570      	push	{r4, r5, r6, lr}
 800061a:	f04f 0cff 	mov.w	ip, #255	; 0xff
 800061e:	f44c 6ce0 	orr.w	ip, ip, #1792	; 0x700
 8000622:	ea1c 5411 	ands.w	r4, ip, r1, lsr #20
 8000626:	bf1d      	ittte	ne
 8000628:	ea1c 5513 	andsne.w	r5, ip, r3, lsr #20
 800062c:	ea94 0f0c 	teqne	r4, ip
 8000630:	ea95 0f0c 	teqne	r5, ip
 8000634:	f000 f8de 	bleq	80007f4 <__aeabi_dmul+0x1dc>
 8000638:	442c      	add	r4, r5
 800063a:	ea81 0603 	eor.w	r6, r1, r3
 800063e:	ea21 514c 	bic.w	r1, r1, ip, lsl #21
 8000642:	ea23 534c 	bic.w	r3, r3, ip, lsl #21
 8000646:	ea50 3501 	orrs.w	r5, r0, r1, lsl #12
 800064a:	bf18      	it	ne
 800064c:	ea52 3503 	orrsne.w	r5, r2, r3, lsl #12
 8000650:	f441 1180 	orr.w	r1, r1, #1048576	; 0x100000
 8000654:	f443 1380 	orr.w	r3, r3, #1048576	; 0x100000
 8000658:	d038      	beq.n	80006cc <__aeabi_dmul+0xb4>
 800065a:	fba0 ce02 	umull	ip, lr, r0, r2
 800065e:	f04f 0500 	mov.w	r5, #0
 8000662:	fbe1 e502 	umlal	lr, r5, r1, r2
 8000666:	f006 4200 	and.w	r2, r6, #2147483648	; 0x80000000
 800066a:	fbe0 e503 	umlal	lr, r5, r0, r3
 800066e:	f04f 0600 	mov.w	r6, #0
 8000672:	fbe1 5603 	umlal	r5, r6, r1, r3
 8000676:	f09c 0f00 	teq	ip, #0
 800067a:	bf18      	it	ne
 800067c:	f04e 0e01 	orrne.w	lr, lr, #1
 8000680:	f1a4 04ff 	sub.w	r4, r4, #255	; 0xff
 8000684:	f5b6 7f00 	cmp.w	r6, #512	; 0x200
 8000688:	f564 7440 	sbc.w	r4, r4, #768	; 0x300
 800068c:	d204      	bcs.n	8000698 <__aeabi_dmul+0x80>
 800068e:	ea5f 0e4e 	movs.w	lr, lr, lsl #1
 8000692:	416d      	adcs	r5, r5
 8000694:	eb46 0606 	adc.w	r6, r6, r6
 8000698:	ea42 21c6 	orr.w	r1, r2, r6, lsl #11
 800069c:	ea41 5155 	orr.w	r1, r1, r5, lsr #21
 80006a0:	ea4f 20c5 	mov.w	r0, r5, lsl #11
 80006a4:	ea40 505e 	orr.w	r0, r0, lr, lsr #21
 80006a8:	ea4f 2ece 	mov.w	lr, lr, lsl #11
 80006ac:	f1b4 0cfd 	subs.w	ip, r4, #253	; 0xfd
 80006b0:	bf88      	it	hi
 80006b2:	f5bc 6fe0 	cmphi.w	ip, #1792	; 0x700
 80006b6:	d81e      	bhi.n	80006f6 <__aeabi_dmul+0xde>
 80006b8:	f1be 4f00 	cmp.w	lr, #2147483648	; 0x80000000
 80006bc:	bf08      	it	eq
 80006be:	ea5f 0e50 	movseq.w	lr, r0, lsr #1
 80006c2:	f150 0000 	adcs.w	r0, r0, #0
 80006c6:	eb41 5104 	adc.w	r1, r1, r4, lsl #20
 80006ca:	bd70      	pop	{r4, r5, r6, pc}
 80006cc:	f006 4600 	and.w	r6, r6, #2147483648	; 0x80000000
 80006d0:	ea46 0101 	orr.w	r1, r6, r1
 80006d4:	ea40 0002 	orr.w	r0, r0, r2
 80006d8:	ea81 0103 	eor.w	r1, r1, r3
 80006dc:	ebb4 045c 	subs.w	r4, r4, ip, lsr #1
 80006e0:	bfc2      	ittt	gt
 80006e2:	ebd4 050c 	rsbsgt	r5, r4, ip
 80006e6:	ea41 5104 	orrgt.w	r1, r1, r4, lsl #20
 80006ea:	bd70      	popgt	{r4, r5, r6, pc}
 80006ec:	f441 1180 	orr.w	r1, r1, #1048576	; 0x100000
 80006f0:	f04f 0e00 	mov.w	lr, #0
 80006f4:	3c01      	subs	r4, #1
 80006f6:	f300 80ab 	bgt.w	8000850 <__aeabi_dmul+0x238>
 80006fa:	f114 0f36 	cmn.w	r4, #54	; 0x36
 80006fe:	bfde      	ittt	le
 8000700:	2000      	movle	r0, #0
 8000702:	f001 4100 	andle.w	r1, r1, #2147483648	; 0x80000000
 8000706:	bd70      	pople	{r4, r5, r6, pc}
 8000708:	f1c4 0400 	rsb	r4, r4, #0
 800070c:	3c20      	subs	r4, #32
 800070e:	da35      	bge.n	800077c <__aeabi_dmul+0x164>
 8000710:	340c      	adds	r4, #12
 8000712:	dc1b      	bgt.n	800074c <__aeabi_dmul+0x134>
 8000714:	f104 0414 	add.w	r4, r4, #20
 8000718:	f1c4 0520 	rsb	r5, r4, #32
 800071c:	fa00 f305 	lsl.w	r3, r0, r5
 8000720:	fa20 f004 	lsr.w	r0, r0, r4
 8000724:	fa01 f205 	lsl.w	r2, r1, r5
 8000728:	ea40 0002 	orr.w	r0, r0, r2
 800072c:	f001 4200 	and.w	r2, r1, #2147483648	; 0x80000000
 8000730:	f021 4100 	bic.w	r1, r1, #2147483648	; 0x80000000
 8000734:	eb10 70d3 	adds.w	r0, r0, r3, lsr #31
 8000738:	fa21 f604 	lsr.w	r6, r1, r4
 800073c:	eb42 0106 	adc.w	r1, r2, r6
 8000740:	ea5e 0e43 	orrs.w	lr, lr, r3, lsl #1
 8000744:	bf08      	it	eq
 8000746:	ea20 70d3 	biceq.w	r0, r0, r3, lsr #31
 800074a:	bd70      	pop	{r4, r5, r6, pc}
 800074c:	f1c4 040c 	rsb	r4, r4, #12
 8000750:	f1c4 0520 	rsb	r5, r4, #32
 8000754:	fa00 f304 	lsl.w	r3, r0, r4
 8000758:	fa20 f005 	lsr.w	r0, r0, r5
 800075c:	fa01 f204 	lsl.w	r2, r1, r4
 8000760:	ea40 0002 	orr.w	r0, r0, r2
 8000764:	f001 4100 	and.w	r1, r1, #2147483648	; 0x80000000
 8000768:	eb10 70d3 	adds.w	r0, r0, r3, lsr #31
 800076c:	f141 0100 	adc.w	r1, r1, #0
 8000770:	ea5e 0e43 	orrs.w	lr, lr, r3, lsl #1
 8000774:	bf08      	it	eq
 8000776:	ea20 70d3 	biceq.w	r0, r0, r3, lsr #31
 800077a:	bd70      	pop	{r4, r5, r6, pc}
 800077c:	f1c4 0520 	rsb	r5, r4, #32
 8000780:	fa00 f205 	lsl.w	r2, r0, r5
 8000784:	ea4e 0e02 	orr.w	lr, lr, r2
 8000788:	fa20 f304 	lsr.w	r3, r0, r4
 800078c:	fa01 f205 	lsl.w	r2, r1, r5
 8000790:	ea43 0302 	orr.w	r3, r3, r2
 8000794:	fa21 f004 	lsr.w	r0, r1, r4
 8000798:	f001 4100 	and.w	r1, r1, #2147483648	; 0x80000000
 800079c:	fa21 f204 	lsr.w	r2, r1, r4
 80007a0:	ea20 0002 	bic.w	r0, r0, r2
 80007a4:	eb00 70d3 	add.w	r0, r0, r3, lsr #31
 80007a8:	ea5e 0e43 	orrs.w	lr, lr, r3, lsl #1
 80007ac:	bf08      	it	eq
 80007ae:	ea20 70d3 	biceq.w	r0, r0, r3, lsr #31
 80007b2:	bd70      	pop	{r4, r5, r6, pc}
 80007b4:	f094 0f00 	teq	r4, #0
 80007b8:	d10f      	bne.n	80007da <__aeabi_dmul+0x1c2>
 80007ba:	f001 4600 	and.w	r6, r1, #2147483648	; 0x80000000
 80007be:	0040      	lsls	r0, r0, #1
 80007c0:	eb41 0101 	adc.w	r1, r1, r1
 80007c4:	f411 1f80 	tst.w	r1, #1048576	; 0x100000
 80007c8:	bf08      	it	eq
 80007ca:	3c01      	subeq	r4, #1
 80007cc:	d0f7      	beq.n	80007be <__aeabi_dmul+0x1a6>
 80007ce:	ea41 0106 	orr.w	r1, r1, r6
 80007d2:	f095 0f00 	teq	r5, #0
 80007d6:	bf18      	it	ne
 80007d8:	4770      	bxne	lr
 80007da:	f003 4600 	and.w	r6, r3, #2147483648	; 0x80000000
 80007de:	0052      	lsls	r2, r2, #1
 80007e0:	eb43 0303 	adc.w	r3, r3, r3
 80007e4:	f413 1f80 	tst.w	r3, #1048576	; 0x100000
 80007e8:	bf08      	it	eq
 80007ea:	3d01      	subeq	r5, #1
 80007ec:	d0f7      	beq.n	80007de <__aeabi_dmul+0x1c6>
 80007ee:	ea43 0306 	orr.w	r3, r3, r6
 80007f2:	4770      	bx	lr
 80007f4:	ea94 0f0c 	teq	r4, ip
 80007f8:	ea0c 5513 	and.w	r5, ip, r3, lsr #20
 80007fc:	bf18      	it	ne
 80007fe:	ea95 0f0c 	teqne	r5, ip
 8000802:	d00c      	beq.n	800081e <__aeabi_dmul+0x206>
 8000804:	ea50 0641 	orrs.w	r6, r0, r1, lsl #1
 8000808:	bf18      	it	ne
 800080a:	ea52 0643 	orrsne.w	r6, r2, r3, lsl #1
 800080e:	d1d1      	bne.n	80007b4 <__aeabi_dmul+0x19c>
 8000810:	ea81 0103 	eor.w	r1, r1, r3
 8000814:	f001 4100 	and.w	r1, r1, #2147483648	; 0x80000000
 8000818:	f04f 0000 	mov.w	r0, #0
 800081c:	bd70      	pop	{r4, r5, r6, pc}
 800081e:	ea50 0641 	orrs.w	r6, r0, r1, lsl #1
 8000822:	bf06      	itte	eq
 8000824:	4610      	moveq	r0, r2
 8000826:	4619      	moveq	r1, r3
 8000828:	ea52 0643 	orrsne.w	r6, r2, r3, lsl #1
 800082c:	d019      	beq.n	8000862 <__aeabi_dmul+0x24a>
 800082e:	ea94 0f0c 	teq	r4, ip
 8000832:	d102      	bne.n	800083a <__aeabi_dmul+0x222>
 8000834:	ea50 3601 	orrs.w	r6, r0, r1, lsl #12
 8000838:	d113      	bne.n	8000862 <__aeabi_dmul+0x24a>
 800083a:	ea95 0f0c 	teq	r5, ip
 800083e:	d105      	bne.n	800084c <__aeabi_dmul+0x234>
 8000840:	ea52 3603 	orrs.w	r6, r2, r3, lsl #12
 8000844:	bf1c      	itt	ne
 8000846:	4610      	movne	r0, r2
 8000848:	4619      	movne	r1, r3
 800084a:	d10a      	bne.n	8000862 <__aeabi_dmul+0x24a>
 800084c:	ea81 0103 	eor.w	r1, r1, r3
 8000850:	f001 4100 	and.w	r1, r1, #2147483648	; 0x80000000
 8000854:	f041 41fe 	orr.w	r1, r1, #2130706432	; 0x7f000000
 8000858:	f441 0170 	orr.w	r1, r1, #15728640	; 0xf00000
 800085c:	f04f 0000 	mov.w	r0, #0
 8000860:	bd70      	pop	{r4, r5, r6, pc}
 8000862:	f041 41fe 	orr.w	r1, r1, #2130706432	; 0x7f000000
 8000866:	f441 0178 	orr.w	r1, r1, #16252928	; 0xf80000
 800086a:	bd70      	pop	{r4, r5, r6, pc}

0800086c <__aeabi_ddiv>:
 800086c:	b570      	push	{r4, r5, r6, lr}
 800086e:	f04f 0cff 	mov.w	ip, #255	; 0xff
 8000872:	f44c 6ce0 	orr.w	ip, ip, #1792	; 0x700
 8000876:	ea1c 5411 	ands.w	r4, ip, r1, lsr #20
 800087a:	bf1d      	ittte	ne
 800087c:	ea1c 5513 	andsne.w	r5, ip, r3, lsr #20
 8000880:	ea94 0f0c 	teqne	r4, ip
 8000884:	ea95 0f0c 	teqne	r5, ip
 8000888:	f000 f8a7 	bleq	80009da <__aeabi_ddiv+0x16e>
 800088c:	eba4 0405 	sub.w	r4, r4, r5
 8000890:	ea81 0e03 	eor.w	lr, r1, r3
 8000894:	ea52 3503 	orrs.w	r5, r2, r3, lsl #12
 8000898:	ea4f 3101 	mov.w	r1, r1, lsl #12
 800089c:	f000 8088 	beq.w	80009b0 <__aeabi_ddiv+0x144>
 80008a0:	ea4f 3303 	mov.w	r3, r3, lsl #12
 80008a4:	f04f 5580 	mov.w	r5, #268435456	; 0x10000000
 80008a8:	ea45 1313 	orr.w	r3, r5, r3, lsr #4
 80008ac:	ea43 6312 	orr.w	r3, r3, r2, lsr #24
 80008b0:	ea4f 2202 	mov.w	r2, r2, lsl #8
 80008b4:	ea45 1511 	orr.w	r5, r5, r1, lsr #4
 80008b8:	ea45 6510 	orr.w	r5, r5, r0, lsr #24
 80008bc:	ea4f 2600 	mov.w	r6, r0, lsl #8
 80008c0:	f00e 4100 	and.w	r1, lr, #2147483648	; 0x80000000
 80008c4:	429d      	cmp	r5, r3
 80008c6:	bf08      	it	eq
 80008c8:	4296      	cmpeq	r6, r2
 80008ca:	f144 04fd 	adc.w	r4, r4, #253	; 0xfd
 80008ce:	f504 7440 	add.w	r4, r4, #768	; 0x300
 80008d2:	d202      	bcs.n	80008da <__aeabi_ddiv+0x6e>
 80008d4:	085b      	lsrs	r3, r3, #1
 80008d6:	ea4f 0232 	mov.w	r2, r2, rrx
 80008da:	1ab6      	subs	r6, r6, r2
 80008dc:	eb65 0503 	sbc.w	r5, r5, r3
 80008e0:	085b      	lsrs	r3, r3, #1
 80008e2:	ea4f 0232 	mov.w	r2, r2, rrx
 80008e6:	f44f 1080 	mov.w	r0, #1048576	; 0x100000
 80008ea:	f44f 2c00 	mov.w	ip, #524288	; 0x80000
 80008ee:	ebb6 0e02 	subs.w	lr, r6, r2
 80008f2:	eb75 0e03 	sbcs.w	lr, r5, r3
 80008f6:	bf22      	ittt	cs
 80008f8:	1ab6      	subcs	r6, r6, r2
 80008fa:	4675      	movcs	r5, lr
 80008fc:	ea40 000c 	orrcs.w	r0, r0, ip
 8000900:	085b      	lsrs	r3, r3, #1
 8000902:	ea4f 0232 	mov.w	r2, r2, rrx
 8000906:	ebb6 0e02 	subs.w	lr, r6, r2
 800090a:	eb75 0e03 	sbcs.w	lr, r5, r3
 800090e:	bf22      	ittt	cs
 8000910:	1ab6      	subcs	r6, r6, r2
 8000912:	4675      	movcs	r5, lr
 8000914:	ea40 005c 	orrcs.w	r0, r0, ip, lsr #1
 8000918:	085b      	lsrs	r3, r3, #1
 800091a:	ea4f 0232 	mov.w	r2, r2, rrx
 800091e:	ebb6 0e02 	subs.w	lr, r6, r2
 8000922:	eb75 0e03 	sbcs.w	lr, r5, r3
 8000926:	bf22      	ittt	cs
 8000928:	1ab6      	subcs	r6, r6, r2
 800092a:	4675      	movcs	r5, lr
 800092c:	ea40 009c 	orrcs.w	r0, r0, ip, lsr #2
 8000930:	085b      	lsrs	r3, r3, #1
 8000932:	ea4f 0232 	mov.w	r2, r2, rrx
 8000936:	ebb6 0e02 	subs.w	lr, r6, r2
 800093a:	eb75 0e03 	sbcs.w	lr, r5, r3
 800093e:	bf22      	ittt	cs
 8000940:	1ab6      	subcs	r6, r6, r2
 8000942:	4675      	movcs	r5, lr
 8000944:	ea40 00dc 	orrcs.w	r0, r0, ip, lsr #3
 8000948:	ea55 0e06 	orrs.w	lr, r5, r6
 800094c:	d018      	beq.n	8000980 <__aeabi_ddiv+0x114>
 800094e:	ea4f 1505 	mov.w	r5, r5, lsl #4
 8000952:	ea45 7516 	orr.w	r5, r5, r6, lsr #28
 8000956:	ea4f 1606 	mov.w	r6, r6, lsl #4
 800095a:	ea4f 03c3 	mov.w	r3, r3, lsl #3
 800095e:	ea43 7352 	orr.w	r3, r3, r2, lsr #29
 8000962:	ea4f 02c2 	mov.w	r2, r2, lsl #3
 8000966:	ea5f 1c1c 	movs.w	ip, ip, lsr #4
 800096a:	d1c0      	bne.n	80008ee <__aeabi_ddiv+0x82>
 800096c:	f411 1f80 	tst.w	r1, #1048576	; 0x100000
 8000970:	d10b      	bne.n	800098a <__aeabi_ddiv+0x11e>
 8000972:	ea41 0100 	orr.w	r1, r1, r0
 8000976:	f04f 0000 	mov.w	r0, #0
 800097a:	f04f 4c00 	mov.w	ip, #2147483648	; 0x80000000
 800097e:	e7b6      	b.n	80008ee <__aeabi_ddiv+0x82>
 8000980:	f411 1f80 	tst.w	r1, #1048576	; 0x100000
 8000984:	bf04      	itt	eq
 8000986:	4301      	orreq	r1, r0
 8000988:	2000      	moveq	r0, #0
 800098a:	f1b4 0cfd 	subs.w	ip, r4, #253	; 0xfd
 800098e:	bf88      	it	hi
 8000990:	f5bc 6fe0 	cmphi.w	ip, #1792	; 0x700
 8000994:	f63f aeaf 	bhi.w	80006f6 <__aeabi_dmul+0xde>
 8000998:	ebb5 0c03 	subs.w	ip, r5, r3
 800099c:	bf04      	itt	eq
 800099e:	ebb6 0c02 	subseq.w	ip, r6, r2
 80009a2:	ea5f 0c50 	movseq.w	ip, r0, lsr #1
 80009a6:	f150 0000 	adcs.w	r0, r0, #0
 80009aa:	eb41 5104 	adc.w	r1, r1, r4, lsl #20
 80009ae:	bd70      	pop	{r4, r5, r6, pc}
 80009b0:	f00e 4e00 	and.w	lr, lr, #2147483648	; 0x80000000
 80009b4:	ea4e 3111 	orr.w	r1, lr, r1, lsr #12
 80009b8:	eb14 045c 	adds.w	r4, r4, ip, lsr #1
 80009bc:	bfc2      	ittt	gt
 80009be:	ebd4 050c 	rsbsgt	r5, r4, ip
 80009c2:	ea41 5104 	orrgt.w	r1, r1, r4, lsl #20
 80009c6:	bd70      	popgt	{r4, r5, r6, pc}
 80009c8:	f441 1180 	orr.w	r1, r1, #1048576	; 0x100000
 80009cc:	f04f 0e00 	mov.w	lr, #0
 80009d0:	3c01      	subs	r4, #1
 80009d2:	e690      	b.n	80006f6 <__aeabi_dmul+0xde>
 80009d4:	ea45 0e06 	orr.w	lr, r5, r6
 80009d8:	e68d      	b.n	80006f6 <__aeabi_dmul+0xde>
 80009da:	ea0c 5513 	and.w	r5, ip, r3, lsr #20
 80009de:	ea94 0f0c 	teq	r4, ip
 80009e2:	bf08      	it	eq
 80009e4:	ea95 0f0c 	teqeq	r5, ip
 80009e8:	f43f af3b 	beq.w	8000862 <__aeabi_dmul+0x24a>
 80009ec:	ea94 0f0c 	teq	r4, ip
 80009f0:	d10a      	bne.n	8000a08 <__aeabi_ddiv+0x19c>
 80009f2:	ea50 3401 	orrs.w	r4, r0, r1, lsl #12
 80009f6:	f47f af34 	bne.w	8000862 <__aeabi_dmul+0x24a>
 80009fa:	ea95 0f0c 	teq	r5, ip
 80009fe:	f47f af25 	bne.w	800084c <__aeabi_dmul+0x234>
 8000a02:	4610      	mov	r0, r2
 8000a04:	4619      	mov	r1, r3
 8000a06:	e72c      	b.n	8000862 <__aeabi_dmul+0x24a>
 8000a08:	ea95 0f0c 	teq	r5, ip
 8000a0c:	d106      	bne.n	8000a1c <__aeabi_ddiv+0x1b0>
 8000a0e:	ea52 3503 	orrs.w	r5, r2, r3, lsl #12
 8000a12:	f43f aefd 	beq.w	8000810 <__aeabi_dmul+0x1f8>
 8000a16:	4610      	mov	r0, r2
 8000a18:	4619      	mov	r1, r3
 8000a1a:	e722      	b.n	8000862 <__aeabi_dmul+0x24a>
 8000a1c:	ea50 0641 	orrs.w	r6, r0, r1, lsl #1
 8000a20:	bf18      	it	ne
 8000a22:	ea52 0643 	orrsne.w	r6, r2, r3, lsl #1
 8000a26:	f47f aec5 	bne.w	80007b4 <__aeabi_dmul+0x19c>
 8000a2a:	ea50 0441 	orrs.w	r4, r0, r1, lsl #1
 8000a2e:	f47f af0d 	bne.w	800084c <__aeabi_dmul+0x234>
 8000a32:	ea52 0543 	orrs.w	r5, r2, r3, lsl #1
 8000a36:	f47f aeeb 	bne.w	8000810 <__aeabi_dmul+0x1f8>
 8000a3a:	e712      	b.n	8000862 <__aeabi_dmul+0x24a>

08000a3c <__gedf2>:
 8000a3c:	f04f 3cff 	mov.w	ip, #4294967295
 8000a40:	e006      	b.n	8000a50 <__cmpdf2+0x4>
 8000a42:	bf00      	nop

08000a44 <__ledf2>:
 8000a44:	f04f 0c01 	mov.w	ip, #1
 8000a48:	e002      	b.n	8000a50 <__cmpdf2+0x4>
 8000a4a:	bf00      	nop

08000a4c <__cmpdf2>:
 8000a4c:	f04f 0c01 	mov.w	ip, #1
 8000a50:	f84d cd04 	str.w	ip, [sp, #-4]!
 8000a54:	ea4f 0c41 	mov.w	ip, r1, lsl #1
 8000a58:	ea7f 5c6c 	mvns.w	ip, ip, asr #21
 8000a5c:	ea4f 0c43 	mov.w	ip, r3, lsl #1
 8000a60:	bf18      	it	ne
 8000a62:	ea7f 5c6c 	mvnsne.w	ip, ip, asr #21
 8000a66:	d01b      	beq.n	8000aa0 <__cmpdf2+0x54>
 8000a68:	b001      	add	sp, #4
 8000a6a:	ea50 0c41 	orrs.w	ip, r0, r1, lsl #1
 8000a6e:	bf0c      	ite	eq
 8000a70:	ea52 0c43 	orrseq.w	ip, r2, r3, lsl #1
 8000a74:	ea91 0f03 	teqne	r1, r3
 8000a78:	bf02      	ittt	eq
 8000a7a:	ea90 0f02 	teqeq	r0, r2
 8000a7e:	2000      	moveq	r0, #0
 8000a80:	4770      	bxeq	lr
 8000a82:	f110 0f00 	cmn.w	r0, #0
 8000a86:	ea91 0f03 	teq	r1, r3
 8000a8a:	bf58      	it	pl
 8000a8c:	4299      	cmppl	r1, r3
 8000a8e:	bf08      	it	eq
 8000a90:	4290      	cmpeq	r0, r2
 8000a92:	bf2c      	ite	cs
 8000a94:	17d8      	asrcs	r0, r3, #31
 8000a96:	ea6f 70e3 	mvncc.w	r0, r3, asr #31
 8000a9a:	f040 0001 	orr.w	r0, r0, #1
 8000a9e:	4770      	bx	lr
 8000aa0:	ea4f 0c41 	mov.w	ip, r1, lsl #1
 8000aa4:	ea7f 5c6c 	mvns.w	ip, ip, asr #21
 8000aa8:	d102      	bne.n	8000ab0 <__cmpdf2+0x64>
 8000aaa:	ea50 3c01 	orrs.w	ip, r0, r1, lsl #12
 8000aae:	d107      	bne.n	8000ac0 <__cmpdf2+0x74>
 8000ab0:	ea4f 0c43 	mov.w	ip, r3, lsl #1
 8000ab4:	ea7f 5c6c 	mvns.w	ip, ip, asr #21
 8000ab8:	d1d6      	bne.n	8000a68 <__cmpdf2+0x1c>
 8000aba:	ea52 3c03 	orrs.w	ip, r2, r3, lsl #12
 8000abe:	d0d3      	beq.n	8000a68 <__cmpdf2+0x1c>
 8000ac0:	f85d 0b04 	ldr.w	r0, [sp], #4
 8000ac4:	4770      	bx	lr
 8000ac6:	bf00      	nop

08000ac8 <__aeabi_cdrcmple>:
 8000ac8:	4684      	mov	ip, r0
 8000aca:	4610      	mov	r0, r2
 8000acc:	4662      	mov	r2, ip
 8000ace:	468c      	mov	ip, r1
 8000ad0:	4619      	mov	r1, r3
 8000ad2:	4663      	mov	r3, ip
 8000ad4:	e000      	b.n	8000ad8 <__aeabi_cdcmpeq>
 8000ad6:	bf00      	nop

08000ad8 <__aeabi_cdcmpeq>:
 8000ad8:	b501      	push	{r0, lr}
 8000ada:	f7ff ffb7 	bl	8000a4c <__cmpdf2>
 8000ade:	2800      	cmp	r0, #0
 8000ae0:	bf48      	it	mi
 8000ae2:	f110 0f00 	cmnmi.w	r0, #0
 8000ae6:	bd01      	pop	{r0, pc}

08000ae8 <__aeabi_dcmpeq>:
 8000ae8:	f84d ed08 	str.w	lr, [sp, #-8]!
 8000aec:	f7ff fff4 	bl	8000ad8 <__aeabi_cdcmpeq>
 8000af0:	bf0c      	ite	eq
 8000af2:	2001      	moveq	r0, #1
 8000af4:	2000      	movne	r0, #0
 8000af6:	f85d fb08 	ldr.w	pc, [sp], #8
 8000afa:	bf00      	nop

08000afc <__aeabi_dcmplt>:
 8000afc:	f84d ed08 	str.w	lr, [sp, #-8]!
 8000b00:	f7ff ffea 	bl	8000ad8 <__aeabi_cdcmpeq>
 8000b04:	bf34      	ite	cc
 8000b06:	2001      	movcc	r0, #1
 8000b08:	2000      	movcs	r0, #0
 8000b0a:	f85d fb08 	ldr.w	pc, [sp], #8
 8000b0e:	bf00      	nop

08000b10 <__aeabi_dcmple>:
 8000b10:	f84d ed08 	str.w	lr, [sp, #-8]!
 8000b14:	f7ff ffe0 	bl	8000ad8 <__aeabi_cdcmpeq>
 8000b18:	bf94      	ite	ls
 8000b1a:	2001      	movls	r0, #1
 8000b1c:	2000      	movhi	r0, #0
 8000b1e:	f85d fb08 	ldr.w	pc, [sp], #8
 8000b22:	bf00      	nop

08000b24 <__aeabi_dcmpge>:
 8000b24:	f84d ed08 	str.w	lr, [sp, #-8]!
 8000b28:	f7ff ffce 	bl	8000ac8 <__aeabi_cdrcmple>
 8000b2c:	bf94      	ite	ls
 8000b2e:	2001      	movls	r0, #1
 8000b30:	2000      	movhi	r0, #0
 8000b32:	f85d fb08 	ldr.w	pc, [sp], #8
 8000b36:	bf00      	nop

08000b38 <__aeabi_dcmpgt>:
 8000b38:	f84d ed08 	str.w	lr, [sp, #-8]!
 8000b3c:	f7ff ffc4 	bl	8000ac8 <__aeabi_cdrcmple>
 8000b40:	bf34      	ite	cc
 8000b42:	2001      	movcc	r0, #1
 8000b44:	2000      	movcs	r0, #0
 8000b46:	f85d fb08 	ldr.w	pc, [sp], #8
 8000b4a:	bf00      	nop

08000b4c <__aeabi_dcmpun>:
 8000b4c:	ea4f 0c41 	mov.w	ip, r1, lsl #1
 8000b50:	ea7f 5c6c 	mvns.w	ip, ip, asr #21
 8000b54:	d102      	bne.n	8000b5c <__aeabi_dcmpun+0x10>
 8000b56:	ea50 3c01 	orrs.w	ip, r0, r1, lsl #12
 8000b5a:	d10a      	bne.n	8000b72 <__aeabi_dcmpun+0x26>
 8000b5c:	ea4f 0c43 	mov.w	ip, r3, lsl #1
 8000b60:	ea7f 5c6c 	mvns.w	ip, ip, asr #21
 8000b64:	d102      	bne.n	8000b6c <__aeabi_dcmpun+0x20>
 8000b66:	ea52 3c03 	orrs.w	ip, r2, r3, lsl #12
 8000b6a:	d102      	bne.n	8000b72 <__aeabi_dcmpun+0x26>
 8000b6c:	f04f 0000 	mov.w	r0, #0
 8000b70:	4770      	bx	lr
 8000b72:	f04f 0001 	mov.w	r0, #1
 8000b76:	4770      	bx	lr

08000b78 <__aeabi_d2iz>:
 8000b78:	ea4f 0241 	mov.w	r2, r1, lsl #1
 8000b7c:	f512 1200 	adds.w	r2, r2, #2097152	; 0x200000
 8000b80:	d215      	bcs.n	8000bae <__aeabi_d2iz+0x36>
 8000b82:	d511      	bpl.n	8000ba8 <__aeabi_d2iz+0x30>
 8000b84:	f46f 7378 	mvn.w	r3, #992	; 0x3e0
 8000b88:	ebb3 5262 	subs.w	r2, r3, r2, asr #21
 8000b8c:	d912      	bls.n	8000bb4 <__aeabi_d2iz+0x3c>
 8000b8e:	ea4f 23c1 	mov.w	r3, r1, lsl #11
 8000b92:	f043 4300 	orr.w	r3, r3, #2147483648	; 0x80000000
 8000b96:	ea43 5350 	orr.w	r3, r3, r0, lsr #21
 8000b9a:	f011 4f00 	tst.w	r1, #2147483648	; 0x80000000
 8000b9e:	fa23 f002 	lsr.w	r0, r3, r2
 8000ba2:	bf18      	it	ne
 8000ba4:	4240      	negne	r0, r0
 8000ba6:	4770      	bx	lr
 8000ba8:	f04f 0000 	mov.w	r0, #0
 8000bac:	4770      	bx	lr
 8000bae:	ea50 3001 	orrs.w	r0, r0, r1, lsl #12
 8000bb2:	d105      	bne.n	8000bc0 <__aeabi_d2iz+0x48>
 8000bb4:	f011 4000 	ands.w	r0, r1, #2147483648	; 0x80000000
 8000bb8:	bf08      	it	eq
 8000bba:	f06f 4000 	mvneq.w	r0, #2147483648	; 0x80000000
 8000bbe:	4770      	bx	lr
 8000bc0:	f04f 0000 	mov.w	r0, #0
 8000bc4:	4770      	bx	lr
 8000bc6:	bf00      	nop

08000bc8 <__aeabi_d2f>:
 8000bc8:	ea4f 0241 	mov.w	r2, r1, lsl #1
 8000bcc:	f1b2 43e0 	subs.w	r3, r2, #1879048192	; 0x70000000
 8000bd0:	bf24      	itt	cs
 8000bd2:	f5b3 1c00 	subscs.w	ip, r3, #2097152	; 0x200000
 8000bd6:	f1dc 5cfe 	rsbscs	ip, ip, #532676608	; 0x1fc00000
 8000bda:	d90d      	bls.n	8000bf8 <__aeabi_d2f+0x30>
 8000bdc:	f001 4c00 	and.w	ip, r1, #2147483648	; 0x80000000
 8000be0:	ea4f 02c0 	mov.w	r2, r0, lsl #3
 8000be4:	ea4c 7050 	orr.w	r0, ip, r0, lsr #29
 8000be8:	f1b2 4f00 	cmp.w	r2, #2147483648	; 0x80000000
 8000bec:	eb40 0083 	adc.w	r0, r0, r3, lsl #2
 8000bf0:	bf08      	it	eq
 8000bf2:	f020 0001 	biceq.w	r0, r0, #1
 8000bf6:	4770      	bx	lr
 8000bf8:	f011 4f80 	tst.w	r1, #1073741824	; 0x40000000
 8000bfc:	d121      	bne.n	8000c42 <__aeabi_d2f+0x7a>
 8000bfe:	f113 7238 	adds.w	r2, r3, #48234496	; 0x2e00000
 8000c02:	bfbc      	itt	lt
 8000c04:	f001 4000 	andlt.w	r0, r1, #2147483648	; 0x80000000
 8000c08:	4770      	bxlt	lr
 8000c0a:	f441 1180 	orr.w	r1, r1, #1048576	; 0x100000
 8000c0e:	ea4f 5252 	mov.w	r2, r2, lsr #21
 8000c12:	f1c2 0218 	rsb	r2, r2, #24
 8000c16:	f1c2 0c20 	rsb	ip, r2, #32
 8000c1a:	fa10 f30c 	lsls.w	r3, r0, ip
 8000c1e:	fa20 f002 	lsr.w	r0, r0, r2
 8000c22:	bf18      	it	ne
 8000c24:	f040 0001 	orrne.w	r0, r0, #1
 8000c28:	ea4f 23c1 	mov.w	r3, r1, lsl #11
 8000c2c:	ea4f 23d3 	mov.w	r3, r3, lsr #11
 8000c30:	fa03 fc0c 	lsl.w	ip, r3, ip
 8000c34:	ea40 000c 	orr.w	r0, r0, ip
 8000c38:	fa23 f302 	lsr.w	r3, r3, r2
 8000c3c:	ea4f 0343 	mov.w	r3, r3, lsl #1
 8000c40:	e7cc      	b.n	8000bdc <__aeabi_d2f+0x14>
 8000c42:	ea7f 5362 	mvns.w	r3, r2, asr #21
 8000c46:	d107      	bne.n	8000c58 <__aeabi_d2f+0x90>
 8000c48:	ea50 3301 	orrs.w	r3, r0, r1, lsl #12
 8000c4c:	bf1e      	ittt	ne
 8000c4e:	f04f 40fe 	movne.w	r0, #2130706432	; 0x7f000000
 8000c52:	f440 0040 	orrne.w	r0, r0, #12582912	; 0xc00000
 8000c56:	4770      	bxne	lr
 8000c58:	f001 4000 	and.w	r0, r1, #2147483648	; 0x80000000
 8000c5c:	f040 40fe 	orr.w	r0, r0, #2130706432	; 0x7f000000
 8000c60:	f440 0000 	orr.w	r0, r0, #8388608	; 0x800000
 8000c64:	4770      	bx	lr
 8000c66:	bf00      	nop

08000c68 <__aeabi_uldivmod>:
 8000c68:	b953      	cbnz	r3, 8000c80 <__aeabi_uldivmod+0x18>
 8000c6a:	b94a      	cbnz	r2, 8000c80 <__aeabi_uldivmod+0x18>
 8000c6c:	2900      	cmp	r1, #0
 8000c6e:	bf08      	it	eq
 8000c70:	2800      	cmpeq	r0, #0
 8000c72:	bf1c      	itt	ne
 8000c74:	f04f 31ff 	movne.w	r1, #4294967295
 8000c78:	f04f 30ff 	movne.w	r0, #4294967295
 8000c7c:	f000 b974 	b.w	8000f68 <__aeabi_idiv0>
 8000c80:	f1ad 0c08 	sub.w	ip, sp, #8
 8000c84:	e96d ce04 	strd	ip, lr, [sp, #-16]!
 8000c88:	f000 f806 	bl	8000c98 <__udivmoddi4>
 8000c8c:	f8dd e004 	ldr.w	lr, [sp, #4]
 8000c90:	e9dd 2302 	ldrd	r2, r3, [sp, #8]
 8000c94:	b004      	add	sp, #16
 8000c96:	4770      	bx	lr

08000c98 <__udivmoddi4>:
 8000c98:	e92d 47f0 	stmdb	sp!, {r4, r5, r6, r7, r8, r9, sl, lr}
 8000c9c:	9d08      	ldr	r5, [sp, #32]
 8000c9e:	4604      	mov	r4, r0
 8000ca0:	468e      	mov	lr, r1
 8000ca2:	2b00      	cmp	r3, #0
 8000ca4:	d14d      	bne.n	8000d42 <__udivmoddi4+0xaa>
 8000ca6:	428a      	cmp	r2, r1
 8000ca8:	4694      	mov	ip, r2
 8000caa:	d969      	bls.n	8000d80 <__udivmoddi4+0xe8>
 8000cac:	fab2 f282 	clz	r2, r2
 8000cb0:	b152      	cbz	r2, 8000cc8 <__udivmoddi4+0x30>
 8000cb2:	fa01 f302 	lsl.w	r3, r1, r2
 8000cb6:	f1c2 0120 	rsb	r1, r2, #32
 8000cba:	fa20 f101 	lsr.w	r1, r0, r1
 8000cbe:	fa0c fc02 	lsl.w	ip, ip, r2
 8000cc2:	ea41 0e03 	orr.w	lr, r1, r3
 8000cc6:	4094      	lsls	r4, r2
 8000cc8:	ea4f 481c 	mov.w	r8, ip, lsr #16
 8000ccc:	0c21      	lsrs	r1, r4, #16
 8000cce:	fbbe f6f8 	udiv	r6, lr, r8
 8000cd2:	fa1f f78c 	uxth.w	r7, ip
 8000cd6:	fb08 e316 	mls	r3, r8, r6, lr
 8000cda:	ea41 4303 	orr.w	r3, r1, r3, lsl #16
 8000cde:	fb06 f107 	mul.w	r1, r6, r7
 8000ce2:	4299      	cmp	r1, r3
 8000ce4:	d90a      	bls.n	8000cfc <__udivmoddi4+0x64>
 8000ce6:	eb1c 0303 	adds.w	r3, ip, r3
 8000cea:	f106 30ff 	add.w	r0, r6, #4294967295
 8000cee:	f080 811f 	bcs.w	8000f30 <__udivmoddi4+0x298>
 8000cf2:	4299      	cmp	r1, r3
 8000cf4:	f240 811c 	bls.w	8000f30 <__udivmoddi4+0x298>
 8000cf8:	3e02      	subs	r6, #2
 8000cfa:	4463      	add	r3, ip
 8000cfc:	1a5b      	subs	r3, r3, r1
 8000cfe:	b2a4      	uxth	r4, r4
 8000d00:	fbb3 f0f8 	udiv	r0, r3, r8
 8000d04:	fb08 3310 	mls	r3, r8, r0, r3
 8000d08:	ea44 4403 	orr.w	r4, r4, r3, lsl #16
 8000d0c:	fb00 f707 	mul.w	r7, r0, r7
 8000d10:	42a7      	cmp	r7, r4
 8000d12:	d90a      	bls.n	8000d2a <__udivmoddi4+0x92>
 8000d14:	eb1c 0404 	adds.w	r4, ip, r4
 8000d18:	f100 33ff 	add.w	r3, r0, #4294967295
 8000d1c:	f080 810a 	bcs.w	8000f34 <__udivmoddi4+0x29c>
 8000d20:	42a7      	cmp	r7, r4
 8000d22:	f240 8107 	bls.w	8000f34 <__udivmoddi4+0x29c>
 8000d26:	4464      	add	r4, ip
 8000d28:	3802      	subs	r0, #2
 8000d2a:	ea40 4006 	orr.w	r0, r0, r6, lsl #16
 8000d2e:	1be4      	subs	r4, r4, r7
 8000d30:	2600      	movs	r6, #0
 8000d32:	b11d      	cbz	r5, 8000d3c <__udivmoddi4+0xa4>
 8000d34:	40d4      	lsrs	r4, r2
 8000d36:	2300      	movs	r3, #0
 8000d38:	e9c5 4300 	strd	r4, r3, [r5]
 8000d3c:	4631      	mov	r1, r6
 8000d3e:	e8bd 87f0 	ldmia.w	sp!, {r4, r5, r6, r7, r8, r9, sl, pc}
 8000d42:	428b      	cmp	r3, r1
 8000d44:	d909      	bls.n	8000d5a <__udivmoddi4+0xc2>
 8000d46:	2d00      	cmp	r5, #0
 8000d48:	f000 80ef 	beq.w	8000f2a <__udivmoddi4+0x292>
 8000d4c:	2600      	movs	r6, #0
 8000d4e:	e9c5 0100 	strd	r0, r1, [r5]
 8000d52:	4630      	mov	r0, r6
 8000d54:	4631      	mov	r1, r6
 8000d56:	e8bd 87f0 	ldmia.w	sp!, {r4, r5, r6, r7, r8, r9, sl, pc}
 8000d5a:	fab3 f683 	clz	r6, r3
 8000d5e:	2e00      	cmp	r6, #0
 8000d60:	d14a      	bne.n	8000df8 <__udivmoddi4+0x160>
 8000d62:	428b      	cmp	r3, r1
 8000d64:	d302      	bcc.n	8000d6c <__udivmoddi4+0xd4>
 8000d66:	4282      	cmp	r2, r0
 8000d68:	f200 80f9 	bhi.w	8000f5e <__udivmoddi4+0x2c6>
 8000d6c:	1a84      	subs	r4, r0, r2
 8000d6e:	eb61 0303 	sbc.w	r3, r1, r3
 8000d72:	2001      	movs	r0, #1
 8000d74:	469e      	mov	lr, r3
 8000d76:	2d00      	cmp	r5, #0
 8000d78:	d0e0      	beq.n	8000d3c <__udivmoddi4+0xa4>
 8000d7a:	e9c5 4e00 	strd	r4, lr, [r5]
 8000d7e:	e7dd      	b.n	8000d3c <__udivmoddi4+0xa4>
 8000d80:	b902      	cbnz	r2, 8000d84 <__udivmoddi4+0xec>
 8000d82:	deff      	udf	#255	; 0xff
 8000d84:	fab2 f282 	clz	r2, r2
 8000d88:	2a00      	cmp	r2, #0
 8000d8a:	f040 8092 	bne.w	8000eb2 <__udivmoddi4+0x21a>
 8000d8e:	eba1 010c 	sub.w	r1, r1, ip
 8000d92:	ea4f 471c 	mov.w	r7, ip, lsr #16
 8000d96:	fa1f fe8c 	uxth.w	lr, ip
 8000d9a:	2601      	movs	r6, #1
 8000d9c:	0c20      	lsrs	r0, r4, #16
 8000d9e:	fbb1 f3f7 	udiv	r3, r1, r7
 8000da2:	fb07 1113 	mls	r1, r7, r3, r1
 8000da6:	ea40 4101 	orr.w	r1, r0, r1, lsl #16
 8000daa:	fb0e f003 	mul.w	r0, lr, r3
 8000dae:	4288      	cmp	r0, r1
 8000db0:	d908      	bls.n	8000dc4 <__udivmoddi4+0x12c>
 8000db2:	eb1c 0101 	adds.w	r1, ip, r1
 8000db6:	f103 38ff 	add.w	r8, r3, #4294967295
 8000dba:	d202      	bcs.n	8000dc2 <__udivmoddi4+0x12a>
 8000dbc:	4288      	cmp	r0, r1
 8000dbe:	f200 80cb 	bhi.w	8000f58 <__udivmoddi4+0x2c0>
 8000dc2:	4643      	mov	r3, r8
 8000dc4:	1a09      	subs	r1, r1, r0
 8000dc6:	b2a4      	uxth	r4, r4
 8000dc8:	fbb1 f0f7 	udiv	r0, r1, r7
 8000dcc:	fb07 1110 	mls	r1, r7, r0, r1
 8000dd0:	ea44 4401 	orr.w	r4, r4, r1, lsl #16
 8000dd4:	fb0e fe00 	mul.w	lr, lr, r0
 8000dd8:	45a6      	cmp	lr, r4
 8000dda:	d908      	bls.n	8000dee <__udivmoddi4+0x156>
 8000ddc:	eb1c 0404 	adds.w	r4, ip, r4
 8000de0:	f100 31ff 	add.w	r1, r0, #4294967295
 8000de4:	d202      	bcs.n	8000dec <__udivmoddi4+0x154>
 8000de6:	45a6      	cmp	lr, r4
 8000de8:	f200 80bb 	bhi.w	8000f62 <__udivmoddi4+0x2ca>
 8000dec:	4608      	mov	r0, r1
 8000dee:	eba4 040e 	sub.w	r4, r4, lr
 8000df2:	ea40 4003 	orr.w	r0, r0, r3, lsl #16
 8000df6:	e79c      	b.n	8000d32 <__udivmoddi4+0x9a>
 8000df8:	f1c6 0720 	rsb	r7, r6, #32
 8000dfc:	40b3      	lsls	r3, r6
 8000dfe:	fa22 fc07 	lsr.w	ip, r2, r7
 8000e02:	ea4c 0c03 	orr.w	ip, ip, r3
 8000e06:	fa20 f407 	lsr.w	r4, r0, r7
 8000e0a:	fa01 f306 	lsl.w	r3, r1, r6
 8000e0e:	431c      	orrs	r4, r3
 8000e10:	40f9      	lsrs	r1, r7
 8000e12:	ea4f 491c 	mov.w	r9, ip, lsr #16
 8000e16:	fa00 f306 	lsl.w	r3, r0, r6
 8000e1a:	fbb1 f8f9 	udiv	r8, r1, r9
 8000e1e:	0c20      	lsrs	r0, r4, #16
 8000e20:	fa1f fe8c 	uxth.w	lr, ip
 8000e24:	fb09 1118 	mls	r1, r9, r8, r1
 8000e28:	ea40 4101 	orr.w	r1, r0, r1, lsl #16
 8000e2c:	fb08 f00e 	mul.w	r0, r8, lr
 8000e30:	4288      	cmp	r0, r1
 8000e32:	fa02 f206 	lsl.w	r2, r2, r6
 8000e36:	d90b      	bls.n	8000e50 <__udivmoddi4+0x1b8>
 8000e38:	eb1c 0101 	adds.w	r1, ip, r1
 8000e3c:	f108 3aff 	add.w	sl, r8, #4294967295
 8000e40:	f080 8088 	bcs.w	8000f54 <__udivmoddi4+0x2bc>
 8000e44:	4288      	cmp	r0, r1
 8000e46:	f240 8085 	bls.w	8000f54 <__udivmoddi4+0x2bc>
 8000e4a:	f1a8 0802 	sub.w	r8, r8, #2
 8000e4e:	4461      	add	r1, ip
 8000e50:	1a09      	subs	r1, r1, r0
 8000e52:	b2a4      	uxth	r4, r4
 8000e54:	fbb1 f0f9 	udiv	r0, r1, r9
 8000e58:	fb09 1110 	mls	r1, r9, r0, r1
 8000e5c:	ea44 4101 	orr.w	r1, r4, r1, lsl #16
 8000e60:	fb00 fe0e 	mul.w	lr, r0, lr
 8000e64:	458e      	cmp	lr, r1
 8000e66:	d908      	bls.n	8000e7a <__udivmoddi4+0x1e2>
 8000e68:	eb1c 0101 	adds.w	r1, ip, r1
 8000e6c:	f100 34ff 	add.w	r4, r0, #4294967295
 8000e70:	d26c      	bcs.n	8000f4c <__udivmoddi4+0x2b4>
 8000e72:	458e      	cmp	lr, r1
 8000e74:	d96a      	bls.n	8000f4c <__udivmoddi4+0x2b4>
 8000e76:	3802      	subs	r0, #2
 8000e78:	4461      	add	r1, ip
 8000e7a:	ea40 4008 	orr.w	r0, r0, r8, lsl #16
 8000e7e:	fba0 9402 	umull	r9, r4, r0, r2
 8000e82:	eba1 010e 	sub.w	r1, r1, lr
 8000e86:	42a1      	cmp	r1, r4
 8000e88:	46c8      	mov	r8, r9
 8000e8a:	46a6      	mov	lr, r4
 8000e8c:	d356      	bcc.n	8000f3c <__udivmoddi4+0x2a4>
 8000e8e:	d053      	beq.n	8000f38 <__udivmoddi4+0x2a0>
 8000e90:	b15d      	cbz	r5, 8000eaa <__udivmoddi4+0x212>
 8000e92:	ebb3 0208 	subs.w	r2, r3, r8
 8000e96:	eb61 010e 	sbc.w	r1, r1, lr
 8000e9a:	fa01 f707 	lsl.w	r7, r1, r7
 8000e9e:	fa22 f306 	lsr.w	r3, r2, r6
 8000ea2:	40f1      	lsrs	r1, r6
 8000ea4:	431f      	orrs	r7, r3
 8000ea6:	e9c5 7100 	strd	r7, r1, [r5]
 8000eaa:	2600      	movs	r6, #0
 8000eac:	4631      	mov	r1, r6
 8000eae:	e8bd 87f0 	ldmia.w	sp!, {r4, r5, r6, r7, r8, r9, sl, pc}
 8000eb2:	f1c2 0320 	rsb	r3, r2, #32
 8000eb6:	40d8      	lsrs	r0, r3
 8000eb8:	fa0c fc02 	lsl.w	ip, ip, r2
 8000ebc:	fa21 f303 	lsr.w	r3, r1, r3
 8000ec0:	4091      	lsls	r1, r2
 8000ec2:	4301      	orrs	r1, r0
 8000ec4:	ea4f 471c 	mov.w	r7, ip, lsr #16
 8000ec8:	fa1f fe8c 	uxth.w	lr, ip
 8000ecc:	fbb3 f0f7 	udiv	r0, r3, r7
 8000ed0:	fb07 3610 	mls	r6, r7, r0, r3
 8000ed4:	0c0b      	lsrs	r3, r1, #16
 8000ed6:	ea43 4306 	orr.w	r3, r3, r6, lsl #16
 8000eda:	fb00 f60e 	mul.w	r6, r0, lr
 8000ede:	429e      	cmp	r6, r3
 8000ee0:	fa04 f402 	lsl.w	r4, r4, r2
 8000ee4:	d908      	bls.n	8000ef8 <__udivmoddi4+0x260>
 8000ee6:	eb1c 0303 	adds.w	r3, ip, r3
 8000eea:	f100 38ff 	add.w	r8, r0, #4294967295
 8000eee:	d22f      	bcs.n	8000f50 <__udivmoddi4+0x2b8>
 8000ef0:	429e      	cmp	r6, r3
 8000ef2:	d92d      	bls.n	8000f50 <__udivmoddi4+0x2b8>
 8000ef4:	3802      	subs	r0, #2
 8000ef6:	4463      	add	r3, ip
 8000ef8:	1b9b      	subs	r3, r3, r6
 8000efa:	b289      	uxth	r1, r1
 8000efc:	fbb3 f6f7 	udiv	r6, r3, r7
 8000f00:	fb07 3316 	mls	r3, r7, r6, r3
 8000f04:	ea41 4103 	orr.w	r1, r1, r3, lsl #16
 8000f08:	fb06 f30e 	mul.w	r3, r6, lr
 8000f0c:	428b      	cmp	r3, r1
 8000f0e:	d908      	bls.n	8000f22 <__udivmoddi4+0x28a>
 8000f10:	eb1c 0101 	adds.w	r1, ip, r1
 8000f14:	f106 38ff 	add.w	r8, r6, #4294967295
 8000f18:	d216      	bcs.n	8000f48 <__udivmoddi4+0x2b0>
 8000f1a:	428b      	cmp	r3, r1
 8000f1c:	d914      	bls.n	8000f48 <__udivmoddi4+0x2b0>
 8000f1e:	3e02      	subs	r6, #2
 8000f20:	4461      	add	r1, ip
 8000f22:	1ac9      	subs	r1, r1, r3
 8000f24:	ea46 4600 	orr.w	r6, r6, r0, lsl #16
 8000f28:	e738      	b.n	8000d9c <__udivmoddi4+0x104>
 8000f2a:	462e      	mov	r6, r5
 8000f2c:	4628      	mov	r0, r5
 8000f2e:	e705      	b.n	8000d3c <__udivmoddi4+0xa4>
 8000f30:	4606      	mov	r6, r0
 8000f32:	e6e3      	b.n	8000cfc <__udivmoddi4+0x64>
 8000f34:	4618      	mov	r0, r3
 8000f36:	e6f8      	b.n	8000d2a <__udivmoddi4+0x92>
 8000f38:	454b      	cmp	r3, r9
 8000f3a:	d2a9      	bcs.n	8000e90 <__udivmoddi4+0x1f8>
 8000f3c:	ebb9 0802 	subs.w	r8, r9, r2
 8000f40:	eb64 0e0c 	sbc.w	lr, r4, ip
 8000f44:	3801      	subs	r0, #1
 8000f46:	e7a3      	b.n	8000e90 <__udivmoddi4+0x1f8>
 8000f48:	4646      	mov	r6, r8
 8000f4a:	e7ea      	b.n	8000f22 <__udivmoddi4+0x28a>
 8000f4c:	4620      	mov	r0, r4
 8000f4e:	e794      	b.n	8000e7a <__udivmoddi4+0x1e2>
 8000f50:	4640      	mov	r0, r8
 8000f52:	e7d1      	b.n	8000ef8 <__udivmoddi4+0x260>
 8000f54:	46d0      	mov	r8, sl
 8000f56:	e77b      	b.n	8000e50 <__udivmoddi4+0x1b8>
 8000f58:	3b02      	subs	r3, #2
 8000f5a:	4461      	add	r1, ip
 8000f5c:	e732      	b.n	8000dc4 <__udivmoddi4+0x12c>
 8000f5e:	4630      	mov	r0, r6
 8000f60:	e709      	b.n	8000d76 <__udivmoddi4+0xde>
 8000f62:	4464      	add	r4, ip
 8000f64:	3802      	subs	r0, #2
 8000f66:	e742      	b.n	8000dee <__udivmoddi4+0x156>

08000f68 <__aeabi_idiv0>:
 8000f68:	4770      	bx	lr
 8000f6a:	bf00      	nop

08000f6c <main>:
static void MX_GPIO_Init(void);
static void MX_SPI1_Init(void);
static void MX_USART1_UART_Init(void);


int main(void) {
 8000f6c:	b5b0      	push	{r4, r5, r7, lr}
 8000f6e:	b0c8      	sub	sp, #288	; 0x120
 8000f70:	af00      	add	r7, sp, #0

/* MCU Configuration--------------------------------------------------------*/
/* Reset of all peripherals, Initializes the Flash interface and the Systick. */
HAL_Init();
 8000f72:	f000 fdeb 	bl	8001b4c <HAL_Init>

/* Configure the system clock */
SystemClock_Config();
 8000f76:	f000 fabd 	bl	80014f4 <SystemClock_Config>

/* Initialize all configured peripherals */
MX_GPIO_Init();
 8000f7a:	f000 fb87 	bl	800168c <MX_GPIO_Init>
MX_SPI1_Init();
 8000f7e:	f000 fb25 	bl	80015cc <MX_SPI1_Init>
MX_USART1_UART_Init();
 8000f82:	f000 fb59 	bl	8001638 <MX_USART1_UART_Init>

/* USER CODE BEGIN 2 */


/////////////////////////////////////// Variables //////////////////////////////////////////////
uint8_t spi_tx_data_reg = 0x00, i = 0;
 8000f86:	2300      	movs	r3, #0
 8000f88:	f887 30f0 	strb.w	r3, [r7, #240]	; 0xf0
 8000f8c:	2300      	movs	r3, #0
 8000f8e:	f887 311f 	strb.w	r3, [r7, #287]	; 0x11f
uint8_t spi_rx_data[6] = { 0x00 };
 8000f92:	2300      	movs	r3, #0
 8000f94:	f8c7 30e8 	str.w	r3, [r7, #232]	; 0xe8
 8000f98:	2300      	movs	r3, #0
 8000f9a:	f8a7 30ec 	strh.w	r3, [r7, #236]	; 0xec
uint8_t bmp280_Calib_data[5] = { 0x00 };
 8000f9e:	2300      	movs	r3, #0
 8000fa0:	f8c7 30e0 	str.w	r3, [r7, #224]	; 0xe0
 8000fa4:	2300      	movs	r3, #0
 8000fa6:	f887 30e4 	strb.w	r3, [r7, #228]	; 0xe4
int8_t ctrl_meas_bits = 0x00;
 8000faa:	2300      	movs	r3, #0
 8000fac:	f887 3113 	strb.w	r3, [r7, #275]	; 0x113
int32_t raw_temperature = 0;
 8000fb0:	2300      	movs	r3, #0
 8000fb2:	f8c7 310c 	str.w	r3, [r7, #268]	; 0x10c

float temp_degr = 0;
 8000fb6:	f04f 0300 	mov.w	r3, #0
 8000fba:	f8c7 3108 	str.w	r3, [r7, #264]	; 0x108
double var1 = 0;
 8000fbe:	f04f 0200 	mov.w	r2, #0
 8000fc2:	f04f 0300 	mov.w	r3, #0
 8000fc6:	e9c7 2340 	strd	r2, r3, [r7, #256]	; 0x100
double var2 = 0;
 8000fca:	f04f 0200 	mov.w	r2, #0
 8000fce:	f04f 0300 	mov.w	r3, #0
 8000fd2:	e9c7 233e 	strd	r2, r3, [r7, #248]	; 0xf8

char temp_char_num [5];
char skip[] = "\r\n";
 8000fd6:	4aae      	ldr	r2, [pc, #696]	; (8001290 <main+0x324>)
 8000fd8:	f107 03d4 	add.w	r3, r7, #212	; 0xd4
 8000fdc:	6812      	ldr	r2, [r2, #0]
 8000fde:	4611      	mov	r1, r2
 8000fe0:	8019      	strh	r1, [r3, #0]
 8000fe2:	3302      	adds	r3, #2
 8000fe4:	0c12      	lsrs	r2, r2, #16
 8000fe6:	701a      	strb	r2, [r3, #0]
char MGS_star[] = {"Temperature Control system \r\n"};
 8000fe8:	4baa      	ldr	r3, [pc, #680]	; (8001294 <main+0x328>)
 8000fea:	f107 04b4 	add.w	r4, r7, #180	; 0xb4
 8000fee:	461d      	mov	r5, r3
 8000ff0:	cd0f      	ldmia	r5!, {r0, r1, r2, r3}
 8000ff2:	c40f      	stmia	r4!, {r0, r1, r2, r3}
 8000ff4:	e895 000f 	ldmia.w	r5, {r0, r1, r2, r3}
 8000ff8:	c407      	stmia	r4!, {r0, r1, r2}
 8000ffa:	8023      	strh	r3, [r4, #0]
char MGS_parse_CMD[] = {"Put: F to start the temperature measurement or E to stop the temperature measurement\r\n"};
 8000ffc:	4aa6      	ldr	r2, [pc, #664]	; (8001298 <main+0x32c>)
 8000ffe:	f107 035c 	add.w	r3, r7, #92	; 0x5c
 8001002:	4611      	mov	r1, r2
 8001004:	2257      	movs	r2, #87	; 0x57
 8001006:	4618      	mov	r0, r3
 8001008:	f002 ffb0 	bl	8003f6c <memcpy>
char MGS_Meas[]= {"The temperature is: \r\n"};
 800100c:	4ba3      	ldr	r3, [pc, #652]	; (800129c <main+0x330>)
 800100e:	f107 0444 	add.w	r4, r7, #68	; 0x44
 8001012:	461d      	mov	r5, r3
 8001014:	cd0f      	ldmia	r5!, {r0, r1, r2, r3}
 8001016:	c40f      	stmia	r4!, {r0, r1, r2, r3}
 8001018:	e895 0003 	ldmia.w	r5, {r0, r1}
 800101c:	6020      	str	r0, [r4, #0]
 800101e:	3404      	adds	r4, #4
 8001020:	8021      	strh	r1, [r4, #0]
 8001022:	3402      	adds	r4, #2
 8001024:	0c0b      	lsrs	r3, r1, #16
 8001026:	7023      	strb	r3, [r4, #0]
char MGS_stop[]= {"The temperature measurement is stop\r\n"};
 8001028:	f507 7390 	add.w	r3, r7, #288	; 0x120
 800102c:	f5a3 7382 	sub.w	r3, r3, #260	; 0x104
 8001030:	4a9b      	ldr	r2, [pc, #620]	; (80012a0 <main+0x334>)
 8001032:	461c      	mov	r4, r3
 8001034:	4615      	mov	r5, r2
 8001036:	cd0f      	ldmia	r5!, {r0, r1, r2, r3}
 8001038:	c40f      	stmia	r4!, {r0, r1, r2, r3}
 800103a:	cd0f      	ldmia	r5!, {r0, r1, r2, r3}
 800103c:	c40f      	stmia	r4!, {r0, r1, r2, r3}
 800103e:	e895 0003 	ldmia.w	r5, {r0, r1}
 8001042:	6020      	str	r0, [r4, #0]
 8001044:	3404      	adds	r4, #4
 8001046:	8021      	strh	r1, [r4, #0]
char MGS_Alert[]= {"High Temperature: \r\n"};
 8001048:	f507 7390 	add.w	r3, r7, #288	; 0x120
 800104c:	f5a3 738e 	sub.w	r3, r3, #284	; 0x11c
 8001050:	4a94      	ldr	r2, [pc, #592]	; (80012a4 <main+0x338>)
 8001052:	461c      	mov	r4, r3
 8001054:	4615      	mov	r5, r2
 8001056:	cd0f      	ldmia	r5!, {r0, r1, r2, r3}
 8001058:	c40f      	stmia	r4!, {r0, r1, r2, r3}
 800105a:	e895 0003 	ldmia.w	r5, {r0, r1}
 800105e:	6020      	str	r0, [r4, #0]
 8001060:	3404      	adds	r4, #4
 8001062:	7021      	strb	r1, [r4, #0]

uint16_t dig_T1 = 0b0110100110100011;
 8001064:	f646 13a3 	movw	r3, #27043	; 0x69a3
 8001068:	f8a7 30f6 	strh.w	r3, [r7, #246]	; 0xf6
int16_t dig_T2 = 0b0110101001000000;
 800106c:	f646 2340 	movw	r3, #27200	; 0x6a40
 8001070:	f8a7 30f4 	strh.w	r3, [r7, #244]	; 0xf4
int16_t dig_T3 = 0b1111110000011000;
 8001074:	f64f 4318 	movw	r3, #64536	; 0xfc18
 8001078:	f8a7 30f2 	strh.w	r3, [r7, #242]	; 0xf2

uint8_t rx_data = 0;
 800107c:	f507 7390 	add.w	r3, r7, #288	; 0x120
 8001080:	f2a3 131d 	subw	r3, r3, #285	; 0x11d
 8001084:	2200      	movs	r2, #0
 8001086:	701a      	strb	r2, [r3, #0]
uint8_t toogle_meas_enable = 0;
 8001088:	2300      	movs	r3, #0
 800108a:	f887 311e 	strb.w	r3, [r7, #286]	; 0x11e
uint32_t toggle_period_ms = 0;
 800108e:	2300      	movs	r3, #0
 8001090:	f8c7 3118 	str.w	r3, [r7, #280]	; 0x118
uint32_t meas_tick = 0;
 8001094:	2300      	movs	r3, #0
 8001096:	f8c7 3114 	str.w	r3, [r7, #276]	; 0x114

///////////////////////////////////////// Configuration of the BMP280 temperature sensor ///////////////////////////////
// Search the sensor ID
spi_tx_data_reg = BMP280_REG_ADDR_ID;
 800109a:	23d0      	movs	r3, #208	; 0xd0
 800109c:	f887 30f0 	strb.w	r3, [r7, #240]	; 0xf0
HAL_GPIO_WritePin(bmp280_CS_GPIO_Port, bmp280_CS_Pin, GPIO_PIN_RESET);
 80010a0:	2200      	movs	r2, #0
 80010a2:	2110      	movs	r1, #16
 80010a4:	4880      	ldr	r0, [pc, #512]	; (80012a8 <main+0x33c>)
 80010a6:	f001 f879 	bl	800219c <HAL_GPIO_WritePin>
if (HAL_SPI_Transmit(&hspi1, &spi_tx_data_reg, 1, 100) == HAL_OK) {
 80010aa:	f107 01f0 	add.w	r1, r7, #240	; 0xf0
 80010ae:	2364      	movs	r3, #100	; 0x64
 80010b0:	2201      	movs	r2, #1
 80010b2:	487e      	ldr	r0, [pc, #504]	; (80012ac <main+0x340>)
 80010b4:	f001 fdad 	bl	8002c12 <HAL_SPI_Transmit>
 80010b8:	4603      	mov	r3, r0
 80010ba:	2b00      	cmp	r3, #0
 80010bc:	d10c      	bne.n	80010d8 <main+0x16c>
	if (HAL_SPI_Receive(&hspi1, spi_rx_data, 1, 100) == HAL_OK) {
 80010be:	f107 01e8 	add.w	r1, r7, #232	; 0xe8
 80010c2:	2364      	movs	r3, #100	; 0x64
 80010c4:	2201      	movs	r2, #1
 80010c6:	4879      	ldr	r0, [pc, #484]	; (80012ac <main+0x340>)
 80010c8:	f001 fedf 	bl	8002e8a <HAL_SPI_Receive>
 80010cc:	4603      	mov	r3, r0
 80010ce:	2b00      	cmp	r3, #0
 80010d0:	d102      	bne.n	80010d8 <main+0x16c>
		HAL_Delay(100);
 80010d2:	2064      	movs	r0, #100	; 0x64
 80010d4:	f000 fdac 	bl	8001c30 <HAL_Delay>
	}
}
HAL_GPIO_WritePin(bmp280_CS_GPIO_Port, bmp280_CS_Pin, GPIO_PIN_SET);
 80010d8:	2201      	movs	r2, #1
 80010da:	2110      	movs	r1, #16
 80010dc:	4872      	ldr	r0, [pc, #456]	; (80012a8 <main+0x33c>)
 80010de:	f001 f85d 	bl	800219c <HAL_GPIO_WritePin>

// Change the Config sensor (temp over samp x2, skipped the press meas, normal power mode)
uint8_t ctrl_meas_Bytes = 0x23;
 80010e2:	2323      	movs	r3, #35	; 0x23
 80010e4:	f887 30f1 	strb.w	r3, [r7, #241]	; 0xf1
uint8_t spi_config[2] = { 0x74, ctrl_meas_Bytes };
 80010e8:	f507 7390 	add.w	r3, r7, #288	; 0x120
 80010ec:	f5a3 7390 	sub.w	r3, r3, #288	; 0x120
 80010f0:	2274      	movs	r2, #116	; 0x74
 80010f2:	701a      	strb	r2, [r3, #0]
 80010f4:	f507 7390 	add.w	r3, r7, #288	; 0x120
 80010f8:	f5a3 7390 	sub.w	r3, r3, #288	; 0x120
 80010fc:	f897 20f1 	ldrb.w	r2, [r7, #241]	; 0xf1
 8001100:	705a      	strb	r2, [r3, #1]

HAL_GPIO_WritePin(bmp280_CS_GPIO_Port, bmp280_CS_Pin, GPIO_PIN_RESET);
 8001102:	2200      	movs	r2, #0
 8001104:	2110      	movs	r1, #16
 8001106:	4868      	ldr	r0, [pc, #416]	; (80012a8 <main+0x33c>)
 8001108:	f001 f848 	bl	800219c <HAL_GPIO_WritePin>
if (HAL_SPI_Transmit(&hspi1, spi_config, 2, 100) == HAL_OK) {
 800110c:	4639      	mov	r1, r7
 800110e:	2364      	movs	r3, #100	; 0x64
 8001110:	2202      	movs	r2, #2
 8001112:	4866      	ldr	r0, [pc, #408]	; (80012ac <main+0x340>)
 8001114:	f001 fd7d 	bl	8002c12 <HAL_SPI_Transmit>
 8001118:	4603      	mov	r3, r0
 800111a:	2b00      	cmp	r3, #0
 800111c:	d102      	bne.n	8001124 <main+0x1b8>
	HAL_Delay(100);
 800111e:	2064      	movs	r0, #100	; 0x64
 8001120:	f000 fd86 	bl	8001c30 <HAL_Delay>
}
HAL_GPIO_WritePin(bmp280_CS_GPIO_Port, bmp280_CS_Pin, GPIO_PIN_SET);
 8001124:	2201      	movs	r2, #1
 8001126:	2110      	movs	r1, #16
 8001128:	485f      	ldr	r0, [pc, #380]	; (80012a8 <main+0x33c>)
 800112a:	f001 f837 	bl	800219c <HAL_GPIO_WritePin>

// Verify the CTRL_MEAS register configuration
spi_tx_data_reg = BMP280_REG_ADDR_CTRL_MEAS;
 800112e:	23f4      	movs	r3, #244	; 0xf4
 8001130:	f887 30f0 	strb.w	r3, [r7, #240]	; 0xf0
HAL_GPIO_WritePin(bmp280_CS_GPIO_Port, bmp280_CS_Pin, GPIO_PIN_RESET);
 8001134:	2200      	movs	r2, #0
 8001136:	2110      	movs	r1, #16
 8001138:	485b      	ldr	r0, [pc, #364]	; (80012a8 <main+0x33c>)
 800113a:	f001 f82f 	bl	800219c <HAL_GPIO_WritePin>
if (HAL_SPI_Transmit(&hspi1, &spi_tx_data_reg, 1, 100) == HAL_OK) {
 800113e:	f107 01f0 	add.w	r1, r7, #240	; 0xf0
 8001142:	2364      	movs	r3, #100	; 0x64
 8001144:	2201      	movs	r2, #1
 8001146:	4859      	ldr	r0, [pc, #356]	; (80012ac <main+0x340>)
 8001148:	f001 fd63 	bl	8002c12 <HAL_SPI_Transmit>
 800114c:	4603      	mov	r3, r0
 800114e:	2b00      	cmp	r3, #0
 8001150:	d10c      	bne.n	800116c <main+0x200>
	if (HAL_SPI_Receive(&hspi1, spi_rx_data, 1, 100) == HAL_OK) {
 8001152:	f107 01e8 	add.w	r1, r7, #232	; 0xe8
 8001156:	2364      	movs	r3, #100	; 0x64
 8001158:	2201      	movs	r2, #1
 800115a:	4854      	ldr	r0, [pc, #336]	; (80012ac <main+0x340>)
 800115c:	f001 fe95 	bl	8002e8a <HAL_SPI_Receive>
 8001160:	4603      	mov	r3, r0
 8001162:	2b00      	cmp	r3, #0
 8001164:	d102      	bne.n	800116c <main+0x200>
		HAL_Delay(100);
 8001166:	2064      	movs	r0, #100	; 0x64
 8001168:	f000 fd62 	bl	8001c30 <HAL_Delay>
	}

}
HAL_GPIO_WritePin(bmp280_CS_GPIO_Port, bmp280_CS_Pin, GPIO_PIN_SET);
 800116c:	2201      	movs	r2, #1
 800116e:	2110      	movs	r1, #16
 8001170:	484d      	ldr	r0, [pc, #308]	; (80012a8 <main+0x33c>)
 8001172:	f001 f813 	bl	800219c <HAL_GPIO_WritePin>
HAL_Delay(100);
 8001176:	2064      	movs	r0, #100	; 0x64
 8001178:	f000 fd5a 	bl	8001c30 <HAL_Delay>

// Extraction of dig_T1, dig_T2 and dig_T3
HAL_GPIO_WritePin(bmp280_CS_GPIO_Port, bmp280_CS_Pin, GPIO_PIN_RESET);
 800117c:	2200      	movs	r2, #0
 800117e:	2110      	movs	r1, #16
 8001180:	4849      	ldr	r0, [pc, #292]	; (80012a8 <main+0x33c>)
 8001182:	f001 f80b 	bl	800219c <HAL_GPIO_WritePin>
for (i=0; i < 6; i++) {
 8001186:	2300      	movs	r3, #0
 8001188:	f887 311f 	strb.w	r3, [r7, #287]	; 0x11f
 800118c:	e02d      	b.n	80011ea <main+0x27e>
	spi_tx_data_reg = BMP280_REG_ADDR_CAL_START_ADDR + i;
 800118e:	f897 311f 	ldrb.w	r3, [r7, #287]	; 0x11f
 8001192:	3b78      	subs	r3, #120	; 0x78
 8001194:	b2db      	uxtb	r3, r3
 8001196:	f887 30f0 	strb.w	r3, [r7, #240]	; 0xf0
	if (HAL_SPI_Transmit(&hspi1, &spi_tx_data_reg, 1, 100) == HAL_OK) {
 800119a:	f107 01f0 	add.w	r1, r7, #240	; 0xf0
 800119e:	2364      	movs	r3, #100	; 0x64
 80011a0:	2201      	movs	r2, #1
 80011a2:	4842      	ldr	r0, [pc, #264]	; (80012ac <main+0x340>)
 80011a4:	f001 fd35 	bl	8002c12 <HAL_SPI_Transmit>
 80011a8:	4603      	mov	r3, r0
 80011aa:	2b00      	cmp	r3, #0
 80011ac:	d115      	bne.n	80011da <main+0x26e>
		if (HAL_SPI_Receive(&hspi1, spi_rx_data, 1, 100) == HAL_OK) {
 80011ae:	f107 01e8 	add.w	r1, r7, #232	; 0xe8
 80011b2:	2364      	movs	r3, #100	; 0x64
 80011b4:	2201      	movs	r2, #1
 80011b6:	483d      	ldr	r0, [pc, #244]	; (80012ac <main+0x340>)
 80011b8:	f001 fe67 	bl	8002e8a <HAL_SPI_Receive>
 80011bc:	4603      	mov	r3, r0
 80011be:	2b00      	cmp	r3, #0
 80011c0:	d10b      	bne.n	80011da <main+0x26e>
			HAL_Delay(100);
 80011c2:	2064      	movs	r0, #100	; 0x64
 80011c4:	f000 fd34 	bl	8001c30 <HAL_Delay>
			bmp280_Calib_data[i] = spi_rx_data[0];
 80011c8:	f897 311f 	ldrb.w	r3, [r7, #287]	; 0x11f
 80011cc:	f897 20e8 	ldrb.w	r2, [r7, #232]	; 0xe8
 80011d0:	f503 7390 	add.w	r3, r3, #288	; 0x120
 80011d4:	443b      	add	r3, r7
 80011d6:	f803 2c40 	strb.w	r2, [r3, #-64]
		}
	}
	HAL_Delay(100);
 80011da:	2064      	movs	r0, #100	; 0x64
 80011dc:	f000 fd28 	bl	8001c30 <HAL_Delay>
for (i=0; i < 6; i++) {
 80011e0:	f897 311f 	ldrb.w	r3, [r7, #287]	; 0x11f
 80011e4:	3301      	adds	r3, #1
 80011e6:	f887 311f 	strb.w	r3, [r7, #287]	; 0x11f
 80011ea:	f897 311f 	ldrb.w	r3, [r7, #287]	; 0x11f
 80011ee:	2b05      	cmp	r3, #5
 80011f0:	d9cd      	bls.n	800118e <main+0x222>
}
HAL_GPIO_WritePin(bmp280_CS_GPIO_Port, bmp280_CS_Pin, GPIO_PIN_SET);
 80011f2:	2201      	movs	r2, #1
 80011f4:	2110      	movs	r1, #16
 80011f6:	482c      	ldr	r0, [pc, #176]	; (80012a8 <main+0x33c>)
 80011f8:	f000 ffd0 	bl	800219c <HAL_GPIO_WritePin>

/////////////////////////////////Send Startup message ///////////////////////////////////////////
HAL_UART_Transmit(&huart1,MGS_star,sizeof(MGS_star)-1, 500);
 80011fc:	f107 01b4 	add.w	r1, r7, #180	; 0xb4
 8001200:	f44f 73fa 	mov.w	r3, #500	; 0x1f4
 8001204:	221d      	movs	r2, #29
 8001206:	482a      	ldr	r0, [pc, #168]	; (80012b0 <main+0x344>)
 8001208:	f002 fa6f 	bl	80036ea <HAL_UART_Transmit>

/////////////////////////////////Send instruction message fot the parse command/////////////////
HAL_UART_Transmit(&huart1,MGS_parse_CMD,sizeof(MGS_parse_CMD)-1, 500);
 800120c:	f107 015c 	add.w	r1, r7, #92	; 0x5c
 8001210:	f44f 73fa 	mov.w	r3, #500	; 0x1f4
 8001214:	2256      	movs	r2, #86	; 0x56
 8001216:	4826      	ldr	r0, [pc, #152]	; (80012b0 <main+0x344>)
 8001218:	f002 fa67 	bl	80036ea <HAL_UART_Transmit>
/* Infinite loop */
/* USER CODE BEGIN WHILE */
while (1) {

	/* USER CODE END WHILE */
	if (HAL_UART_Receive(&huart1, &rx_data, 1, 500) == HAL_OK) {   // Wait for the letter command
 800121c:	1cf9      	adds	r1, r7, #3
 800121e:	f44f 73fa 	mov.w	r3, #500	; 0x1f4
 8001222:	2201      	movs	r2, #1
 8001224:	4822      	ldr	r0, [pc, #136]	; (80012b0 <main+0x344>)
 8001226:	f002 faf2 	bl	800380e <HAL_UART_Receive>
 800122a:	4603      	mov	r3, r0
 800122c:	2b00      	cmp	r3, #0
 800122e:	d143      	bne.n	80012b8 <main+0x34c>


		// Parse the command
		switch (rx_data) {
 8001230:	f507 7390 	add.w	r3, r7, #288	; 0x120
 8001234:	f2a3 131d 	subw	r3, r3, #285	; 0x11d
 8001238:	781b      	ldrb	r3, [r3, #0]
 800123a:	2b45      	cmp	r3, #69	; 0x45
 800123c:	d002      	beq.n	8001244 <main+0x2d8>
 800123e:	2b46      	cmp	r3, #70	; 0x46
 8001240:	d015      	beq.n	800126e <main+0x302>
			toggle_period_ms = 1000;										// Set the measurement period
			break;

		default:
			// the command was ignored
			break;
 8001242:	e03a      	b.n	80012ba <main+0x34e>
			HAL_UART_Transmit(&huart1,MGS_stop,sizeof(MGS_stop)-1, 500);	// Send Stop message
 8001244:	f107 011c 	add.w	r1, r7, #28
 8001248:	f44f 73fa 	mov.w	r3, #500	; 0x1f4
 800124c:	2225      	movs	r2, #37	; 0x25
 800124e:	4818      	ldr	r0, [pc, #96]	; (80012b0 <main+0x344>)
 8001250:	f002 fa4b 	bl	80036ea <HAL_UART_Transmit>
			toogle_meas_enable = 0;											// disable the temperature measurement
 8001254:	2300      	movs	r3, #0
 8001256:	f887 311e 	strb.w	r3, [r7, #286]	; 0x11e
			HAL_GPIO_WritePin(LED_4_GPIO_Port, LED_4_Pin, GPIO_PIN_RESET);	// Put the LED OFF
 800125a:	2200      	movs	r2, #0
 800125c:	f44f 4180 	mov.w	r1, #16384	; 0x4000
 8001260:	4814      	ldr	r0, [pc, #80]	; (80012b4 <main+0x348>)
 8001262:	f000 ff9b 	bl	800219c <HAL_GPIO_WritePin>
			HAL_Delay(100);
 8001266:	2064      	movs	r0, #100	; 0x64
 8001268:	f000 fce2 	bl	8001c30 <HAL_Delay>
			break;
 800126c:	e025      	b.n	80012ba <main+0x34e>
			HAL_UART_Transmit(&huart1,MGS_Meas,sizeof(MGS_Meas)-1, 500);	// Send the temperature message
 800126e:	f107 0144 	add.w	r1, r7, #68	; 0x44
 8001272:	f44f 73fa 	mov.w	r3, #500	; 0x1f4
 8001276:	2216      	movs	r2, #22
 8001278:	480d      	ldr	r0, [pc, #52]	; (80012b0 <main+0x344>)
 800127a:	f002 fa36 	bl	80036ea <HAL_UART_Transmit>
			toogle_meas_enable = 1;											// Enable the temperature measurement
 800127e:	2301      	movs	r3, #1
 8001280:	f887 311e 	strb.w	r3, [r7, #286]	; 0x11e
			toggle_period_ms = 1000;										// Set the measurement period
 8001284:	f44f 737a 	mov.w	r3, #1000	; 0x3e8
 8001288:	f8c7 3118 	str.w	r3, [r7, #280]	; 0x118
			break;
 800128c:	e015      	b.n	80012ba <main+0x34e>
 800128e:	bf00      	nop
 8001290:	08006d64 	.word	0x08006d64
 8001294:	08006d68 	.word	0x08006d68
 8001298:	08006d88 	.word	0x08006d88
 800129c:	08006de0 	.word	0x08006de0
 80012a0:	08006df8 	.word	0x08006df8
 80012a4:	08006e20 	.word	0x08006e20
 80012a8:	40020800 	.word	0x40020800
 80012ac:	200001f8 	.word	0x200001f8
 80012b0:	20000250 	.word	0x20000250
 80012b4:	40021800 	.word	0x40021800
		}
	}
 80012b8:	bf00      	nop

	if (toogle_meas_enable) {
 80012ba:	f897 311e 	ldrb.w	r3, [r7, #286]	; 0x11e
 80012be:	2b00      	cmp	r3, #0
 80012c0:	d0ac      	beq.n	800121c <main+0x2b0>
		if ((HAL_GetTick() - meas_tick) > toggle_period_ms) {    //temperature measurement
 80012c2:	f000 fca9 	bl	8001c18 <HAL_GetTick>
 80012c6:	4602      	mov	r2, r0
 80012c8:	f8d7 3114 	ldr.w	r3, [r7, #276]	; 0x114
 80012cc:	1ad3      	subs	r3, r2, r3
 80012ce:	f8d7 2118 	ldr.w	r2, [r7, #280]	; 0x118
 80012d2:	429a      	cmp	r2, r3
 80012d4:	d2a2      	bcs.n	800121c <main+0x2b0>
			meas_tick = HAL_GetTick();							 // Evaluate the period
 80012d6:	f000 fc9f 	bl	8001c18 <HAL_GetTick>
 80012da:	f8c7 0114 	str.w	r0, [r7, #276]	; 0x114

///////////////// Take the temperature measurement /////////////////////////////////////////
			spi_tx_data_reg = BMP280_REG_ADDR_TEMP_MSB;
 80012de:	23fa      	movs	r3, #250	; 0xfa
 80012e0:	f887 30f0 	strb.w	r3, [r7, #240]	; 0xf0
			HAL_GPIO_WritePin(bmp280_CS_GPIO_Port, bmp280_CS_Pin,
 80012e4:	2200      	movs	r2, #0
 80012e6:	2110      	movs	r1, #16
 80012e8:	4878      	ldr	r0, [pc, #480]	; (80014cc <main+0x560>)
 80012ea:	f000 ff57 	bl	800219c <HAL_GPIO_WritePin>
					GPIO_PIN_RESET);
			if (HAL_SPI_Transmit(&hspi1, &spi_tx_data_reg, 1, 100)
 80012ee:	f107 01f0 	add.w	r1, r7, #240	; 0xf0
 80012f2:	2364      	movs	r3, #100	; 0x64
 80012f4:	2201      	movs	r2, #1
 80012f6:	4876      	ldr	r0, [pc, #472]	; (80014d0 <main+0x564>)
 80012f8:	f001 fc8b 	bl	8002c12 <HAL_SPI_Transmit>
 80012fc:	4603      	mov	r3, r0
 80012fe:	2b00      	cmp	r3, #0
 8001300:	f040 80db 	bne.w	80014ba <main+0x54e>
					== HAL_OK) {
				if (HAL_SPI_Receive(&hspi1, spi_rx_data, 1, 100)
 8001304:	f107 01e8 	add.w	r1, r7, #232	; 0xe8
 8001308:	2364      	movs	r3, #100	; 0x64
 800130a:	2201      	movs	r2, #1
 800130c:	4870      	ldr	r0, [pc, #448]	; (80014d0 <main+0x564>)
 800130e:	f001 fdbc 	bl	8002e8a <HAL_SPI_Receive>
 8001312:	4603      	mov	r3, r0
 8001314:	2b00      	cmp	r3, #0
 8001316:	f040 80d0 	bne.w	80014ba <main+0x54e>
						== HAL_OK) {
					HAL_Delay(100);
 800131a:	2064      	movs	r0, #100	; 0x64
 800131c:	f000 fc88 	bl	8001c30 <HAL_Delay>
					raw_temperature =
							(int32_t) (spi_rx_data[2] & 0b00001111)
 8001320:	f897 30ea 	ldrb.w	r3, [r7, #234]	; 0xea
 8001324:	f003 020f 	and.w	r2, r3, #15
									| (spi_rx_data[1] << 4)
 8001328:	f897 30e9 	ldrb.w	r3, [r7, #233]	; 0xe9
 800132c:	011b      	lsls	r3, r3, #4
 800132e:	431a      	orrs	r2, r3
									| (spi_rx_data[0] << 12);
 8001330:	f897 30e8 	ldrb.w	r3, [r7, #232]	; 0xe8
 8001334:	031b      	lsls	r3, r3, #12
					raw_temperature =
 8001336:	4313      	orrs	r3, r2
 8001338:	f8c7 310c 	str.w	r3, [r7, #268]	; 0x10c



					var1 = (((double) raw_temperature) / 16384.0
 800133c:	f8d7 010c 	ldr.w	r0, [r7, #268]	; 0x10c
 8001340:	f7ff f900 	bl	8000544 <__aeabi_i2d>
 8001344:	f04f 0200 	mov.w	r2, #0
 8001348:	4b62      	ldr	r3, [pc, #392]	; (80014d4 <main+0x568>)
 800134a:	f7ff fa8f 	bl	800086c <__aeabi_ddiv>
 800134e:	4602      	mov	r2, r0
 8001350:	460b      	mov	r3, r1
 8001352:	4614      	mov	r4, r2
 8001354:	461d      	mov	r5, r3
							- ((double) dig_T1) / 1024.0)
 8001356:	f8b7 30f6 	ldrh.w	r3, [r7, #246]	; 0xf6
 800135a:	4618      	mov	r0, r3
 800135c:	f7ff f8e2 	bl	8000524 <__aeabi_ui2d>
 8001360:	f04f 0200 	mov.w	r2, #0
 8001364:	4b5c      	ldr	r3, [pc, #368]	; (80014d8 <main+0x56c>)
 8001366:	f7ff fa81 	bl	800086c <__aeabi_ddiv>
 800136a:	4602      	mov	r2, r0
 800136c:	460b      	mov	r3, r1
 800136e:	4620      	mov	r0, r4
 8001370:	4629      	mov	r1, r5
 8001372:	f7fe ff99 	bl	80002a8 <__aeabi_dsub>
 8001376:	4602      	mov	r2, r0
 8001378:	460b      	mov	r3, r1
 800137a:	4614      	mov	r4, r2
 800137c:	461d      	mov	r5, r3
							* ((double) dig_T2);
 800137e:	f9b7 30f4 	ldrsh.w	r3, [r7, #244]	; 0xf4
 8001382:	4618      	mov	r0, r3
 8001384:	f7ff f8de 	bl	8000544 <__aeabi_i2d>
 8001388:	4602      	mov	r2, r0
 800138a:	460b      	mov	r3, r1
					var1 = (((double) raw_temperature) / 16384.0
 800138c:	4620      	mov	r0, r4
 800138e:	4629      	mov	r1, r5
 8001390:	f7ff f942 	bl	8000618 <__aeabi_dmul>
 8001394:	4602      	mov	r2, r0
 8001396:	460b      	mov	r3, r1
 8001398:	e9c7 2340 	strd	r2, r3, [r7, #256]	; 0x100

					var2 = ((double) raw_temperature) / 131072.0
 800139c:	f8d7 010c 	ldr.w	r0, [r7, #268]	; 0x10c
 80013a0:	f7ff f8d0 	bl	8000544 <__aeabi_i2d>
 80013a4:	f04f 0200 	mov.w	r2, #0
 80013a8:	f04f 4382 	mov.w	r3, #1090519040	; 0x41000000
 80013ac:	f7ff fa5e 	bl	800086c <__aeabi_ddiv>
 80013b0:	4602      	mov	r2, r0
 80013b2:	460b      	mov	r3, r1
 80013b4:	4614      	mov	r4, r2
 80013b6:	461d      	mov	r5, r3
							- ((double) dig_T1) / 8192.0;
 80013b8:	f8b7 30f6 	ldrh.w	r3, [r7, #246]	; 0xf6
 80013bc:	4618      	mov	r0, r3
 80013be:	f7ff f8b1 	bl	8000524 <__aeabi_ui2d>
 80013c2:	f04f 0200 	mov.w	r2, #0
 80013c6:	4b45      	ldr	r3, [pc, #276]	; (80014dc <main+0x570>)
 80013c8:	f7ff fa50 	bl	800086c <__aeabi_ddiv>
 80013cc:	4602      	mov	r2, r0
 80013ce:	460b      	mov	r3, r1
					var2 = ((double) raw_temperature) / 131072.0
 80013d0:	4620      	mov	r0, r4
 80013d2:	4629      	mov	r1, r5
 80013d4:	f7fe ff68 	bl	80002a8 <__aeabi_dsub>
 80013d8:	4602      	mov	r2, r0
 80013da:	460b      	mov	r3, r1
 80013dc:	e9c7 233e 	strd	r2, r3, [r7, #248]	; 0xf8

					var2 = (var2 * var2) * ((double) dig_T3);
 80013e0:	e9d7 233e 	ldrd	r2, r3, [r7, #248]	; 0xf8
 80013e4:	e9d7 013e 	ldrd	r0, r1, [r7, #248]	; 0xf8
 80013e8:	f7ff f916 	bl	8000618 <__aeabi_dmul>
 80013ec:	4602      	mov	r2, r0
 80013ee:	460b      	mov	r3, r1
 80013f0:	4614      	mov	r4, r2
 80013f2:	461d      	mov	r5, r3
 80013f4:	f9b7 30f2 	ldrsh.w	r3, [r7, #242]	; 0xf2
 80013f8:	4618      	mov	r0, r3
 80013fa:	f7ff f8a3 	bl	8000544 <__aeabi_i2d>
 80013fe:	4602      	mov	r2, r0
 8001400:	460b      	mov	r3, r1
 8001402:	4620      	mov	r0, r4
 8001404:	4629      	mov	r1, r5
 8001406:	f7ff f907 	bl	8000618 <__aeabi_dmul>
 800140a:	4602      	mov	r2, r0
 800140c:	460b      	mov	r3, r1
 800140e:	e9c7 233e 	strd	r2, r3, [r7, #248]	; 0xf8

					temp_degr = (float) (var1 + var2) / 5120.0;
 8001412:	e9d7 233e 	ldrd	r2, r3, [r7, #248]	; 0xf8
 8001416:	e9d7 0140 	ldrd	r0, r1, [r7, #256]	; 0x100
 800141a:	f7fe ff47 	bl	80002ac <__adddf3>
 800141e:	4602      	mov	r2, r0
 8001420:	460b      	mov	r3, r1
 8001422:	4610      	mov	r0, r2
 8001424:	4619      	mov	r1, r3
 8001426:	f7ff fbcf 	bl	8000bc8 <__aeabi_d2f>
 800142a:	ee06 0a90 	vmov	s13, r0
 800142e:	ed9f 7a2c 	vldr	s14, [pc, #176]	; 80014e0 <main+0x574>
 8001432:	eec6 7a87 	vdiv.f32	s15, s13, s14
 8001436:	edc7 7a42 	vstr	s15, [r7, #264]	; 0x108

					sprintf(temp_char_num, "%f", temp_degr);
 800143a:	f8d7 0108 	ldr.w	r0, [r7, #264]	; 0x108
 800143e:	f7ff f893 	bl	8000568 <__aeabi_f2d>
 8001442:	4602      	mov	r2, r0
 8001444:	460b      	mov	r3, r1
 8001446:	f107 00d8 	add.w	r0, r7, #216	; 0xd8
 800144a:	4926      	ldr	r1, [pc, #152]	; (80014e4 <main+0x578>)
 800144c:	f003 fa0e 	bl	800486c <siprintf>
					HAL_UART_Transmit(&huart1,temp_char_num,sizeof(temp_char_num), 500);
 8001450:	f107 01d8 	add.w	r1, r7, #216	; 0xd8
 8001454:	f44f 73fa 	mov.w	r3, #500	; 0x1f4
 8001458:	2205      	movs	r2, #5
 800145a:	4823      	ldr	r0, [pc, #140]	; (80014e8 <main+0x57c>)
 800145c:	f002 f945 	bl	80036ea <HAL_UART_Transmit>
					HAL_UART_Transmit(&huart1,skip,sizeof(skip)-1, 500);
 8001460:	f107 01d4 	add.w	r1, r7, #212	; 0xd4
 8001464:	f44f 73fa 	mov.w	r3, #500	; 0x1f4
 8001468:	2202      	movs	r2, #2
 800146a:	481f      	ldr	r0, [pc, #124]	; (80014e8 <main+0x57c>)
 800146c:	f002 f93d 	bl	80036ea <HAL_UART_Transmit>



					if (temp_degr > 40.0){
 8001470:	edd7 7a42 	vldr	s15, [r7, #264]	; 0x108
 8001474:	ed9f 7a1d 	vldr	s14, [pc, #116]	; 80014ec <main+0x580>
 8001478:	eef4 7ac7 	vcmpe.f32	s15, s14
 800147c:	eef1 fa10 	vmrs	APSR_nzcv, fpscr
 8001480:	dd0c      	ble.n	800149c <main+0x530>
						HAL_GPIO_WritePin(LED_4_GPIO_Port, LED_4_Pin, GPIO_PIN_SET);
 8001482:	2201      	movs	r2, #1
 8001484:	f44f 4180 	mov.w	r1, #16384	; 0x4000
 8001488:	4819      	ldr	r0, [pc, #100]	; (80014f0 <main+0x584>)
 800148a:	f000 fe87 	bl	800219c <HAL_GPIO_WritePin>
						HAL_UART_Transmit(&huart1,MGS_Alert,sizeof(MGS_Alert)-1, 500);
 800148e:	1d39      	adds	r1, r7, #4
 8001490:	f44f 73fa 	mov.w	r3, #500	; 0x1f4
 8001494:	2214      	movs	r2, #20
 8001496:	4814      	ldr	r0, [pc, #80]	; (80014e8 <main+0x57c>)
 8001498:	f002 f927 	bl	80036ea <HAL_UART_Transmit>

					}

					if (temp_degr < 40.0){
 800149c:	edd7 7a42 	vldr	s15, [r7, #264]	; 0x108
 80014a0:	ed9f 7a12 	vldr	s14, [pc, #72]	; 80014ec <main+0x580>
 80014a4:	eef4 7ac7 	vcmpe.f32	s15, s14
 80014a8:	eef1 fa10 	vmrs	APSR_nzcv, fpscr
 80014ac:	d505      	bpl.n	80014ba <main+0x54e>
						HAL_GPIO_WritePin(LED_4_GPIO_Port, LED_4_Pin, GPIO_PIN_RESET);
 80014ae:	2200      	movs	r2, #0
 80014b0:	f44f 4180 	mov.w	r1, #16384	; 0x4000
 80014b4:	480e      	ldr	r0, [pc, #56]	; (80014f0 <main+0x584>)
 80014b6:	f000 fe71 	bl	800219c <HAL_GPIO_WritePin>
					}

				}
			}
			HAL_GPIO_WritePin(bmp280_CS_GPIO_Port, bmp280_CS_Pin,
 80014ba:	2201      	movs	r2, #1
 80014bc:	2110      	movs	r1, #16
 80014be:	4803      	ldr	r0, [pc, #12]	; (80014cc <main+0x560>)
 80014c0:	f000 fe6c 	bl	800219c <HAL_GPIO_WritePin>
					GPIO_PIN_SET);
			HAL_Delay(100);
 80014c4:	2064      	movs	r0, #100	; 0x64
 80014c6:	f000 fbb3 	bl	8001c30 <HAL_Delay>
	if (HAL_UART_Receive(&huart1, &rx_data, 1, 500) == HAL_OK) {   // Wait for the letter command
 80014ca:	e6a7      	b.n	800121c <main+0x2b0>
 80014cc:	40020800 	.word	0x40020800
 80014d0:	200001f8 	.word	0x200001f8
 80014d4:	40d00000 	.word	0x40d00000
 80014d8:	40900000 	.word	0x40900000
 80014dc:	40c00000 	.word	0x40c00000
 80014e0:	45a00000 	.word	0x45a00000
 80014e4:	08006d60 	.word	0x08006d60
 80014e8:	20000250 	.word	0x20000250
 80014ec:	42200000 	.word	0x42200000
 80014f0:	40021800 	.word	0x40021800

080014f4 <SystemClock_Config>:

/**
* @brief System Clock Configuration
* @retval None
*/
void SystemClock_Config(void) {
 80014f4:	b580      	push	{r7, lr}
 80014f6:	b094      	sub	sp, #80	; 0x50
 80014f8:	af00      	add	r7, sp, #0
RCC_OscInitTypeDef RCC_OscInitStruct = { 0 };
 80014fa:	f107 0320 	add.w	r3, r7, #32
 80014fe:	2230      	movs	r2, #48	; 0x30
 8001500:	2100      	movs	r1, #0
 8001502:	4618      	mov	r0, r3
 8001504:	f002 fd40 	bl	8003f88 <memset>
RCC_ClkInitTypeDef RCC_ClkInitStruct = { 0 };
 8001508:	f107 030c 	add.w	r3, r7, #12
 800150c:	2200      	movs	r2, #0
 800150e:	601a      	str	r2, [r3, #0]
 8001510:	605a      	str	r2, [r3, #4]
 8001512:	609a      	str	r2, [r3, #8]
 8001514:	60da      	str	r2, [r3, #12]
 8001516:	611a      	str	r2, [r3, #16]

/** Configure the main internal regulator output voltage
 */
__HAL_RCC_PWR_CLK_ENABLE();
 8001518:	2300      	movs	r3, #0
 800151a:	60bb      	str	r3, [r7, #8]
 800151c:	4b29      	ldr	r3, [pc, #164]	; (80015c4 <SystemClock_Config+0xd0>)
 800151e:	6c1b      	ldr	r3, [r3, #64]	; 0x40
 8001520:	4a28      	ldr	r2, [pc, #160]	; (80015c4 <SystemClock_Config+0xd0>)
 8001522:	f043 5380 	orr.w	r3, r3, #268435456	; 0x10000000
 8001526:	6413      	str	r3, [r2, #64]	; 0x40
 8001528:	4b26      	ldr	r3, [pc, #152]	; (80015c4 <SystemClock_Config+0xd0>)
 800152a:	6c1b      	ldr	r3, [r3, #64]	; 0x40
 800152c:	f003 5380 	and.w	r3, r3, #268435456	; 0x10000000
 8001530:	60bb      	str	r3, [r7, #8]
 8001532:	68bb      	ldr	r3, [r7, #8]
__HAL_PWR_VOLTAGESCALING_CONFIG(PWR_REGULATOR_VOLTAGE_SCALE3);
 8001534:	2300      	movs	r3, #0
 8001536:	607b      	str	r3, [r7, #4]
 8001538:	4b23      	ldr	r3, [pc, #140]	; (80015c8 <SystemClock_Config+0xd4>)
 800153a:	681b      	ldr	r3, [r3, #0]
 800153c:	f423 4340 	bic.w	r3, r3, #49152	; 0xc000
 8001540:	4a21      	ldr	r2, [pc, #132]	; (80015c8 <SystemClock_Config+0xd4>)
 8001542:	f443 4380 	orr.w	r3, r3, #16384	; 0x4000
 8001546:	6013      	str	r3, [r2, #0]
 8001548:	4b1f      	ldr	r3, [pc, #124]	; (80015c8 <SystemClock_Config+0xd4>)
 800154a:	681b      	ldr	r3, [r3, #0]
 800154c:	f403 4340 	and.w	r3, r3, #49152	; 0xc000
 8001550:	607b      	str	r3, [r7, #4]
 8001552:	687b      	ldr	r3, [r7, #4]

/** Initializes the RCC Oscillators according to the specified parameters
 * in the RCC_OscInitTypeDef structure.
 */
RCC_OscInitStruct.OscillatorType = RCC_OSCILLATORTYPE_HSI;
 8001554:	2302      	movs	r3, #2
 8001556:	623b      	str	r3, [r7, #32]
RCC_OscInitStruct.HSIState = RCC_HSI_ON;
 8001558:	2301      	movs	r3, #1
 800155a:	62fb      	str	r3, [r7, #44]	; 0x2c
RCC_OscInitStruct.HSICalibrationValue = RCC_HSICALIBRATION_DEFAULT;
 800155c:	2310      	movs	r3, #16
 800155e:	633b      	str	r3, [r7, #48]	; 0x30
RCC_OscInitStruct.PLL.PLLState = RCC_PLL_ON;
 8001560:	2302      	movs	r3, #2
 8001562:	63bb      	str	r3, [r7, #56]	; 0x38
RCC_OscInitStruct.PLL.PLLSource = RCC_PLLSOURCE_HSI;
 8001564:	2300      	movs	r3, #0
 8001566:	63fb      	str	r3, [r7, #60]	; 0x3c
RCC_OscInitStruct.PLL.PLLM = 8;
 8001568:	2308      	movs	r3, #8
 800156a:	643b      	str	r3, [r7, #64]	; 0x40
RCC_OscInitStruct.PLL.PLLN = 64;
 800156c:	2340      	movs	r3, #64	; 0x40
 800156e:	647b      	str	r3, [r7, #68]	; 0x44
RCC_OscInitStruct.PLL.PLLP = RCC_PLLP_DIV2;
 8001570:	2302      	movs	r3, #2
 8001572:	64bb      	str	r3, [r7, #72]	; 0x48
RCC_OscInitStruct.PLL.PLLQ = 7;
 8001574:	2307      	movs	r3, #7
 8001576:	64fb      	str	r3, [r7, #76]	; 0x4c
if (HAL_RCC_OscConfig(&RCC_OscInitStruct) != HAL_OK) {
 8001578:	f107 0320 	add.w	r3, r7, #32
 800157c:	4618      	mov	r0, r3
 800157e:	f000 fe27 	bl	80021d0 <HAL_RCC_OscConfig>
 8001582:	4603      	mov	r3, r0
 8001584:	2b00      	cmp	r3, #0
 8001586:	d001      	beq.n	800158c <SystemClock_Config+0x98>
	Error_Handler();
 8001588:	f000 f8f6 	bl	8001778 <Error_Handler>
}

/** Initializes the CPU, AHB and APB buses clocks
 */
RCC_ClkInitStruct.ClockType = RCC_CLOCKTYPE_HCLK | RCC_CLOCKTYPE_SYSCLK
 800158c:	230f      	movs	r3, #15
 800158e:	60fb      	str	r3, [r7, #12]
		| RCC_CLOCKTYPE_PCLK1 | RCC_CLOCKTYPE_PCLK2;
RCC_ClkInitStruct.SYSCLKSource = RCC_SYSCLKSOURCE_PLLCLK;
 8001590:	2302      	movs	r3, #2
 8001592:	613b      	str	r3, [r7, #16]
RCC_ClkInitStruct.AHBCLKDivider = RCC_SYSCLK_DIV1;
 8001594:	2300      	movs	r3, #0
 8001596:	617b      	str	r3, [r7, #20]
RCC_ClkInitStruct.APB1CLKDivider = RCC_HCLK_DIV2;
 8001598:	f44f 5380 	mov.w	r3, #4096	; 0x1000
 800159c:	61bb      	str	r3, [r7, #24]
RCC_ClkInitStruct.APB2CLKDivider = RCC_HCLK_DIV4;
 800159e:	f44f 53a0 	mov.w	r3, #5120	; 0x1400
 80015a2:	61fb      	str	r3, [r7, #28]

if (HAL_RCC_ClockConfig(&RCC_ClkInitStruct, FLASH_LATENCY_2) != HAL_OK) {
 80015a4:	f107 030c 	add.w	r3, r7, #12
 80015a8:	2102      	movs	r1, #2
 80015aa:	4618      	mov	r0, r3
 80015ac:	f001 f888 	bl	80026c0 <HAL_RCC_ClockConfig>
 80015b0:	4603      	mov	r3, r0
 80015b2:	2b00      	cmp	r3, #0
 80015b4:	d001      	beq.n	80015ba <SystemClock_Config+0xc6>
	Error_Handler();
 80015b6:	f000 f8df 	bl	8001778 <Error_Handler>
}
}
 80015ba:	bf00      	nop
 80015bc:	3750      	adds	r7, #80	; 0x50
 80015be:	46bd      	mov	sp, r7
 80015c0:	bd80      	pop	{r7, pc}
 80015c2:	bf00      	nop
 80015c4:	40023800 	.word	0x40023800
 80015c8:	40007000 	.word	0x40007000

080015cc <MX_SPI1_Init>:
/**
* @brief SPI1 Initialization Function
* @param None
* @retval None
*/
static void MX_SPI1_Init(void) {
 80015cc:	b580      	push	{r7, lr}
 80015ce:	af00      	add	r7, sp, #0

/* USER CODE BEGIN SPI1_Init 1 */

/* USER CODE END SPI1_Init 1 */
/* SPI1 parameter configuration*/
hspi1.Instance = SPI1;
 80015d0:	4b17      	ldr	r3, [pc, #92]	; (8001630 <MX_SPI1_Init+0x64>)
 80015d2:	4a18      	ldr	r2, [pc, #96]	; (8001634 <MX_SPI1_Init+0x68>)
 80015d4:	601a      	str	r2, [r3, #0]
hspi1.Init.Mode = SPI_MODE_MASTER;
 80015d6:	4b16      	ldr	r3, [pc, #88]	; (8001630 <MX_SPI1_Init+0x64>)
 80015d8:	f44f 7282 	mov.w	r2, #260	; 0x104
 80015dc:	605a      	str	r2, [r3, #4]
hspi1.Init.Direction = SPI_DIRECTION_2LINES;
 80015de:	4b14      	ldr	r3, [pc, #80]	; (8001630 <MX_SPI1_Init+0x64>)
 80015e0:	2200      	movs	r2, #0
 80015e2:	609a      	str	r2, [r3, #8]
hspi1.Init.DataSize = SPI_DATASIZE_8BIT;
 80015e4:	4b12      	ldr	r3, [pc, #72]	; (8001630 <MX_SPI1_Init+0x64>)
 80015e6:	2200      	movs	r2, #0
 80015e8:	60da      	str	r2, [r3, #12]
hspi1.Init.CLKPolarity = SPI_POLARITY_LOW;
 80015ea:	4b11      	ldr	r3, [pc, #68]	; (8001630 <MX_SPI1_Init+0x64>)
 80015ec:	2200      	movs	r2, #0
 80015ee:	611a      	str	r2, [r3, #16]
hspi1.Init.CLKPhase = SPI_PHASE_1EDGE;
 80015f0:	4b0f      	ldr	r3, [pc, #60]	; (8001630 <MX_SPI1_Init+0x64>)
 80015f2:	2200      	movs	r2, #0
 80015f4:	615a      	str	r2, [r3, #20]
hspi1.Init.NSS = SPI_NSS_SOFT;
 80015f6:	4b0e      	ldr	r3, [pc, #56]	; (8001630 <MX_SPI1_Init+0x64>)
 80015f8:	f44f 7200 	mov.w	r2, #512	; 0x200
 80015fc:	619a      	str	r2, [r3, #24]
hspi1.Init.BaudRatePrescaler = SPI_BAUDRATEPRESCALER_2;
 80015fe:	4b0c      	ldr	r3, [pc, #48]	; (8001630 <MX_SPI1_Init+0x64>)
 8001600:	2200      	movs	r2, #0
 8001602:	61da      	str	r2, [r3, #28]
hspi1.Init.FirstBit = SPI_FIRSTBIT_MSB;
 8001604:	4b0a      	ldr	r3, [pc, #40]	; (8001630 <MX_SPI1_Init+0x64>)
 8001606:	2200      	movs	r2, #0
 8001608:	621a      	str	r2, [r3, #32]
hspi1.Init.TIMode = SPI_TIMODE_DISABLE;
 800160a:	4b09      	ldr	r3, [pc, #36]	; (8001630 <MX_SPI1_Init+0x64>)
 800160c:	2200      	movs	r2, #0
 800160e:	625a      	str	r2, [r3, #36]	; 0x24
hspi1.Init.CRCCalculation = SPI_CRCCALCULATION_DISABLE;
 8001610:	4b07      	ldr	r3, [pc, #28]	; (8001630 <MX_SPI1_Init+0x64>)
 8001612:	2200      	movs	r2, #0
 8001614:	629a      	str	r2, [r3, #40]	; 0x28
hspi1.Init.CRCPolynomial = 10;
 8001616:	4b06      	ldr	r3, [pc, #24]	; (8001630 <MX_SPI1_Init+0x64>)
 8001618:	220a      	movs	r2, #10
 800161a:	62da      	str	r2, [r3, #44]	; 0x2c
if (HAL_SPI_Init(&hspi1) != HAL_OK) {
 800161c:	4804      	ldr	r0, [pc, #16]	; (8001630 <MX_SPI1_Init+0x64>)
 800161e:	f001 fa6f 	bl	8002b00 <HAL_SPI_Init>
 8001622:	4603      	mov	r3, r0
 8001624:	2b00      	cmp	r3, #0
 8001626:	d001      	beq.n	800162c <MX_SPI1_Init+0x60>
	Error_Handler();
 8001628:	f000 f8a6 	bl	8001778 <Error_Handler>
}
/* USER CODE BEGIN SPI1_Init 2 */

/* USER CODE END SPI1_Init 2 */

}
 800162c:	bf00      	nop
 800162e:	bd80      	pop	{r7, pc}
 8001630:	200001f8 	.word	0x200001f8
 8001634:	40013000 	.word	0x40013000

08001638 <MX_USART1_UART_Init>:
/**
* @brief USART1 Initialization Function
* @param None
* @retval None
*/
static void MX_USART1_UART_Init(void) {
 8001638:	b580      	push	{r7, lr}
 800163a:	af00      	add	r7, sp, #0
/* USER CODE END USART1_Init 0 */

/* USER CODE BEGIN USART1_Init 1 */

/* USER CODE END USART1_Init 1 */
huart1.Instance = USART1;
 800163c:	4b11      	ldr	r3, [pc, #68]	; (8001684 <MX_USART1_UART_Init+0x4c>)
 800163e:	4a12      	ldr	r2, [pc, #72]	; (8001688 <MX_USART1_UART_Init+0x50>)
 8001640:	601a      	str	r2, [r3, #0]
huart1.Init.BaudRate = 115200;
 8001642:	4b10      	ldr	r3, [pc, #64]	; (8001684 <MX_USART1_UART_Init+0x4c>)
 8001644:	f44f 32e1 	mov.w	r2, #115200	; 0x1c200
 8001648:	605a      	str	r2, [r3, #4]
huart1.Init.WordLength = UART_WORDLENGTH_8B;
 800164a:	4b0e      	ldr	r3, [pc, #56]	; (8001684 <MX_USART1_UART_Init+0x4c>)
 800164c:	2200      	movs	r2, #0
 800164e:	609a      	str	r2, [r3, #8]
huart1.Init.StopBits = UART_STOPBITS_1;
 8001650:	4b0c      	ldr	r3, [pc, #48]	; (8001684 <MX_USART1_UART_Init+0x4c>)
 8001652:	2200      	movs	r2, #0
 8001654:	60da      	str	r2, [r3, #12]
huart1.Init.Parity = UART_PARITY_NONE;
 8001656:	4b0b      	ldr	r3, [pc, #44]	; (8001684 <MX_USART1_UART_Init+0x4c>)
 8001658:	2200      	movs	r2, #0
 800165a:	611a      	str	r2, [r3, #16]
huart1.Init.Mode = UART_MODE_TX_RX;
 800165c:	4b09      	ldr	r3, [pc, #36]	; (8001684 <MX_USART1_UART_Init+0x4c>)
 800165e:	220c      	movs	r2, #12
 8001660:	615a      	str	r2, [r3, #20]
huart1.Init.HwFlowCtl = UART_HWCONTROL_NONE;
 8001662:	4b08      	ldr	r3, [pc, #32]	; (8001684 <MX_USART1_UART_Init+0x4c>)
 8001664:	2200      	movs	r2, #0
 8001666:	619a      	str	r2, [r3, #24]
huart1.Init.OverSampling = UART_OVERSAMPLING_16;
 8001668:	4b06      	ldr	r3, [pc, #24]	; (8001684 <MX_USART1_UART_Init+0x4c>)
 800166a:	2200      	movs	r2, #0
 800166c:	61da      	str	r2, [r3, #28]
if (HAL_UART_Init(&huart1) != HAL_OK) {
 800166e:	4805      	ldr	r0, [pc, #20]	; (8001684 <MX_USART1_UART_Init+0x4c>)
 8001670:	f001 ffee 	bl	8003650 <HAL_UART_Init>
 8001674:	4603      	mov	r3, r0
 8001676:	2b00      	cmp	r3, #0
 8001678:	d001      	beq.n	800167e <MX_USART1_UART_Init+0x46>
	Error_Handler();
 800167a:	f000 f87d 	bl	8001778 <Error_Handler>
}
/* USER CODE BEGIN USART1_Init 2 */

/* USER CODE END USART1_Init 2 */

}
 800167e:	bf00      	nop
 8001680:	bd80      	pop	{r7, pc}
 8001682:	bf00      	nop
 8001684:	20000250 	.word	0x20000250
 8001688:	40011000 	.word	0x40011000

0800168c <MX_GPIO_Init>:
/**
* @brief GPIO Initialization Function
* @param None
* @retval None
*/
static void MX_GPIO_Init(void) {
 800168c:	b580      	push	{r7, lr}
 800168e:	b08a      	sub	sp, #40	; 0x28
 8001690:	af00      	add	r7, sp, #0
GPIO_InitTypeDef GPIO_InitStruct = { 0 };
 8001692:	f107 0314 	add.w	r3, r7, #20
 8001696:	2200      	movs	r2, #0
 8001698:	601a      	str	r2, [r3, #0]
 800169a:	605a      	str	r2, [r3, #4]
 800169c:	609a      	str	r2, [r3, #8]
 800169e:	60da      	str	r2, [r3, #12]
 80016a0:	611a      	str	r2, [r3, #16]

/* GPIO Ports Clock Enable */
__HAL_RCC_GPIOH_CLK_ENABLE();
 80016a2:	2300      	movs	r3, #0
 80016a4:	613b      	str	r3, [r7, #16]
 80016a6:	4b31      	ldr	r3, [pc, #196]	; (800176c <MX_GPIO_Init+0xe0>)
 80016a8:	6b1b      	ldr	r3, [r3, #48]	; 0x30
 80016aa:	4a30      	ldr	r2, [pc, #192]	; (800176c <MX_GPIO_Init+0xe0>)
 80016ac:	f043 0380 	orr.w	r3, r3, #128	; 0x80
 80016b0:	6313      	str	r3, [r2, #48]	; 0x30
 80016b2:	4b2e      	ldr	r3, [pc, #184]	; (800176c <MX_GPIO_Init+0xe0>)
 80016b4:	6b1b      	ldr	r3, [r3, #48]	; 0x30
 80016b6:	f003 0380 	and.w	r3, r3, #128	; 0x80
 80016ba:	613b      	str	r3, [r7, #16]
 80016bc:	693b      	ldr	r3, [r7, #16]
__HAL_RCC_GPIOA_CLK_ENABLE();
 80016be:	2300      	movs	r3, #0
 80016c0:	60fb      	str	r3, [r7, #12]
 80016c2:	4b2a      	ldr	r3, [pc, #168]	; (800176c <MX_GPIO_Init+0xe0>)
 80016c4:	6b1b      	ldr	r3, [r3, #48]	; 0x30
 80016c6:	4a29      	ldr	r2, [pc, #164]	; (800176c <MX_GPIO_Init+0xe0>)
 80016c8:	f043 0301 	orr.w	r3, r3, #1
 80016cc:	6313      	str	r3, [r2, #48]	; 0x30
 80016ce:	4b27      	ldr	r3, [pc, #156]	; (800176c <MX_GPIO_Init+0xe0>)
 80016d0:	6b1b      	ldr	r3, [r3, #48]	; 0x30
 80016d2:	f003 0301 	and.w	r3, r3, #1
 80016d6:	60fb      	str	r3, [r7, #12]
 80016d8:	68fb      	ldr	r3, [r7, #12]
__HAL_RCC_GPIOC_CLK_ENABLE();
 80016da:	2300      	movs	r3, #0
 80016dc:	60bb      	str	r3, [r7, #8]
 80016de:	4b23      	ldr	r3, [pc, #140]	; (800176c <MX_GPIO_Init+0xe0>)
 80016e0:	6b1b      	ldr	r3, [r3, #48]	; 0x30
 80016e2:	4a22      	ldr	r2, [pc, #136]	; (800176c <MX_GPIO_Init+0xe0>)
 80016e4:	f043 0304 	orr.w	r3, r3, #4
 80016e8:	6313      	str	r3, [r2, #48]	; 0x30
 80016ea:	4b20      	ldr	r3, [pc, #128]	; (800176c <MX_GPIO_Init+0xe0>)
 80016ec:	6b1b      	ldr	r3, [r3, #48]	; 0x30
 80016ee:	f003 0304 	and.w	r3, r3, #4
 80016f2:	60bb      	str	r3, [r7, #8]
 80016f4:	68bb      	ldr	r3, [r7, #8]
__HAL_RCC_GPIOG_CLK_ENABLE();
 80016f6:	2300      	movs	r3, #0
 80016f8:	607b      	str	r3, [r7, #4]
 80016fa:	4b1c      	ldr	r3, [pc, #112]	; (800176c <MX_GPIO_Init+0xe0>)
 80016fc:	6b1b      	ldr	r3, [r3, #48]	; 0x30
 80016fe:	4a1b      	ldr	r2, [pc, #108]	; (800176c <MX_GPIO_Init+0xe0>)
 8001700:	f043 0340 	orr.w	r3, r3, #64	; 0x40
 8001704:	6313      	str	r3, [r2, #48]	; 0x30
 8001706:	4b19      	ldr	r3, [pc, #100]	; (800176c <MX_GPIO_Init+0xe0>)
 8001708:	6b1b      	ldr	r3, [r3, #48]	; 0x30
 800170a:	f003 0340 	and.w	r3, r3, #64	; 0x40
 800170e:	607b      	str	r3, [r7, #4]
 8001710:	687b      	ldr	r3, [r7, #4]

/*Configure GPIO pin Output Level */
HAL_GPIO_WritePin(bmp280_CS_GPIO_Port, bmp280_CS_Pin, GPIO_PIN_RESET);
 8001712:	2200      	movs	r2, #0
 8001714:	2110      	movs	r1, #16
 8001716:	4816      	ldr	r0, [pc, #88]	; (8001770 <MX_GPIO_Init+0xe4>)
 8001718:	f000 fd40 	bl	800219c <HAL_GPIO_WritePin>

/*Configure GPIO pin Output Level */
HAL_GPIO_WritePin(LED_4_GPIO_Port, LED_4_Pin, GPIO_PIN_RESET);
 800171c:	2200      	movs	r2, #0
 800171e:	f44f 4180 	mov.w	r1, #16384	; 0x4000
 8001722:	4814      	ldr	r0, [pc, #80]	; (8001774 <MX_GPIO_Init+0xe8>)
 8001724:	f000 fd3a 	bl	800219c <HAL_GPIO_WritePin>

/*Configure GPIO pin : bmp280_CS_Pin */
GPIO_InitStruct.Pin = bmp280_CS_Pin;
 8001728:	2310      	movs	r3, #16
 800172a:	617b      	str	r3, [r7, #20]
GPIO_InitStruct.Mode = GPIO_MODE_OUTPUT_PP;
 800172c:	2301      	movs	r3, #1
 800172e:	61bb      	str	r3, [r7, #24]
GPIO_InitStruct.Pull = GPIO_NOPULL;
 8001730:	2300      	movs	r3, #0
 8001732:	61fb      	str	r3, [r7, #28]
GPIO_InitStruct.Speed = GPIO_SPEED_FREQ_LOW;
 8001734:	2300      	movs	r3, #0
 8001736:	623b      	str	r3, [r7, #32]
HAL_GPIO_Init(bmp280_CS_GPIO_Port, &GPIO_InitStruct);
 8001738:	f107 0314 	add.w	r3, r7, #20
 800173c:	4619      	mov	r1, r3
 800173e:	480c      	ldr	r0, [pc, #48]	; (8001770 <MX_GPIO_Init+0xe4>)
 8001740:	f000 fb80 	bl	8001e44 <HAL_GPIO_Init>

/*Configure GPIO pin : LED_4_Pin */
GPIO_InitStruct.Pin = LED_4_Pin;
 8001744:	f44f 4380 	mov.w	r3, #16384	; 0x4000
 8001748:	617b      	str	r3, [r7, #20]
GPIO_InitStruct.Mode = GPIO_MODE_OUTPUT_PP;
 800174a:	2301      	movs	r3, #1
 800174c:	61bb      	str	r3, [r7, #24]
GPIO_InitStruct.Pull = GPIO_NOPULL;
 800174e:	2300      	movs	r3, #0
 8001750:	61fb      	str	r3, [r7, #28]
GPIO_InitStruct.Speed = GPIO_SPEED_FREQ_LOW;
 8001752:	2300      	movs	r3, #0
 8001754:	623b      	str	r3, [r7, #32]
HAL_GPIO_Init(LED_4_GPIO_Port, &GPIO_InitStruct);
 8001756:	f107 0314 	add.w	r3, r7, #20
 800175a:	4619      	mov	r1, r3
 800175c:	4805      	ldr	r0, [pc, #20]	; (8001774 <MX_GPIO_Init+0xe8>)
 800175e:	f000 fb71 	bl	8001e44 <HAL_GPIO_Init>

}
 8001762:	bf00      	nop
 8001764:	3728      	adds	r7, #40	; 0x28
 8001766:	46bd      	mov	sp, r7
 8001768:	bd80      	pop	{r7, pc}
 800176a:	bf00      	nop
 800176c:	40023800 	.word	0x40023800
 8001770:	40020800 	.word	0x40020800
 8001774:	40021800 	.word	0x40021800

08001778 <Error_Handler>:

/**
* @brief  This function is executed in case of error occurrence.
* @retval None
*/
void Error_Handler(void) {
 8001778:	b480      	push	{r7}
 800177a:	af00      	add	r7, sp, #0
  \details Disables IRQ interrupts by setting the I-bit in the CPSR.
           Can only be executed in Privileged modes.
 */
__STATIC_FORCEINLINE void __disable_irq(void)
{
  __ASM volatile ("cpsid i" : : : "memory");
 800177c:	b672      	cpsid	i
}
 800177e:	bf00      	nop
/* USER CODE BEGIN Error_Handler_Debug */
/* User can add his own implementation to report the HAL error return state */
__disable_irq();
while (1) {
 8001780:	e7fe      	b.n	8001780 <Error_Handler+0x8>
	...

08001784 <HAL_MspInit>:
/* USER CODE END 0 */
/**
  * Initializes the Global MSP.
  */
void HAL_MspInit(void)
{
 8001784:	b580      	push	{r7, lr}
 8001786:	b082      	sub	sp, #8
 8001788:	af00      	add	r7, sp, #0
  /* USER CODE BEGIN MspInit 0 */

  /* USER CODE END MspInit 0 */

  __HAL_RCC_SYSCFG_CLK_ENABLE();
 800178a:	2300      	movs	r3, #0
 800178c:	607b      	str	r3, [r7, #4]
 800178e:	4b10      	ldr	r3, [pc, #64]	; (80017d0 <HAL_MspInit+0x4c>)
 8001790:	6c5b      	ldr	r3, [r3, #68]	; 0x44
 8001792:	4a0f      	ldr	r2, [pc, #60]	; (80017d0 <HAL_MspInit+0x4c>)
 8001794:	f443 4380 	orr.w	r3, r3, #16384	; 0x4000
 8001798:	6453      	str	r3, [r2, #68]	; 0x44
 800179a:	4b0d      	ldr	r3, [pc, #52]	; (80017d0 <HAL_MspInit+0x4c>)
 800179c:	6c5b      	ldr	r3, [r3, #68]	; 0x44
 800179e:	f403 4380 	and.w	r3, r3, #16384	; 0x4000
 80017a2:	607b      	str	r3, [r7, #4]
 80017a4:	687b      	ldr	r3, [r7, #4]
  __HAL_RCC_PWR_CLK_ENABLE();
 80017a6:	2300      	movs	r3, #0
 80017a8:	603b      	str	r3, [r7, #0]
 80017aa:	4b09      	ldr	r3, [pc, #36]	; (80017d0 <HAL_MspInit+0x4c>)
 80017ac:	6c1b      	ldr	r3, [r3, #64]	; 0x40
 80017ae:	4a08      	ldr	r2, [pc, #32]	; (80017d0 <HAL_MspInit+0x4c>)
 80017b0:	f043 5380 	orr.w	r3, r3, #268435456	; 0x10000000
 80017b4:	6413      	str	r3, [r2, #64]	; 0x40
 80017b6:	4b06      	ldr	r3, [pc, #24]	; (80017d0 <HAL_MspInit+0x4c>)
 80017b8:	6c1b      	ldr	r3, [r3, #64]	; 0x40
 80017ba:	f003 5380 	and.w	r3, r3, #268435456	; 0x10000000
 80017be:	603b      	str	r3, [r7, #0]
 80017c0:	683b      	ldr	r3, [r7, #0]

  HAL_NVIC_SetPriorityGrouping(NVIC_PRIORITYGROUP_0);
 80017c2:	2007      	movs	r0, #7
 80017c4:	f000 fb0a 	bl	8001ddc <HAL_NVIC_SetPriorityGrouping>
  /* System interrupt init*/

  /* USER CODE BEGIN MspInit 1 */

  /* USER CODE END MspInit 1 */
}
 80017c8:	bf00      	nop
 80017ca:	3708      	adds	r7, #8
 80017cc:	46bd      	mov	sp, r7
 80017ce:	bd80      	pop	{r7, pc}
 80017d0:	40023800 	.word	0x40023800

080017d4 <HAL_SPI_MspInit>:
* This function configures the hardware resources used in this example
* @param hspi: SPI handle pointer
* @retval None
*/
void HAL_SPI_MspInit(SPI_HandleTypeDef* hspi)
{
 80017d4:	b580      	push	{r7, lr}
 80017d6:	b08a      	sub	sp, #40	; 0x28
 80017d8:	af00      	add	r7, sp, #0
 80017da:	6078      	str	r0, [r7, #4]
  GPIO_InitTypeDef GPIO_InitStruct = {0};
 80017dc:	f107 0314 	add.w	r3, r7, #20
 80017e0:	2200      	movs	r2, #0
 80017e2:	601a      	str	r2, [r3, #0]
 80017e4:	605a      	str	r2, [r3, #4]
 80017e6:	609a      	str	r2, [r3, #8]
 80017e8:	60da      	str	r2, [r3, #12]
 80017ea:	611a      	str	r2, [r3, #16]
  if(hspi->Instance==SPI1)
 80017ec:	687b      	ldr	r3, [r7, #4]
 80017ee:	681b      	ldr	r3, [r3, #0]
 80017f0:	4a19      	ldr	r2, [pc, #100]	; (8001858 <HAL_SPI_MspInit+0x84>)
 80017f2:	4293      	cmp	r3, r2
 80017f4:	d12b      	bne.n	800184e <HAL_SPI_MspInit+0x7a>
  {
  /* USER CODE BEGIN SPI1_MspInit 0 */

  /* USER CODE END SPI1_MspInit 0 */
    /* Peripheral clock enable */
    __HAL_RCC_SPI1_CLK_ENABLE();
 80017f6:	2300      	movs	r3, #0
 80017f8:	613b      	str	r3, [r7, #16]
 80017fa:	4b18      	ldr	r3, [pc, #96]	; (800185c <HAL_SPI_MspInit+0x88>)
 80017fc:	6c5b      	ldr	r3, [r3, #68]	; 0x44
 80017fe:	4a17      	ldr	r2, [pc, #92]	; (800185c <HAL_SPI_MspInit+0x88>)
 8001800:	f443 5380 	orr.w	r3, r3, #4096	; 0x1000
 8001804:	6453      	str	r3, [r2, #68]	; 0x44
 8001806:	4b15      	ldr	r3, [pc, #84]	; (800185c <HAL_SPI_MspInit+0x88>)
 8001808:	6c5b      	ldr	r3, [r3, #68]	; 0x44
 800180a:	f403 5380 	and.w	r3, r3, #4096	; 0x1000
 800180e:	613b      	str	r3, [r7, #16]
 8001810:	693b      	ldr	r3, [r7, #16]

    __HAL_RCC_GPIOA_CLK_ENABLE();
 8001812:	2300      	movs	r3, #0
 8001814:	60fb      	str	r3, [r7, #12]
 8001816:	4b11      	ldr	r3, [pc, #68]	; (800185c <HAL_SPI_MspInit+0x88>)
 8001818:	6b1b      	ldr	r3, [r3, #48]	; 0x30
 800181a:	4a10      	ldr	r2, [pc, #64]	; (800185c <HAL_SPI_MspInit+0x88>)
 800181c:	f043 0301 	orr.w	r3, r3, #1
 8001820:	6313      	str	r3, [r2, #48]	; 0x30
 8001822:	4b0e      	ldr	r3, [pc, #56]	; (800185c <HAL_SPI_MspInit+0x88>)
 8001824:	6b1b      	ldr	r3, [r3, #48]	; 0x30
 8001826:	f003 0301 	and.w	r3, r3, #1
 800182a:	60fb      	str	r3, [r7, #12]
 800182c:	68fb      	ldr	r3, [r7, #12]
    /**SPI1 GPIO Configuration
    PA5     ------> SPI1_SCK
    PA6     ------> SPI1_MISO
    PA7     ------> SPI1_MOSI
    */
    GPIO_InitStruct.Pin = GPIO_PIN_5|GPIO_PIN_6|GPIO_PIN_7;
 800182e:	23e0      	movs	r3, #224	; 0xe0
 8001830:	617b      	str	r3, [r7, #20]
    GPIO_InitStruct.Mode = GPIO_MODE_AF_PP;
 8001832:	2302      	movs	r3, #2
 8001834:	61bb      	str	r3, [r7, #24]
    GPIO_InitStruct.Pull = GPIO_NOPULL;
 8001836:	2300      	movs	r3, #0
 8001838:	61fb      	str	r3, [r7, #28]
    GPIO_InitStruct.Speed = GPIO_SPEED_FREQ_VERY_HIGH;
 800183a:	2303      	movs	r3, #3
 800183c:	623b      	str	r3, [r7, #32]
    GPIO_InitStruct.Alternate = GPIO_AF5_SPI1;
 800183e:	2305      	movs	r3, #5
 8001840:	627b      	str	r3, [r7, #36]	; 0x24
    HAL_GPIO_Init(GPIOA, &GPIO_InitStruct);
 8001842:	f107 0314 	add.w	r3, r7, #20
 8001846:	4619      	mov	r1, r3
 8001848:	4805      	ldr	r0, [pc, #20]	; (8001860 <HAL_SPI_MspInit+0x8c>)
 800184a:	f000 fafb 	bl	8001e44 <HAL_GPIO_Init>
  /* USER CODE BEGIN SPI1_MspInit 1 */

  /* USER CODE END SPI1_MspInit 1 */
  }

}
 800184e:	bf00      	nop
 8001850:	3728      	adds	r7, #40	; 0x28
 8001852:	46bd      	mov	sp, r7
 8001854:	bd80      	pop	{r7, pc}
 8001856:	bf00      	nop
 8001858:	40013000 	.word	0x40013000
 800185c:	40023800 	.word	0x40023800
 8001860:	40020000 	.word	0x40020000

08001864 <HAL_UART_MspInit>:
* This function configures the hardware resources used in this example
* @param huart: UART handle pointer
* @retval None
*/
void HAL_UART_MspInit(UART_HandleTypeDef* huart)
{
 8001864:	b580      	push	{r7, lr}
 8001866:	b08a      	sub	sp, #40	; 0x28
 8001868:	af00      	add	r7, sp, #0
 800186a:	6078      	str	r0, [r7, #4]
  GPIO_InitTypeDef GPIO_InitStruct = {0};
 800186c:	f107 0314 	add.w	r3, r7, #20
 8001870:	2200      	movs	r2, #0
 8001872:	601a      	str	r2, [r3, #0]
 8001874:	605a      	str	r2, [r3, #4]
 8001876:	609a      	str	r2, [r3, #8]
 8001878:	60da      	str	r2, [r3, #12]
 800187a:	611a      	str	r2, [r3, #16]
  if(huart->Instance==USART1)
 800187c:	687b      	ldr	r3, [r7, #4]
 800187e:	681b      	ldr	r3, [r3, #0]
 8001880:	4a19      	ldr	r2, [pc, #100]	; (80018e8 <HAL_UART_MspInit+0x84>)
 8001882:	4293      	cmp	r3, r2
 8001884:	d12c      	bne.n	80018e0 <HAL_UART_MspInit+0x7c>
  {
  /* USER CODE BEGIN USART1_MspInit 0 */

  /* USER CODE END USART1_MspInit 0 */
    /* Peripheral clock enable */
    __HAL_RCC_USART1_CLK_ENABLE();
 8001886:	2300      	movs	r3, #0
 8001888:	613b      	str	r3, [r7, #16]
 800188a:	4b18      	ldr	r3, [pc, #96]	; (80018ec <HAL_UART_MspInit+0x88>)
 800188c:	6c5b      	ldr	r3, [r3, #68]	; 0x44
 800188e:	4a17      	ldr	r2, [pc, #92]	; (80018ec <HAL_UART_MspInit+0x88>)
 8001890:	f043 0310 	orr.w	r3, r3, #16
 8001894:	6453      	str	r3, [r2, #68]	; 0x44
 8001896:	4b15      	ldr	r3, [pc, #84]	; (80018ec <HAL_UART_MspInit+0x88>)
 8001898:	6c5b      	ldr	r3, [r3, #68]	; 0x44
 800189a:	f003 0310 	and.w	r3, r3, #16
 800189e:	613b      	str	r3, [r7, #16]
 80018a0:	693b      	ldr	r3, [r7, #16]

    __HAL_RCC_GPIOA_CLK_ENABLE();
 80018a2:	2300      	movs	r3, #0
 80018a4:	60fb      	str	r3, [r7, #12]
 80018a6:	4b11      	ldr	r3, [pc, #68]	; (80018ec <HAL_UART_MspInit+0x88>)
 80018a8:	6b1b      	ldr	r3, [r3, #48]	; 0x30
 80018aa:	4a10      	ldr	r2, [pc, #64]	; (80018ec <HAL_UART_MspInit+0x88>)
 80018ac:	f043 0301 	orr.w	r3, r3, #1
 80018b0:	6313      	str	r3, [r2, #48]	; 0x30
 80018b2:	4b0e      	ldr	r3, [pc, #56]	; (80018ec <HAL_UART_MspInit+0x88>)
 80018b4:	6b1b      	ldr	r3, [r3, #48]	; 0x30
 80018b6:	f003 0301 	and.w	r3, r3, #1
 80018ba:	60fb      	str	r3, [r7, #12]
 80018bc:	68fb      	ldr	r3, [r7, #12]
    /**USART1 GPIO Configuration
    PA9     ------> USART1_TX
    PA10     ------> USART1_RX
    */
    GPIO_InitStruct.Pin = GPIO_PIN_9|GPIO_PIN_10;
 80018be:	f44f 63c0 	mov.w	r3, #1536	; 0x600
 80018c2:	617b      	str	r3, [r7, #20]
    GPIO_InitStruct.Mode = GPIO_MODE_AF_PP;
 80018c4:	2302      	movs	r3, #2
 80018c6:	61bb      	str	r3, [r7, #24]
    GPIO_InitStruct.Pull = GPIO_NOPULL;
 80018c8:	2300      	movs	r3, #0
 80018ca:	61fb      	str	r3, [r7, #28]
    GPIO_InitStruct.Speed = GPIO_SPEED_FREQ_VERY_HIGH;
 80018cc:	2303      	movs	r3, #3
 80018ce:	623b      	str	r3, [r7, #32]
    GPIO_InitStruct.Alternate = GPIO_AF7_USART1;
 80018d0:	2307      	movs	r3, #7
 80018d2:	627b      	str	r3, [r7, #36]	; 0x24
    HAL_GPIO_Init(GPIOA, &GPIO_InitStruct);
 80018d4:	f107 0314 	add.w	r3, r7, #20
 80018d8:	4619      	mov	r1, r3
 80018da:	4805      	ldr	r0, [pc, #20]	; (80018f0 <HAL_UART_MspInit+0x8c>)
 80018dc:	f000 fab2 	bl	8001e44 <HAL_GPIO_Init>
  /* USER CODE BEGIN USART1_MspInit 1 */

  /* USER CODE END USART1_MspInit 1 */
  }

}
 80018e0:	bf00      	nop
 80018e2:	3728      	adds	r7, #40	; 0x28
 80018e4:	46bd      	mov	sp, r7
 80018e6:	bd80      	pop	{r7, pc}
 80018e8:	40011000 	.word	0x40011000
 80018ec:	40023800 	.word	0x40023800
 80018f0:	40020000 	.word	0x40020000

080018f4 <NMI_Handler>:
/******************************************************************************/
/**
  * @brief This function handles Non maskable interrupt.
  */
void NMI_Handler(void)
{
 80018f4:	b480      	push	{r7}
 80018f6:	af00      	add	r7, sp, #0
  /* USER CODE BEGIN NonMaskableInt_IRQn 0 */

  /* USER CODE END NonMaskableInt_IRQn 0 */
  /* USER CODE BEGIN NonMaskableInt_IRQn 1 */
  while (1)
 80018f8:	e7fe      	b.n	80018f8 <NMI_Handler+0x4>

080018fa <HardFault_Handler>:

/**
  * @brief This function handles Hard fault interrupt.
  */
void HardFault_Handler(void)
{
 80018fa:	b480      	push	{r7}
 80018fc:	af00      	add	r7, sp, #0
  /* USER CODE BEGIN HardFault_IRQn 0 */

  /* USER CODE END HardFault_IRQn 0 */
  while (1)
 80018fe:	e7fe      	b.n	80018fe <HardFault_Handler+0x4>

08001900 <MemManage_Handler>:

/**
  * @brief This function handles Memory management fault.
  */
void MemManage_Handler(void)
{
 8001900:	b480      	push	{r7}
 8001902:	af00      	add	r7, sp, #0
  /* USER CODE BEGIN MemoryManagement_IRQn 0 */

  /* USER CODE END MemoryManagement_IRQn 0 */
  while (1)
 8001904:	e7fe      	b.n	8001904 <MemManage_Handler+0x4>

08001906 <BusFault_Handler>:

/**
  * @brief This function handles Pre-fetch fault, memory access fault.
  */
void BusFault_Handler(void)
{
 8001906:	b480      	push	{r7}
 8001908:	af00      	add	r7, sp, #0
  /* USER CODE BEGIN BusFault_IRQn 0 */

  /* USER CODE END BusFault_IRQn 0 */
  while (1)
 800190a:	e7fe      	b.n	800190a <BusFault_Handler+0x4>

0800190c <UsageFault_Handler>:

/**
  * @brief This function handles Undefined instruction or illegal state.
  */
void UsageFault_Handler(void)
{
 800190c:	b480      	push	{r7}
 800190e:	af00      	add	r7, sp, #0
  /* USER CODE BEGIN UsageFault_IRQn 0 */

  /* USER CODE END UsageFault_IRQn 0 */
  while (1)
 8001910:	e7fe      	b.n	8001910 <UsageFault_Handler+0x4>

08001912 <SVC_Handler>:

/**
  * @brief This function handles System service call via SWI instruction.
  */
void SVC_Handler(void)
{
 8001912:	b480      	push	{r7}
 8001914:	af00      	add	r7, sp, #0

  /* USER CODE END SVCall_IRQn 0 */
  /* USER CODE BEGIN SVCall_IRQn 1 */

  /* USER CODE END SVCall_IRQn 1 */
}
 8001916:	bf00      	nop
 8001918:	46bd      	mov	sp, r7
 800191a:	f85d 7b04 	ldr.w	r7, [sp], #4
 800191e:	4770      	bx	lr

08001920 <DebugMon_Handler>:

/**
  * @brief This function handles Debug monitor.
  */
void DebugMon_Handler(void)
{
 8001920:	b480      	push	{r7}
 8001922:	af00      	add	r7, sp, #0

  /* USER CODE END DebugMonitor_IRQn 0 */
  /* USER CODE BEGIN DebugMonitor_IRQn 1 */

  /* USER CODE END DebugMonitor_IRQn 1 */
}
 8001924:	bf00      	nop
 8001926:	46bd      	mov	sp, r7
 8001928:	f85d 7b04 	ldr.w	r7, [sp], #4
 800192c:	4770      	bx	lr

0800192e <PendSV_Handler>:

/**
  * @brief This function handles Pendable request for system service.
  */
void PendSV_Handler(void)
{
 800192e:	b480      	push	{r7}
 8001930:	af00      	add	r7, sp, #0

  /* USER CODE END PendSV_IRQn 0 */
  /* USER CODE BEGIN PendSV_IRQn 1 */

  /* USER CODE END PendSV_IRQn 1 */
}
 8001932:	bf00      	nop
 8001934:	46bd      	mov	sp, r7
 8001936:	f85d 7b04 	ldr.w	r7, [sp], #4
 800193a:	4770      	bx	lr

0800193c <SysTick_Handler>:

/**
  * @brief This function handles System tick timer.
  */
void SysTick_Handler(void)
{
 800193c:	b580      	push	{r7, lr}
 800193e:	af00      	add	r7, sp, #0
  /* USER CODE BEGIN SysTick_IRQn 0 */

  /* USER CODE END SysTick_IRQn 0 */
  HAL_IncTick();
 8001940:	f000 f956 	bl	8001bf0 <HAL_IncTick>
  /* USER CODE BEGIN SysTick_IRQn 1 */

  /* USER CODE END SysTick_IRQn 1 */
}
 8001944:	bf00      	nop
 8001946:	bd80      	pop	{r7, pc}

08001948 <_getpid>:
void initialise_monitor_handles()
{
}

int _getpid(void)
{
 8001948:	b480      	push	{r7}
 800194a:	af00      	add	r7, sp, #0
	return 1;
 800194c:	2301      	movs	r3, #1
}
 800194e:	4618      	mov	r0, r3
 8001950:	46bd      	mov	sp, r7
 8001952:	f85d 7b04 	ldr.w	r7, [sp], #4
 8001956:	4770      	bx	lr

08001958 <_kill>:

int _kill(int pid, int sig)
{
 8001958:	b580      	push	{r7, lr}
 800195a:	b082      	sub	sp, #8
 800195c:	af00      	add	r7, sp, #0
 800195e:	6078      	str	r0, [r7, #4]
 8001960:	6039      	str	r1, [r7, #0]
	errno = EINVAL;
 8001962:	f002 fad9 	bl	8003f18 <__errno>
 8001966:	4603      	mov	r3, r0
 8001968:	2216      	movs	r2, #22
 800196a:	601a      	str	r2, [r3, #0]
	return -1;
 800196c:	f04f 33ff 	mov.w	r3, #4294967295
}
 8001970:	4618      	mov	r0, r3
 8001972:	3708      	adds	r7, #8
 8001974:	46bd      	mov	sp, r7
 8001976:	bd80      	pop	{r7, pc}

08001978 <_exit>:

void _exit (int status)
{
 8001978:	b580      	push	{r7, lr}
 800197a:	b082      	sub	sp, #8
 800197c:	af00      	add	r7, sp, #0
 800197e:	6078      	str	r0, [r7, #4]
	_kill(status, -1);
 8001980:	f04f 31ff 	mov.w	r1, #4294967295
 8001984:	6878      	ldr	r0, [r7, #4]
 8001986:	f7ff ffe7 	bl	8001958 <_kill>
	while (1) {}		/* Make sure we hang here */
 800198a:	e7fe      	b.n	800198a <_exit+0x12>

0800198c <_read>:
}

__attribute__((weak)) int _read(int file, char *ptr, int len)
{
 800198c:	b580      	push	{r7, lr}
 800198e:	b086      	sub	sp, #24
 8001990:	af00      	add	r7, sp, #0
 8001992:	60f8      	str	r0, [r7, #12]
 8001994:	60b9      	str	r1, [r7, #8]
 8001996:	607a      	str	r2, [r7, #4]
	int DataIdx;

	for (DataIdx = 0; DataIdx < len; DataIdx++)
 8001998:	2300      	movs	r3, #0
 800199a:	617b      	str	r3, [r7, #20]
 800199c:	e00a      	b.n	80019b4 <_read+0x28>
	{
		*ptr++ = __io_getchar();
 800199e:	f3af 8000 	nop.w
 80019a2:	4601      	mov	r1, r0
 80019a4:	68bb      	ldr	r3, [r7, #8]
 80019a6:	1c5a      	adds	r2, r3, #1
 80019a8:	60ba      	str	r2, [r7, #8]
 80019aa:	b2ca      	uxtb	r2, r1
 80019ac:	701a      	strb	r2, [r3, #0]
	for (DataIdx = 0; DataIdx < len; DataIdx++)
 80019ae:	697b      	ldr	r3, [r7, #20]
 80019b0:	3301      	adds	r3, #1
 80019b2:	617b      	str	r3, [r7, #20]
 80019b4:	697a      	ldr	r2, [r7, #20]
 80019b6:	687b      	ldr	r3, [r7, #4]
 80019b8:	429a      	cmp	r2, r3
 80019ba:	dbf0      	blt.n	800199e <_read+0x12>
	}

return len;
 80019bc:	687b      	ldr	r3, [r7, #4]
}
 80019be:	4618      	mov	r0, r3
 80019c0:	3718      	adds	r7, #24
 80019c2:	46bd      	mov	sp, r7
 80019c4:	bd80      	pop	{r7, pc}

080019c6 <_write>:

__attribute__((weak)) int _write(int file, char *ptr, int len)
{
 80019c6:	b580      	push	{r7, lr}
 80019c8:	b086      	sub	sp, #24
 80019ca:	af00      	add	r7, sp, #0
 80019cc:	60f8      	str	r0, [r7, #12]
 80019ce:	60b9      	str	r1, [r7, #8]
 80019d0:	607a      	str	r2, [r7, #4]
	int DataIdx;

	for (DataIdx = 0; DataIdx < len; DataIdx++)
 80019d2:	2300      	movs	r3, #0
 80019d4:	617b      	str	r3, [r7, #20]
 80019d6:	e009      	b.n	80019ec <_write+0x26>
	{
		__io_putchar(*ptr++);
 80019d8:	68bb      	ldr	r3, [r7, #8]
 80019da:	1c5a      	adds	r2, r3, #1
 80019dc:	60ba      	str	r2, [r7, #8]
 80019de:	781b      	ldrb	r3, [r3, #0]
 80019e0:	4618      	mov	r0, r3
 80019e2:	f3af 8000 	nop.w
	for (DataIdx = 0; DataIdx < len; DataIdx++)
 80019e6:	697b      	ldr	r3, [r7, #20]
 80019e8:	3301      	adds	r3, #1
 80019ea:	617b      	str	r3, [r7, #20]
 80019ec:	697a      	ldr	r2, [r7, #20]
 80019ee:	687b      	ldr	r3, [r7, #4]
 80019f0:	429a      	cmp	r2, r3
 80019f2:	dbf1      	blt.n	80019d8 <_write+0x12>
	}
	return len;
 80019f4:	687b      	ldr	r3, [r7, #4]
}
 80019f6:	4618      	mov	r0, r3
 80019f8:	3718      	adds	r7, #24
 80019fa:	46bd      	mov	sp, r7
 80019fc:	bd80      	pop	{r7, pc}

080019fe <_close>:

int _close(int file)
{
 80019fe:	b480      	push	{r7}
 8001a00:	b083      	sub	sp, #12
 8001a02:	af00      	add	r7, sp, #0
 8001a04:	6078      	str	r0, [r7, #4]
	return -1;
 8001a06:	f04f 33ff 	mov.w	r3, #4294967295
}
 8001a0a:	4618      	mov	r0, r3
 8001a0c:	370c      	adds	r7, #12
 8001a0e:	46bd      	mov	sp, r7
 8001a10:	f85d 7b04 	ldr.w	r7, [sp], #4
 8001a14:	4770      	bx	lr

08001a16 <_fstat>:


int _fstat(int file, struct stat *st)
{
 8001a16:	b480      	push	{r7}
 8001a18:	b083      	sub	sp, #12
 8001a1a:	af00      	add	r7, sp, #0
 8001a1c:	6078      	str	r0, [r7, #4]
 8001a1e:	6039      	str	r1, [r7, #0]
	st->st_mode = S_IFCHR;
 8001a20:	683b      	ldr	r3, [r7, #0]
 8001a22:	f44f 5200 	mov.w	r2, #8192	; 0x2000
 8001a26:	605a      	str	r2, [r3, #4]
	return 0;
 8001a28:	2300      	movs	r3, #0
}
 8001a2a:	4618      	mov	r0, r3
 8001a2c:	370c      	adds	r7, #12
 8001a2e:	46bd      	mov	sp, r7
 8001a30:	f85d 7b04 	ldr.w	r7, [sp], #4
 8001a34:	4770      	bx	lr

08001a36 <_isatty>:

int _isatty(int file)
{
 8001a36:	b480      	push	{r7}
 8001a38:	b083      	sub	sp, #12
 8001a3a:	af00      	add	r7, sp, #0
 8001a3c:	6078      	str	r0, [r7, #4]
	return 1;
 8001a3e:	2301      	movs	r3, #1
}
 8001a40:	4618      	mov	r0, r3
 8001a42:	370c      	adds	r7, #12
 8001a44:	46bd      	mov	sp, r7
 8001a46:	f85d 7b04 	ldr.w	r7, [sp], #4
 8001a4a:	4770      	bx	lr

08001a4c <_lseek>:

int _lseek(int file, int ptr, int dir)
{
 8001a4c:	b480      	push	{r7}
 8001a4e:	b085      	sub	sp, #20
 8001a50:	af00      	add	r7, sp, #0
 8001a52:	60f8      	str	r0, [r7, #12]
 8001a54:	60b9      	str	r1, [r7, #8]
 8001a56:	607a      	str	r2, [r7, #4]
	return 0;
 8001a58:	2300      	movs	r3, #0
}
 8001a5a:	4618      	mov	r0, r3
 8001a5c:	3714      	adds	r7, #20
 8001a5e:	46bd      	mov	sp, r7
 8001a60:	f85d 7b04 	ldr.w	r7, [sp], #4
 8001a64:	4770      	bx	lr
	...

08001a68 <_sbrk>:
 *
 * @param incr Memory size
 * @return Pointer to allocated memory
 */
void *_sbrk(ptrdiff_t incr)
{
 8001a68:	b580      	push	{r7, lr}
 8001a6a:	b086      	sub	sp, #24
 8001a6c:	af00      	add	r7, sp, #0
 8001a6e:	6078      	str	r0, [r7, #4]
  extern uint8_t _end; /* Symbol defined in the linker script */
  extern uint8_t _estack; /* Symbol defined in the linker script */
  extern uint32_t _Min_Stack_Size; /* Symbol defined in the linker script */
  const uint32_t stack_limit = (uint32_t)&_estack - (uint32_t)&_Min_Stack_Size;
 8001a70:	4a14      	ldr	r2, [pc, #80]	; (8001ac4 <_sbrk+0x5c>)
 8001a72:	4b15      	ldr	r3, [pc, #84]	; (8001ac8 <_sbrk+0x60>)
 8001a74:	1ad3      	subs	r3, r2, r3
 8001a76:	617b      	str	r3, [r7, #20]
  const uint8_t *max_heap = (uint8_t *)stack_limit;
 8001a78:	697b      	ldr	r3, [r7, #20]
 8001a7a:	613b      	str	r3, [r7, #16]
  uint8_t *prev_heap_end;

  /* Initialize heap end at first call */
  if (NULL == __sbrk_heap_end)
 8001a7c:	4b13      	ldr	r3, [pc, #76]	; (8001acc <_sbrk+0x64>)
 8001a7e:	681b      	ldr	r3, [r3, #0]
 8001a80:	2b00      	cmp	r3, #0
 8001a82:	d102      	bne.n	8001a8a <_sbrk+0x22>
  {
    __sbrk_heap_end = &_end;
 8001a84:	4b11      	ldr	r3, [pc, #68]	; (8001acc <_sbrk+0x64>)
 8001a86:	4a12      	ldr	r2, [pc, #72]	; (8001ad0 <_sbrk+0x68>)
 8001a88:	601a      	str	r2, [r3, #0]
  }

  /* Protect heap from growing into the reserved MSP stack */
  if (__sbrk_heap_end + incr > max_heap)
 8001a8a:	4b10      	ldr	r3, [pc, #64]	; (8001acc <_sbrk+0x64>)
 8001a8c:	681a      	ldr	r2, [r3, #0]
 8001a8e:	687b      	ldr	r3, [r7, #4]
 8001a90:	4413      	add	r3, r2
 8001a92:	693a      	ldr	r2, [r7, #16]
 8001a94:	429a      	cmp	r2, r3
 8001a96:	d207      	bcs.n	8001aa8 <_sbrk+0x40>
  {
    errno = ENOMEM;
 8001a98:	f002 fa3e 	bl	8003f18 <__errno>
 8001a9c:	4603      	mov	r3, r0
 8001a9e:	220c      	movs	r2, #12
 8001aa0:	601a      	str	r2, [r3, #0]
    return (void *)-1;
 8001aa2:	f04f 33ff 	mov.w	r3, #4294967295
 8001aa6:	e009      	b.n	8001abc <_sbrk+0x54>
  }

  prev_heap_end = __sbrk_heap_end;
 8001aa8:	4b08      	ldr	r3, [pc, #32]	; (8001acc <_sbrk+0x64>)
 8001aaa:	681b      	ldr	r3, [r3, #0]
 8001aac:	60fb      	str	r3, [r7, #12]
  __sbrk_heap_end += incr;
 8001aae:	4b07      	ldr	r3, [pc, #28]	; (8001acc <_sbrk+0x64>)
 8001ab0:	681a      	ldr	r2, [r3, #0]
 8001ab2:	687b      	ldr	r3, [r7, #4]
 8001ab4:	4413      	add	r3, r2
 8001ab6:	4a05      	ldr	r2, [pc, #20]	; (8001acc <_sbrk+0x64>)
 8001ab8:	6013      	str	r3, [r2, #0]

  return (void *)prev_heap_end;
 8001aba:	68fb      	ldr	r3, [r7, #12]
}
 8001abc:	4618      	mov	r0, r3
 8001abe:	3718      	adds	r7, #24
 8001ac0:	46bd      	mov	sp, r7
 8001ac2:	bd80      	pop	{r7, pc}
 8001ac4:	20030000 	.word	0x20030000
 8001ac8:	00000400 	.word	0x00000400
 8001acc:	20000294 	.word	0x20000294
 8001ad0:	200002b0 	.word	0x200002b0

08001ad4 <SystemInit>:
  *         configuration.
  * @param  None
  * @retval None
  */
void SystemInit(void)
{
 8001ad4:	b480      	push	{r7}
 8001ad6:	af00      	add	r7, sp, #0
  /* FPU settings ------------------------------------------------------------*/
  #if (__FPU_PRESENT == 1) && (__FPU_USED == 1)
    SCB->CPACR |= ((3UL << 10*2)|(3UL << 11*2));  /* set CP10 and CP11 Full Access */
 8001ad8:	4b06      	ldr	r3, [pc, #24]	; (8001af4 <SystemInit+0x20>)
 8001ada:	f8d3 3088 	ldr.w	r3, [r3, #136]	; 0x88
 8001ade:	4a05      	ldr	r2, [pc, #20]	; (8001af4 <SystemInit+0x20>)
 8001ae0:	f443 0370 	orr.w	r3, r3, #15728640	; 0xf00000
 8001ae4:	f8c2 3088 	str.w	r3, [r2, #136]	; 0x88

  /* Configure the Vector Table location -------------------------------------*/
#if defined(USER_VECT_TAB_ADDRESS)
  SCB->VTOR = VECT_TAB_BASE_ADDRESS | VECT_TAB_OFFSET; /* Vector Table Relocation in Internal SRAM */
#endif /* USER_VECT_TAB_ADDRESS */
}
 8001ae8:	bf00      	nop
 8001aea:	46bd      	mov	sp, r7
 8001aec:	f85d 7b04 	ldr.w	r7, [sp], #4
 8001af0:	4770      	bx	lr
 8001af2:	bf00      	nop
 8001af4:	e000ed00 	.word	0xe000ed00

08001af8 <Reset_Handler>:

    .section  .text.Reset_Handler
  .weak  Reset_Handler
  .type  Reset_Handler, %function
Reset_Handler: 
  ldr   sp, =_estack       /* set stack pointer */
 8001af8:	f8df d034 	ldr.w	sp, [pc, #52]	; 8001b30 <LoopFillZerobss+0x12>
 
/* Copy the data segment initializers from flash to SRAM */  
  ldr r0, =_sdata
 8001afc:	480d      	ldr	r0, [pc, #52]	; (8001b34 <LoopFillZerobss+0x16>)
  ldr r1, =_edata
 8001afe:	490e      	ldr	r1, [pc, #56]	; (8001b38 <LoopFillZerobss+0x1a>)
  ldr r2, =_sidata
 8001b00:	4a0e      	ldr	r2, [pc, #56]	; (8001b3c <LoopFillZerobss+0x1e>)
  movs r3, #0
 8001b02:	2300      	movs	r3, #0
  b LoopCopyDataInit
 8001b04:	e002      	b.n	8001b0c <LoopCopyDataInit>

08001b06 <CopyDataInit>:

CopyDataInit:
  ldr r4, [r2, r3]
 8001b06:	58d4      	ldr	r4, [r2, r3]
  str r4, [r0, r3]
 8001b08:	50c4      	str	r4, [r0, r3]
  adds r3, r3, #4
 8001b0a:	3304      	adds	r3, #4

08001b0c <LoopCopyDataInit>:

LoopCopyDataInit:
  adds r4, r0, r3
 8001b0c:	18c4      	adds	r4, r0, r3
  cmp r4, r1
 8001b0e:	428c      	cmp	r4, r1
  bcc CopyDataInit
 8001b10:	d3f9      	bcc.n	8001b06 <CopyDataInit>
  
/* Zero fill the bss segment. */
  ldr r2, =_sbss
 8001b12:	4a0b      	ldr	r2, [pc, #44]	; (8001b40 <LoopFillZerobss+0x22>)
  ldr r4, =_ebss
 8001b14:	4c0b      	ldr	r4, [pc, #44]	; (8001b44 <LoopFillZerobss+0x26>)
  movs r3, #0
 8001b16:	2300      	movs	r3, #0
  b LoopFillZerobss
 8001b18:	e001      	b.n	8001b1e <LoopFillZerobss>

08001b1a <FillZerobss>:

FillZerobss:
  str  r3, [r2]
 8001b1a:	6013      	str	r3, [r2, #0]
  adds r2, r2, #4
 8001b1c:	3204      	adds	r2, #4

08001b1e <LoopFillZerobss>:

LoopFillZerobss:
  cmp r2, r4
 8001b1e:	42a2      	cmp	r2, r4
  bcc FillZerobss
 8001b20:	d3fb      	bcc.n	8001b1a <FillZerobss>

/* Call the clock system initialization function.*/
  bl  SystemInit   
 8001b22:	f7ff ffd7 	bl	8001ad4 <SystemInit>
/* Call static constructors */
    bl __libc_init_array
 8001b26:	f002 f9fd 	bl	8003f24 <__libc_init_array>
/* Call the application's entry point.*/
  bl  main
 8001b2a:	f7ff fa1f 	bl	8000f6c <main>
  bx  lr    
 8001b2e:	4770      	bx	lr
  ldr   sp, =_estack       /* set stack pointer */
 8001b30:	20030000 	.word	0x20030000
  ldr r0, =_sdata
 8001b34:	20000000 	.word	0x20000000
  ldr r1, =_edata
 8001b38:	200001dc 	.word	0x200001dc
  ldr r2, =_sidata
 8001b3c:	0800723c 	.word	0x0800723c
  ldr r2, =_sbss
 8001b40:	200001dc 	.word	0x200001dc
  ldr r4, =_ebss
 8001b44:	200002ac 	.word	0x200002ac

08001b48 <ADC_IRQHandler>:
 * @retval None       
*/
    .section  .text.Default_Handler,"ax",%progbits
Default_Handler:
Infinite_Loop:
  b  Infinite_Loop
 8001b48:	e7fe      	b.n	8001b48 <ADC_IRQHandler>
	...

08001b4c <HAL_Init>:
  *         need to ensure that the SysTick time base is always set to 1 millisecond
  *         to have correct HAL operation.
  * @retval HAL status
  */
HAL_StatusTypeDef HAL_Init(void)
{
 8001b4c:	b580      	push	{r7, lr}
 8001b4e:	af00      	add	r7, sp, #0
  /* Configure Flash prefetch, Instruction cache, Data cache */ 
#if (INSTRUCTION_CACHE_ENABLE != 0U)
  __HAL_FLASH_INSTRUCTION_CACHE_ENABLE();
 8001b50:	4b0e      	ldr	r3, [pc, #56]	; (8001b8c <HAL_Init+0x40>)
 8001b52:	681b      	ldr	r3, [r3, #0]
 8001b54:	4a0d      	ldr	r2, [pc, #52]	; (8001b8c <HAL_Init+0x40>)
 8001b56:	f443 7300 	orr.w	r3, r3, #512	; 0x200
 8001b5a:	6013      	str	r3, [r2, #0]
#endif /* INSTRUCTION_CACHE_ENABLE */

#if (DATA_CACHE_ENABLE != 0U)
  __HAL_FLASH_DATA_CACHE_ENABLE();
 8001b5c:	4b0b      	ldr	r3, [pc, #44]	; (8001b8c <HAL_Init+0x40>)
 8001b5e:	681b      	ldr	r3, [r3, #0]
 8001b60:	4a0a      	ldr	r2, [pc, #40]	; (8001b8c <HAL_Init+0x40>)
 8001b62:	f443 6380 	orr.w	r3, r3, #1024	; 0x400
 8001b66:	6013      	str	r3, [r2, #0]
#endif /* DATA_CACHE_ENABLE */

#if (PREFETCH_ENABLE != 0U)
  __HAL_FLASH_PREFETCH_BUFFER_ENABLE();
 8001b68:	4b08      	ldr	r3, [pc, #32]	; (8001b8c <HAL_Init+0x40>)
 8001b6a:	681b      	ldr	r3, [r3, #0]
 8001b6c:	4a07      	ldr	r2, [pc, #28]	; (8001b8c <HAL_Init+0x40>)
 8001b6e:	f443 7380 	orr.w	r3, r3, #256	; 0x100
 8001b72:	6013      	str	r3, [r2, #0]
#endif /* PREFETCH_ENABLE */

  /* Set Interrupt Group Priority */
  HAL_NVIC_SetPriorityGrouping(NVIC_PRIORITYGROUP_4);
 8001b74:	2003      	movs	r0, #3
 8001b76:	f000 f931 	bl	8001ddc <HAL_NVIC_SetPriorityGrouping>

  /* Use systick as time base source and configure 1ms tick (default clock after Reset is HSI) */
  HAL_InitTick(TICK_INT_PRIORITY);
 8001b7a:	2000      	movs	r0, #0
 8001b7c:	f000 f808 	bl	8001b90 <HAL_InitTick>

  /* Init the low level hardware */
  HAL_MspInit();
 8001b80:	f7ff fe00 	bl	8001784 <HAL_MspInit>

  /* Return function status */
  return HAL_OK;
 8001b84:	2300      	movs	r3, #0
}
 8001b86:	4618      	mov	r0, r3
 8001b88:	bd80      	pop	{r7, pc}
 8001b8a:	bf00      	nop
 8001b8c:	40023c00 	.word	0x40023c00

08001b90 <HAL_InitTick>:
  *       implementation  in user file.
  * @param TickPriority Tick interrupt priority.
  * @retval HAL status
  */
__weak HAL_StatusTypeDef HAL_InitTick(uint32_t TickPriority)
{
 8001b90:	b580      	push	{r7, lr}
 8001b92:	b082      	sub	sp, #8
 8001b94:	af00      	add	r7, sp, #0
 8001b96:	6078      	str	r0, [r7, #4]
  /* Configure the SysTick to have interrupt in 1ms time basis*/
  if (HAL_SYSTICK_Config(SystemCoreClock / (1000U / uwTickFreq)) > 0U)
 8001b98:	4b12      	ldr	r3, [pc, #72]	; (8001be4 <HAL_InitTick+0x54>)
 8001b9a:	681a      	ldr	r2, [r3, #0]
 8001b9c:	4b12      	ldr	r3, [pc, #72]	; (8001be8 <HAL_InitTick+0x58>)
 8001b9e:	781b      	ldrb	r3, [r3, #0]
 8001ba0:	4619      	mov	r1, r3
 8001ba2:	f44f 737a 	mov.w	r3, #1000	; 0x3e8
 8001ba6:	fbb3 f3f1 	udiv	r3, r3, r1
 8001baa:	fbb2 f3f3 	udiv	r3, r2, r3
 8001bae:	4618      	mov	r0, r3
 8001bb0:	f000 f93b 	bl	8001e2a <HAL_SYSTICK_Config>
 8001bb4:	4603      	mov	r3, r0
 8001bb6:	2b00      	cmp	r3, #0
 8001bb8:	d001      	beq.n	8001bbe <HAL_InitTick+0x2e>
  {
    return HAL_ERROR;
 8001bba:	2301      	movs	r3, #1
 8001bbc:	e00e      	b.n	8001bdc <HAL_InitTick+0x4c>
  }

  /* Configure the SysTick IRQ priority */
  if (TickPriority < (1UL << __NVIC_PRIO_BITS))
 8001bbe:	687b      	ldr	r3, [r7, #4]
 8001bc0:	2b0f      	cmp	r3, #15
 8001bc2:	d80a      	bhi.n	8001bda <HAL_InitTick+0x4a>
  {
    HAL_NVIC_SetPriority(SysTick_IRQn, TickPriority, 0U);
 8001bc4:	2200      	movs	r2, #0
 8001bc6:	6879      	ldr	r1, [r7, #4]
 8001bc8:	f04f 30ff 	mov.w	r0, #4294967295
 8001bcc:	f000 f911 	bl	8001df2 <HAL_NVIC_SetPriority>
    uwTickPrio = TickPriority;
 8001bd0:	4a06      	ldr	r2, [pc, #24]	; (8001bec <HAL_InitTick+0x5c>)
 8001bd2:	687b      	ldr	r3, [r7, #4]
 8001bd4:	6013      	str	r3, [r2, #0]
  {
    return HAL_ERROR;
  }

  /* Return function status */
  return HAL_OK;
 8001bd6:	2300      	movs	r3, #0
 8001bd8:	e000      	b.n	8001bdc <HAL_InitTick+0x4c>
    return HAL_ERROR;
 8001bda:	2301      	movs	r3, #1
}
 8001bdc:	4618      	mov	r0, r3
 8001bde:	3708      	adds	r7, #8
 8001be0:	46bd      	mov	sp, r7
 8001be2:	bd80      	pop	{r7, pc}
 8001be4:	20000000 	.word	0x20000000
 8001be8:	20000008 	.word	0x20000008
 8001bec:	20000004 	.word	0x20000004

08001bf0 <HAL_IncTick>:
 * @note This function is declared as __weak to be overwritten in case of other 
  *      implementations in user file.
  * @retval None
  */
__weak void HAL_IncTick(void)
{
 8001bf0:	b480      	push	{r7}
 8001bf2:	af00      	add	r7, sp, #0
  uwTick += uwTickFreq;
 8001bf4:	4b06      	ldr	r3, [pc, #24]	; (8001c10 <HAL_IncTick+0x20>)
 8001bf6:	781b      	ldrb	r3, [r3, #0]
 8001bf8:	461a      	mov	r2, r3
 8001bfa:	4b06      	ldr	r3, [pc, #24]	; (8001c14 <HAL_IncTick+0x24>)
 8001bfc:	681b      	ldr	r3, [r3, #0]
 8001bfe:	4413      	add	r3, r2
 8001c00:	4a04      	ldr	r2, [pc, #16]	; (8001c14 <HAL_IncTick+0x24>)
 8001c02:	6013      	str	r3, [r2, #0]
}
 8001c04:	bf00      	nop
 8001c06:	46bd      	mov	sp, r7
 8001c08:	f85d 7b04 	ldr.w	r7, [sp], #4
 8001c0c:	4770      	bx	lr
 8001c0e:	bf00      	nop
 8001c10:	20000008 	.word	0x20000008
 8001c14:	20000298 	.word	0x20000298

08001c18 <HAL_GetTick>:
  * @note This function is declared as __weak to be overwritten in case of other 
  *       implementations in user file.
  * @retval tick value
  */
__weak uint32_t HAL_GetTick(void)
{
 8001c18:	b480      	push	{r7}
 8001c1a:	af00      	add	r7, sp, #0
  return uwTick;
 8001c1c:	4b03      	ldr	r3, [pc, #12]	; (8001c2c <HAL_GetTick+0x14>)
 8001c1e:	681b      	ldr	r3, [r3, #0]
}
 8001c20:	4618      	mov	r0, r3
 8001c22:	46bd      	mov	sp, r7
 8001c24:	f85d 7b04 	ldr.w	r7, [sp], #4
 8001c28:	4770      	bx	lr
 8001c2a:	bf00      	nop
 8001c2c:	20000298 	.word	0x20000298

08001c30 <HAL_Delay>:
  *       implementations in user file.
  * @param Delay specifies the delay time length, in milliseconds.
  * @retval None
  */
__weak void HAL_Delay(uint32_t Delay)
{
 8001c30:	b580      	push	{r7, lr}
 8001c32:	b084      	sub	sp, #16
 8001c34:	af00      	add	r7, sp, #0
 8001c36:	6078      	str	r0, [r7, #4]
  uint32_t tickstart = HAL_GetTick();
 8001c38:	f7ff ffee 	bl	8001c18 <HAL_GetTick>
 8001c3c:	60b8      	str	r0, [r7, #8]
  uint32_t wait = Delay;
 8001c3e:	687b      	ldr	r3, [r7, #4]
 8001c40:	60fb      	str	r3, [r7, #12]

  /* Add a freq to guarantee minimum wait */
  if (wait < HAL_MAX_DELAY)
 8001c42:	68fb      	ldr	r3, [r7, #12]
 8001c44:	f1b3 3fff 	cmp.w	r3, #4294967295
 8001c48:	d005      	beq.n	8001c56 <HAL_Delay+0x26>
  {
    wait += (uint32_t)(uwTickFreq);
 8001c4a:	4b0a      	ldr	r3, [pc, #40]	; (8001c74 <HAL_Delay+0x44>)
 8001c4c:	781b      	ldrb	r3, [r3, #0]
 8001c4e:	461a      	mov	r2, r3
 8001c50:	68fb      	ldr	r3, [r7, #12]
 8001c52:	4413      	add	r3, r2
 8001c54:	60fb      	str	r3, [r7, #12]
  }

  while((HAL_GetTick() - tickstart) < wait)
 8001c56:	bf00      	nop
 8001c58:	f7ff ffde 	bl	8001c18 <HAL_GetTick>
 8001c5c:	4602      	mov	r2, r0
 8001c5e:	68bb      	ldr	r3, [r7, #8]
 8001c60:	1ad3      	subs	r3, r2, r3
 8001c62:	68fa      	ldr	r2, [r7, #12]
 8001c64:	429a      	cmp	r2, r3
 8001c66:	d8f7      	bhi.n	8001c58 <HAL_Delay+0x28>
  {
  }
}
 8001c68:	bf00      	nop
 8001c6a:	bf00      	nop
 8001c6c:	3710      	adds	r7, #16
 8001c6e:	46bd      	mov	sp, r7
 8001c70:	bd80      	pop	{r7, pc}
 8001c72:	bf00      	nop
 8001c74:	20000008 	.word	0x20000008

08001c78 <__NVIC_SetPriorityGrouping>:
           In case of a conflict between priority grouping and available
           priority bits (__NVIC_PRIO_BITS), the smallest possible priority group is set.
  \param [in]      PriorityGroup  Priority grouping field.
 */
__STATIC_INLINE void __NVIC_SetPriorityGrouping(uint32_t PriorityGroup)
{
 8001c78:	b480      	push	{r7}
 8001c7a:	b085      	sub	sp, #20
 8001c7c:	af00      	add	r7, sp, #0
 8001c7e:	6078      	str	r0, [r7, #4]
  uint32_t reg_value;
  uint32_t PriorityGroupTmp = (PriorityGroup & (uint32_t)0x07UL);             /* only values 0..7 are used          */
 8001c80:	687b      	ldr	r3, [r7, #4]
 8001c82:	f003 0307 	and.w	r3, r3, #7
 8001c86:	60fb      	str	r3, [r7, #12]

  reg_value  =  SCB->AIRCR;                                                   /* read old register configuration    */
 8001c88:	4b0c      	ldr	r3, [pc, #48]	; (8001cbc <__NVIC_SetPriorityGrouping+0x44>)
 8001c8a:	68db      	ldr	r3, [r3, #12]
 8001c8c:	60bb      	str	r3, [r7, #8]
  reg_value &= ~((uint32_t)(SCB_AIRCR_VECTKEY_Msk | SCB_AIRCR_PRIGROUP_Msk)); /* clear bits to change               */
 8001c8e:	68ba      	ldr	r2, [r7, #8]
 8001c90:	f64f 03ff 	movw	r3, #63743	; 0xf8ff
 8001c94:	4013      	ands	r3, r2
 8001c96:	60bb      	str	r3, [r7, #8]
  reg_value  =  (reg_value                                   |
                ((uint32_t)0x5FAUL << SCB_AIRCR_VECTKEY_Pos) |
                (PriorityGroupTmp << SCB_AIRCR_PRIGROUP_Pos)  );              /* Insert write key and priority group */
 8001c98:	68fb      	ldr	r3, [r7, #12]
 8001c9a:	021a      	lsls	r2, r3, #8
                ((uint32_t)0x5FAUL << SCB_AIRCR_VECTKEY_Pos) |
 8001c9c:	68bb      	ldr	r3, [r7, #8]
 8001c9e:	4313      	orrs	r3, r2
  reg_value  =  (reg_value                                   |
 8001ca0:	f043 63bf 	orr.w	r3, r3, #100139008	; 0x5f80000
 8001ca4:	f443 3300 	orr.w	r3, r3, #131072	; 0x20000
 8001ca8:	60bb      	str	r3, [r7, #8]
  SCB->AIRCR =  reg_value;
 8001caa:	4a04      	ldr	r2, [pc, #16]	; (8001cbc <__NVIC_SetPriorityGrouping+0x44>)
 8001cac:	68bb      	ldr	r3, [r7, #8]
 8001cae:	60d3      	str	r3, [r2, #12]
}
 8001cb0:	bf00      	nop
 8001cb2:	3714      	adds	r7, #20
 8001cb4:	46bd      	mov	sp, r7
 8001cb6:	f85d 7b04 	ldr.w	r7, [sp], #4
 8001cba:	4770      	bx	lr
 8001cbc:	e000ed00 	.word	0xe000ed00

08001cc0 <__NVIC_GetPriorityGrouping>:
  \brief   Get Priority Grouping
  \details Reads the priority grouping field from the NVIC Interrupt Controller.
  \return                Priority grouping field (SCB->AIRCR [10:8] PRIGROUP field).
 */
__STATIC_INLINE uint32_t __NVIC_GetPriorityGrouping(void)
{
 8001cc0:	b480      	push	{r7}
 8001cc2:	af00      	add	r7, sp, #0
  return ((uint32_t)((SCB->AIRCR & SCB_AIRCR_PRIGROUP_Msk) >> SCB_AIRCR_PRIGROUP_Pos));
 8001cc4:	4b04      	ldr	r3, [pc, #16]	; (8001cd8 <__NVIC_GetPriorityGrouping+0x18>)
 8001cc6:	68db      	ldr	r3, [r3, #12]
 8001cc8:	0a1b      	lsrs	r3, r3, #8
 8001cca:	f003 0307 	and.w	r3, r3, #7
}
 8001cce:	4618      	mov	r0, r3
 8001cd0:	46bd      	mov	sp, r7
 8001cd2:	f85d 7b04 	ldr.w	r7, [sp], #4
 8001cd6:	4770      	bx	lr
 8001cd8:	e000ed00 	.word	0xe000ed00

08001cdc <__NVIC_SetPriority>:
  \param [in]      IRQn  Interrupt number.
  \param [in]  priority  Priority to set.
  \note    The priority cannot be set for every processor exception.
 */
__STATIC_INLINE void __NVIC_SetPriority(IRQn_Type IRQn, uint32_t priority)
{
 8001cdc:	b480      	push	{r7}
 8001cde:	b083      	sub	sp, #12
 8001ce0:	af00      	add	r7, sp, #0
 8001ce2:	4603      	mov	r3, r0
 8001ce4:	6039      	str	r1, [r7, #0]
 8001ce6:	71fb      	strb	r3, [r7, #7]
  if ((int32_t)(IRQn) >= 0)
 8001ce8:	f997 3007 	ldrsb.w	r3, [r7, #7]
 8001cec:	2b00      	cmp	r3, #0
 8001cee:	db0a      	blt.n	8001d06 <__NVIC_SetPriority+0x2a>
  {
    NVIC->IP[((uint32_t)IRQn)]               = (uint8_t)((priority << (8U - __NVIC_PRIO_BITS)) & (uint32_t)0xFFUL);
 8001cf0:	683b      	ldr	r3, [r7, #0]
 8001cf2:	b2da      	uxtb	r2, r3
 8001cf4:	490c      	ldr	r1, [pc, #48]	; (8001d28 <__NVIC_SetPriority+0x4c>)
 8001cf6:	f997 3007 	ldrsb.w	r3, [r7, #7]
 8001cfa:	0112      	lsls	r2, r2, #4
 8001cfc:	b2d2      	uxtb	r2, r2
 8001cfe:	440b      	add	r3, r1
 8001d00:	f883 2300 	strb.w	r2, [r3, #768]	; 0x300
  }
  else
  {
    SCB->SHP[(((uint32_t)IRQn) & 0xFUL)-4UL] = (uint8_t)((priority << (8U - __NVIC_PRIO_BITS)) & (uint32_t)0xFFUL);
  }
}
 8001d04:	e00a      	b.n	8001d1c <__NVIC_SetPriority+0x40>
    SCB->SHP[(((uint32_t)IRQn) & 0xFUL)-4UL] = (uint8_t)((priority << (8U - __NVIC_PRIO_BITS)) & (uint32_t)0xFFUL);
 8001d06:	683b      	ldr	r3, [r7, #0]
 8001d08:	b2da      	uxtb	r2, r3
 8001d0a:	4908      	ldr	r1, [pc, #32]	; (8001d2c <__NVIC_SetPriority+0x50>)
 8001d0c:	79fb      	ldrb	r3, [r7, #7]
 8001d0e:	f003 030f 	and.w	r3, r3, #15
 8001d12:	3b04      	subs	r3, #4
 8001d14:	0112      	lsls	r2, r2, #4
 8001d16:	b2d2      	uxtb	r2, r2
 8001d18:	440b      	add	r3, r1
 8001d1a:	761a      	strb	r2, [r3, #24]
}
 8001d1c:	bf00      	nop
 8001d1e:	370c      	adds	r7, #12
 8001d20:	46bd      	mov	sp, r7
 8001d22:	f85d 7b04 	ldr.w	r7, [sp], #4
 8001d26:	4770      	bx	lr
 8001d28:	e000e100 	.word	0xe000e100
 8001d2c:	e000ed00 	.word	0xe000ed00

08001d30 <NVIC_EncodePriority>:
  \param [in]   PreemptPriority  Preemptive priority value (starting from 0).
  \param [in]       SubPriority  Subpriority value (starting from 0).
  \return                        Encoded priority. Value can be used in the function \ref NVIC_SetPriority().
 */
__STATIC_INLINE uint32_t NVIC_EncodePriority (uint32_t PriorityGroup, uint32_t PreemptPriority, uint32_t SubPriority)
{
 8001d30:	b480      	push	{r7}
 8001d32:	b089      	sub	sp, #36	; 0x24
 8001d34:	af00      	add	r7, sp, #0
 8001d36:	60f8      	str	r0, [r7, #12]
 8001d38:	60b9      	str	r1, [r7, #8]
 8001d3a:	607a      	str	r2, [r7, #4]
  uint32_t PriorityGroupTmp = (PriorityGroup & (uint32_t)0x07UL);   /* only values 0..7 are used          */
 8001d3c:	68fb      	ldr	r3, [r7, #12]
 8001d3e:	f003 0307 	and.w	r3, r3, #7
 8001d42:	61fb      	str	r3, [r7, #28]
  uint32_t PreemptPriorityBits;
  uint32_t SubPriorityBits;

  PreemptPriorityBits = ((7UL - PriorityGroupTmp) > (uint32_t)(__NVIC_PRIO_BITS)) ? (uint32_t)(__NVIC_PRIO_BITS) : (uint32_t)(7UL - PriorityGroupTmp);
 8001d44:	69fb      	ldr	r3, [r7, #28]
 8001d46:	f1c3 0307 	rsb	r3, r3, #7
 8001d4a:	2b04      	cmp	r3, #4
 8001d4c:	bf28      	it	cs
 8001d4e:	2304      	movcs	r3, #4
 8001d50:	61bb      	str	r3, [r7, #24]
  SubPriorityBits     = ((PriorityGroupTmp + (uint32_t)(__NVIC_PRIO_BITS)) < (uint32_t)7UL) ? (uint32_t)0UL : (uint32_t)((PriorityGroupTmp - 7UL) + (uint32_t)(__NVIC_PRIO_BITS));
 8001d52:	69fb      	ldr	r3, [r7, #28]
 8001d54:	3304      	adds	r3, #4
 8001d56:	2b06      	cmp	r3, #6
 8001d58:	d902      	bls.n	8001d60 <NVIC_EncodePriority+0x30>
 8001d5a:	69fb      	ldr	r3, [r7, #28]
 8001d5c:	3b03      	subs	r3, #3
 8001d5e:	e000      	b.n	8001d62 <NVIC_EncodePriority+0x32>
 8001d60:	2300      	movs	r3, #0
 8001d62:	617b      	str	r3, [r7, #20]

  return (
           ((PreemptPriority & (uint32_t)((1UL << (PreemptPriorityBits)) - 1UL)) << SubPriorityBits) |
 8001d64:	f04f 32ff 	mov.w	r2, #4294967295
 8001d68:	69bb      	ldr	r3, [r7, #24]
 8001d6a:	fa02 f303 	lsl.w	r3, r2, r3
 8001d6e:	43da      	mvns	r2, r3
 8001d70:	68bb      	ldr	r3, [r7, #8]
 8001d72:	401a      	ands	r2, r3
 8001d74:	697b      	ldr	r3, [r7, #20]
 8001d76:	409a      	lsls	r2, r3
           ((SubPriority     & (uint32_t)((1UL << (SubPriorityBits    )) - 1UL)))
 8001d78:	f04f 31ff 	mov.w	r1, #4294967295
 8001d7c:	697b      	ldr	r3, [r7, #20]
 8001d7e:	fa01 f303 	lsl.w	r3, r1, r3
 8001d82:	43d9      	mvns	r1, r3
 8001d84:	687b      	ldr	r3, [r7, #4]
 8001d86:	400b      	ands	r3, r1
           ((PreemptPriority & (uint32_t)((1UL << (PreemptPriorityBits)) - 1UL)) << SubPriorityBits) |
 8001d88:	4313      	orrs	r3, r2
         );
}
 8001d8a:	4618      	mov	r0, r3
 8001d8c:	3724      	adds	r7, #36	; 0x24
 8001d8e:	46bd      	mov	sp, r7
 8001d90:	f85d 7b04 	ldr.w	r7, [sp], #4
 8001d94:	4770      	bx	lr
	...

08001d98 <SysTick_Config>:
  \note    When the variable <b>__Vendor_SysTickConfig</b> is set to 1, then the
           function <b>SysTick_Config</b> is not included. In this case, the file <b><i>device</i>.h</b>
           must contain a vendor-specific implementation of this function.
 */
__STATIC_INLINE uint32_t SysTick_Config(uint32_t ticks)
{
 8001d98:	b580      	push	{r7, lr}
 8001d9a:	b082      	sub	sp, #8
 8001d9c:	af00      	add	r7, sp, #0
 8001d9e:	6078      	str	r0, [r7, #4]
  if ((ticks - 1UL) > SysTick_LOAD_RELOAD_Msk)
 8001da0:	687b      	ldr	r3, [r7, #4]
 8001da2:	3b01      	subs	r3, #1
 8001da4:	f1b3 7f80 	cmp.w	r3, #16777216	; 0x1000000
 8001da8:	d301      	bcc.n	8001dae <SysTick_Config+0x16>
  {
    return (1UL);                                                   /* Reload value impossible */
 8001daa:	2301      	movs	r3, #1
 8001dac:	e00f      	b.n	8001dce <SysTick_Config+0x36>
  }

  SysTick->LOAD  = (uint32_t)(ticks - 1UL);                         /* set reload register */
 8001dae:	4a0a      	ldr	r2, [pc, #40]	; (8001dd8 <SysTick_Config+0x40>)
 8001db0:	687b      	ldr	r3, [r7, #4]
 8001db2:	3b01      	subs	r3, #1
 8001db4:	6053      	str	r3, [r2, #4]
  NVIC_SetPriority (SysTick_IRQn, (1UL << __NVIC_PRIO_BITS) - 1UL); /* set Priority for Systick Interrupt */
 8001db6:	210f      	movs	r1, #15
 8001db8:	f04f 30ff 	mov.w	r0, #4294967295
 8001dbc:	f7ff ff8e 	bl	8001cdc <__NVIC_SetPriority>
  SysTick->VAL   = 0UL;                                             /* Load the SysTick Counter Value */
 8001dc0:	4b05      	ldr	r3, [pc, #20]	; (8001dd8 <SysTick_Config+0x40>)
 8001dc2:	2200      	movs	r2, #0
 8001dc4:	609a      	str	r2, [r3, #8]
  SysTick->CTRL  = SysTick_CTRL_CLKSOURCE_Msk |
 8001dc6:	4b04      	ldr	r3, [pc, #16]	; (8001dd8 <SysTick_Config+0x40>)
 8001dc8:	2207      	movs	r2, #7
 8001dca:	601a      	str	r2, [r3, #0]
                   SysTick_CTRL_TICKINT_Msk   |
                   SysTick_CTRL_ENABLE_Msk;                         /* Enable SysTick IRQ and SysTick Timer */
  return (0UL);                                                     /* Function successful */
 8001dcc:	2300      	movs	r3, #0
}
 8001dce:	4618      	mov	r0, r3
 8001dd0:	3708      	adds	r7, #8
 8001dd2:	46bd      	mov	sp, r7
 8001dd4:	bd80      	pop	{r7, pc}
 8001dd6:	bf00      	nop
 8001dd8:	e000e010 	.word	0xe000e010

08001ddc <HAL_NVIC_SetPriorityGrouping>:
  * @note   When the NVIC_PriorityGroup_0 is selected, IRQ preemption is no more possible. 
  *         The pending IRQ priority will be managed only by the subpriority. 
  * @retval None
  */
void HAL_NVIC_SetPriorityGrouping(uint32_t PriorityGroup)
{
 8001ddc:	b580      	push	{r7, lr}
 8001dde:	b082      	sub	sp, #8
 8001de0:	af00      	add	r7, sp, #0
 8001de2:	6078      	str	r0, [r7, #4]
  /* Check the parameters */
  assert_param(IS_NVIC_PRIORITY_GROUP(PriorityGroup));
  
  /* Set the PRIGROUP[10:8] bits according to the PriorityGroup parameter value */
  NVIC_SetPriorityGrouping(PriorityGroup);
 8001de4:	6878      	ldr	r0, [r7, #4]
 8001de6:	f7ff ff47 	bl	8001c78 <__NVIC_SetPriorityGrouping>
}
 8001dea:	bf00      	nop
 8001dec:	3708      	adds	r7, #8
 8001dee:	46bd      	mov	sp, r7
 8001df0:	bd80      	pop	{r7, pc}

08001df2 <HAL_NVIC_SetPriority>:
  *         This parameter can be a value between 0 and 15
  *         A lower priority value indicates a higher priority.          
  * @retval None
  */
void HAL_NVIC_SetPriority(IRQn_Type IRQn, uint32_t PreemptPriority, uint32_t SubPriority)
{ 
 8001df2:	b580      	push	{r7, lr}
 8001df4:	b086      	sub	sp, #24
 8001df6:	af00      	add	r7, sp, #0
 8001df8:	4603      	mov	r3, r0
 8001dfa:	60b9      	str	r1, [r7, #8]
 8001dfc:	607a      	str	r2, [r7, #4]
 8001dfe:	73fb      	strb	r3, [r7, #15]
  uint32_t prioritygroup = 0x00U;
 8001e00:	2300      	movs	r3, #0
 8001e02:	617b      	str	r3, [r7, #20]
  
  /* Check the parameters */
  assert_param(IS_NVIC_SUB_PRIORITY(SubPriority));
  assert_param(IS_NVIC_PREEMPTION_PRIORITY(PreemptPriority));
  
  prioritygroup = NVIC_GetPriorityGrouping();
 8001e04:	f7ff ff5c 	bl	8001cc0 <__NVIC_GetPriorityGrouping>
 8001e08:	6178      	str	r0, [r7, #20]
  
  NVIC_SetPriority(IRQn, NVIC_EncodePriority(prioritygroup, PreemptPriority, SubPriority));
 8001e0a:	687a      	ldr	r2, [r7, #4]
 8001e0c:	68b9      	ldr	r1, [r7, #8]
 8001e0e:	6978      	ldr	r0, [r7, #20]
 8001e10:	f7ff ff8e 	bl	8001d30 <NVIC_EncodePriority>
 8001e14:	4602      	mov	r2, r0
 8001e16:	f997 300f 	ldrsb.w	r3, [r7, #15]
 8001e1a:	4611      	mov	r1, r2
 8001e1c:	4618      	mov	r0, r3
 8001e1e:	f7ff ff5d 	bl	8001cdc <__NVIC_SetPriority>
}
 8001e22:	bf00      	nop
 8001e24:	3718      	adds	r7, #24
 8001e26:	46bd      	mov	sp, r7
 8001e28:	bd80      	pop	{r7, pc}

08001e2a <HAL_SYSTICK_Config>:
  * @param  TicksNumb Specifies the ticks Number of ticks between two interrupts.
  * @retval status:  - 0  Function succeeded.
  *                  - 1  Function failed.
  */
uint32_t HAL_SYSTICK_Config(uint32_t TicksNumb)
{
 8001e2a:	b580      	push	{r7, lr}
 8001e2c:	b082      	sub	sp, #8
 8001e2e:	af00      	add	r7, sp, #0
 8001e30:	6078      	str	r0, [r7, #4]
   return SysTick_Config(TicksNumb);
 8001e32:	6878      	ldr	r0, [r7, #4]
 8001e34:	f7ff ffb0 	bl	8001d98 <SysTick_Config>
 8001e38:	4603      	mov	r3, r0
}
 8001e3a:	4618      	mov	r0, r3
 8001e3c:	3708      	adds	r7, #8
 8001e3e:	46bd      	mov	sp, r7
 8001e40:	bd80      	pop	{r7, pc}
	...

08001e44 <HAL_GPIO_Init>:
  * @param  GPIO_Init pointer to a GPIO_InitTypeDef structure that contains
  *         the configuration information for the specified GPIO peripheral.
  * @retval None
  */
void HAL_GPIO_Init(GPIO_TypeDef  *GPIOx, GPIO_InitTypeDef *GPIO_Init)
{
 8001e44:	b480      	push	{r7}
 8001e46:	b089      	sub	sp, #36	; 0x24
 8001e48:	af00      	add	r7, sp, #0
 8001e4a:	6078      	str	r0, [r7, #4]
 8001e4c:	6039      	str	r1, [r7, #0]
  uint32_t position;
  uint32_t ioposition = 0x00U;
 8001e4e:	2300      	movs	r3, #0
 8001e50:	617b      	str	r3, [r7, #20]
  uint32_t iocurrent = 0x00U;
 8001e52:	2300      	movs	r3, #0
 8001e54:	613b      	str	r3, [r7, #16]
  uint32_t temp = 0x00U;
 8001e56:	2300      	movs	r3, #0
 8001e58:	61bb      	str	r3, [r7, #24]
  assert_param(IS_GPIO_ALL_INSTANCE(GPIOx));
  assert_param(IS_GPIO_PIN(GPIO_Init->Pin));
  assert_param(IS_GPIO_MODE(GPIO_Init->Mode));

  /* Configure the port pins */
  for(position = 0U; position < GPIO_NUMBER; position++)
 8001e5a:	2300      	movs	r3, #0
 8001e5c:	61fb      	str	r3, [r7, #28]
 8001e5e:	e177      	b.n	8002150 <HAL_GPIO_Init+0x30c>
  {
    /* Get the IO position */
    ioposition = 0x01U << position;
 8001e60:	2201      	movs	r2, #1
 8001e62:	69fb      	ldr	r3, [r7, #28]
 8001e64:	fa02 f303 	lsl.w	r3, r2, r3
 8001e68:	617b      	str	r3, [r7, #20]
    /* Get the current IO position */
    iocurrent = (uint32_t)(GPIO_Init->Pin) & ioposition;
 8001e6a:	683b      	ldr	r3, [r7, #0]
 8001e6c:	681b      	ldr	r3, [r3, #0]
 8001e6e:	697a      	ldr	r2, [r7, #20]
 8001e70:	4013      	ands	r3, r2
 8001e72:	613b      	str	r3, [r7, #16]

    if(iocurrent == ioposition)
 8001e74:	693a      	ldr	r2, [r7, #16]
 8001e76:	697b      	ldr	r3, [r7, #20]
 8001e78:	429a      	cmp	r2, r3
 8001e7a:	f040 8166 	bne.w	800214a <HAL_GPIO_Init+0x306>
    {
      /*--------------------- GPIO Mode Configuration ------------------------*/
      /* In case of Output or Alternate function mode selection */
      if(((GPIO_Init->Mode & GPIO_MODE) == MODE_OUTPUT) || \
 8001e7e:	683b      	ldr	r3, [r7, #0]
 8001e80:	685b      	ldr	r3, [r3, #4]
 8001e82:	f003 0303 	and.w	r3, r3, #3
 8001e86:	2b01      	cmp	r3, #1
 8001e88:	d005      	beq.n	8001e96 <HAL_GPIO_Init+0x52>
          (GPIO_Init->Mode & GPIO_MODE) == MODE_AF)
 8001e8a:	683b      	ldr	r3, [r7, #0]
 8001e8c:	685b      	ldr	r3, [r3, #4]
 8001e8e:	f003 0303 	and.w	r3, r3, #3
      if(((GPIO_Init->Mode & GPIO_MODE) == MODE_OUTPUT) || \
 8001e92:	2b02      	cmp	r3, #2
 8001e94:	d130      	bne.n	8001ef8 <HAL_GPIO_Init+0xb4>
      {
        /* Check the Speed parameter */
        assert_param(IS_GPIO_SPEED(GPIO_Init->Speed));
        /* Configure the IO Speed */
        temp = GPIOx->OSPEEDR; 
 8001e96:	687b      	ldr	r3, [r7, #4]
 8001e98:	689b      	ldr	r3, [r3, #8]
 8001e9a:	61bb      	str	r3, [r7, #24]
        temp &= ~(GPIO_OSPEEDER_OSPEEDR0 << (position * 2U));
 8001e9c:	69fb      	ldr	r3, [r7, #28]
 8001e9e:	005b      	lsls	r3, r3, #1
 8001ea0:	2203      	movs	r2, #3
 8001ea2:	fa02 f303 	lsl.w	r3, r2, r3
 8001ea6:	43db      	mvns	r3, r3
 8001ea8:	69ba      	ldr	r2, [r7, #24]
 8001eaa:	4013      	ands	r3, r2
 8001eac:	61bb      	str	r3, [r7, #24]
        temp |= (GPIO_Init->Speed << (position * 2U));
 8001eae:	683b      	ldr	r3, [r7, #0]
 8001eb0:	68da      	ldr	r2, [r3, #12]
 8001eb2:	69fb      	ldr	r3, [r7, #28]
 8001eb4:	005b      	lsls	r3, r3, #1
 8001eb6:	fa02 f303 	lsl.w	r3, r2, r3
 8001eba:	69ba      	ldr	r2, [r7, #24]
 8001ebc:	4313      	orrs	r3, r2
 8001ebe:	61bb      	str	r3, [r7, #24]
        GPIOx->OSPEEDR = temp;
 8001ec0:	687b      	ldr	r3, [r7, #4]
 8001ec2:	69ba      	ldr	r2, [r7, #24]
 8001ec4:	609a      	str	r2, [r3, #8]

        /* Configure the IO Output Type */
        temp = GPIOx->OTYPER;
 8001ec6:	687b      	ldr	r3, [r7, #4]
 8001ec8:	685b      	ldr	r3, [r3, #4]
 8001eca:	61bb      	str	r3, [r7, #24]
        temp &= ~(GPIO_OTYPER_OT_0 << position) ;
 8001ecc:	2201      	movs	r2, #1
 8001ece:	69fb      	ldr	r3, [r7, #28]
 8001ed0:	fa02 f303 	lsl.w	r3, r2, r3
 8001ed4:	43db      	mvns	r3, r3
 8001ed6:	69ba      	ldr	r2, [r7, #24]
 8001ed8:	4013      	ands	r3, r2
 8001eda:	61bb      	str	r3, [r7, #24]
        temp |= (((GPIO_Init->Mode & OUTPUT_TYPE) >> OUTPUT_TYPE_Pos) << position);
 8001edc:	683b      	ldr	r3, [r7, #0]
 8001ede:	685b      	ldr	r3, [r3, #4]
 8001ee0:	091b      	lsrs	r3, r3, #4
 8001ee2:	f003 0201 	and.w	r2, r3, #1
 8001ee6:	69fb      	ldr	r3, [r7, #28]
 8001ee8:	fa02 f303 	lsl.w	r3, r2, r3
 8001eec:	69ba      	ldr	r2, [r7, #24]
 8001eee:	4313      	orrs	r3, r2
 8001ef0:	61bb      	str	r3, [r7, #24]
        GPIOx->OTYPER = temp;
 8001ef2:	687b      	ldr	r3, [r7, #4]
 8001ef4:	69ba      	ldr	r2, [r7, #24]
 8001ef6:	605a      	str	r2, [r3, #4]
       }

      if((GPIO_Init->Mode & GPIO_MODE) != MODE_ANALOG)
 8001ef8:	683b      	ldr	r3, [r7, #0]
 8001efa:	685b      	ldr	r3, [r3, #4]
 8001efc:	f003 0303 	and.w	r3, r3, #3
 8001f00:	2b03      	cmp	r3, #3
 8001f02:	d017      	beq.n	8001f34 <HAL_GPIO_Init+0xf0>
      {
        /* Check the parameters */
        assert_param(IS_GPIO_PULL(GPIO_Init->Pull));
        
        /* Activate the Pull-up or Pull down resistor for the current IO */
        temp = GPIOx->PUPDR;
 8001f04:	687b      	ldr	r3, [r7, #4]
 8001f06:	68db      	ldr	r3, [r3, #12]
 8001f08:	61bb      	str	r3, [r7, #24]
        temp &= ~(GPIO_PUPDR_PUPDR0 << (position * 2U));
 8001f0a:	69fb      	ldr	r3, [r7, #28]
 8001f0c:	005b      	lsls	r3, r3, #1
 8001f0e:	2203      	movs	r2, #3
 8001f10:	fa02 f303 	lsl.w	r3, r2, r3
 8001f14:	43db      	mvns	r3, r3
 8001f16:	69ba      	ldr	r2, [r7, #24]
 8001f18:	4013      	ands	r3, r2
 8001f1a:	61bb      	str	r3, [r7, #24]
        temp |= ((GPIO_Init->Pull) << (position * 2U));
 8001f1c:	683b      	ldr	r3, [r7, #0]
 8001f1e:	689a      	ldr	r2, [r3, #8]
 8001f20:	69fb      	ldr	r3, [r7, #28]
 8001f22:	005b      	lsls	r3, r3, #1
 8001f24:	fa02 f303 	lsl.w	r3, r2, r3
 8001f28:	69ba      	ldr	r2, [r7, #24]
 8001f2a:	4313      	orrs	r3, r2
 8001f2c:	61bb      	str	r3, [r7, #24]
        GPIOx->PUPDR = temp;
 8001f2e:	687b      	ldr	r3, [r7, #4]
 8001f30:	69ba      	ldr	r2, [r7, #24]
 8001f32:	60da      	str	r2, [r3, #12]
      }

      /* In case of Alternate function mode selection */
      if((GPIO_Init->Mode & GPIO_MODE) == MODE_AF)
 8001f34:	683b      	ldr	r3, [r7, #0]
 8001f36:	685b      	ldr	r3, [r3, #4]
 8001f38:	f003 0303 	and.w	r3, r3, #3
 8001f3c:	2b02      	cmp	r3, #2
 8001f3e:	d123      	bne.n	8001f88 <HAL_GPIO_Init+0x144>
      {
        /* Check the Alternate function parameter */
        assert_param(IS_GPIO_AF(GPIO_Init->Alternate));
        /* Configure Alternate function mapped with the current IO */
        temp = GPIOx->AFR[position >> 3U];
 8001f40:	69fb      	ldr	r3, [r7, #28]
 8001f42:	08da      	lsrs	r2, r3, #3
 8001f44:	687b      	ldr	r3, [r7, #4]
 8001f46:	3208      	adds	r2, #8
 8001f48:	f853 3022 	ldr.w	r3, [r3, r2, lsl #2]
 8001f4c:	61bb      	str	r3, [r7, #24]
        temp &= ~(0xFU << ((uint32_t)(position & 0x07U) * 4U)) ;
 8001f4e:	69fb      	ldr	r3, [r7, #28]
 8001f50:	f003 0307 	and.w	r3, r3, #7
 8001f54:	009b      	lsls	r3, r3, #2
 8001f56:	220f      	movs	r2, #15
 8001f58:	fa02 f303 	lsl.w	r3, r2, r3
 8001f5c:	43db      	mvns	r3, r3
 8001f5e:	69ba      	ldr	r2, [r7, #24]
 8001f60:	4013      	ands	r3, r2
 8001f62:	61bb      	str	r3, [r7, #24]
        temp |= ((uint32_t)(GPIO_Init->Alternate) << (((uint32_t)position & 0x07U) * 4U));
 8001f64:	683b      	ldr	r3, [r7, #0]
 8001f66:	691a      	ldr	r2, [r3, #16]
 8001f68:	69fb      	ldr	r3, [r7, #28]
 8001f6a:	f003 0307 	and.w	r3, r3, #7
 8001f6e:	009b      	lsls	r3, r3, #2
 8001f70:	fa02 f303 	lsl.w	r3, r2, r3
 8001f74:	69ba      	ldr	r2, [r7, #24]
 8001f76:	4313      	orrs	r3, r2
 8001f78:	61bb      	str	r3, [r7, #24]
        GPIOx->AFR[position >> 3U] = temp;
 8001f7a:	69fb      	ldr	r3, [r7, #28]
 8001f7c:	08da      	lsrs	r2, r3, #3
 8001f7e:	687b      	ldr	r3, [r7, #4]
 8001f80:	3208      	adds	r2, #8
 8001f82:	69b9      	ldr	r1, [r7, #24]
 8001f84:	f843 1022 	str.w	r1, [r3, r2, lsl #2]
      }

      /* Configure IO Direction mode (Input, Output, Alternate or Analog) */
      temp = GPIOx->MODER;
 8001f88:	687b      	ldr	r3, [r7, #4]
 8001f8a:	681b      	ldr	r3, [r3, #0]
 8001f8c:	61bb      	str	r3, [r7, #24]
      temp &= ~(GPIO_MODER_MODER0 << (position * 2U));
 8001f8e:	69fb      	ldr	r3, [r7, #28]
 8001f90:	005b      	lsls	r3, r3, #1
 8001f92:	2203      	movs	r2, #3
 8001f94:	fa02 f303 	lsl.w	r3, r2, r3
 8001f98:	43db      	mvns	r3, r3
 8001f9a:	69ba      	ldr	r2, [r7, #24]
 8001f9c:	4013      	ands	r3, r2
 8001f9e:	61bb      	str	r3, [r7, #24]
      temp |= ((GPIO_Init->Mode & GPIO_MODE) << (position * 2U));
 8001fa0:	683b      	ldr	r3, [r7, #0]
 8001fa2:	685b      	ldr	r3, [r3, #4]
 8001fa4:	f003 0203 	and.w	r2, r3, #3
 8001fa8:	69fb      	ldr	r3, [r7, #28]
 8001faa:	005b      	lsls	r3, r3, #1
 8001fac:	fa02 f303 	lsl.w	r3, r2, r3
 8001fb0:	69ba      	ldr	r2, [r7, #24]
 8001fb2:	4313      	orrs	r3, r2
 8001fb4:	61bb      	str	r3, [r7, #24]
      GPIOx->MODER = temp;
 8001fb6:	687b      	ldr	r3, [r7, #4]
 8001fb8:	69ba      	ldr	r2, [r7, #24]
 8001fba:	601a      	str	r2, [r3, #0]

      /*--------------------- EXTI Mode Configuration ------------------------*/
      /* Configure the External Interrupt or event for the current IO */
      if((GPIO_Init->Mode & EXTI_MODE) != 0x00U)
 8001fbc:	683b      	ldr	r3, [r7, #0]
 8001fbe:	685b      	ldr	r3, [r3, #4]
 8001fc0:	f403 3340 	and.w	r3, r3, #196608	; 0x30000
 8001fc4:	2b00      	cmp	r3, #0
 8001fc6:	f000 80c0 	beq.w	800214a <HAL_GPIO_Init+0x306>
      {
        /* Enable SYSCFG Clock */
        __HAL_RCC_SYSCFG_CLK_ENABLE();
 8001fca:	2300      	movs	r3, #0
 8001fcc:	60fb      	str	r3, [r7, #12]
 8001fce:	4b66      	ldr	r3, [pc, #408]	; (8002168 <HAL_GPIO_Init+0x324>)
 8001fd0:	6c5b      	ldr	r3, [r3, #68]	; 0x44
 8001fd2:	4a65      	ldr	r2, [pc, #404]	; (8002168 <HAL_GPIO_Init+0x324>)
 8001fd4:	f443 4380 	orr.w	r3, r3, #16384	; 0x4000
 8001fd8:	6453      	str	r3, [r2, #68]	; 0x44
 8001fda:	4b63      	ldr	r3, [pc, #396]	; (8002168 <HAL_GPIO_Init+0x324>)
 8001fdc:	6c5b      	ldr	r3, [r3, #68]	; 0x44
 8001fde:	f403 4380 	and.w	r3, r3, #16384	; 0x4000
 8001fe2:	60fb      	str	r3, [r7, #12]
 8001fe4:	68fb      	ldr	r3, [r7, #12]

        temp = SYSCFG->EXTICR[position >> 2U];
 8001fe6:	4a61      	ldr	r2, [pc, #388]	; (800216c <HAL_GPIO_Init+0x328>)
 8001fe8:	69fb      	ldr	r3, [r7, #28]
 8001fea:	089b      	lsrs	r3, r3, #2
 8001fec:	3302      	adds	r3, #2
 8001fee:	f852 3023 	ldr.w	r3, [r2, r3, lsl #2]
 8001ff2:	61bb      	str	r3, [r7, #24]
        temp &= ~(0x0FU << (4U * (position & 0x03U)));
 8001ff4:	69fb      	ldr	r3, [r7, #28]
 8001ff6:	f003 0303 	and.w	r3, r3, #3
 8001ffa:	009b      	lsls	r3, r3, #2
 8001ffc:	220f      	movs	r2, #15
 8001ffe:	fa02 f303 	lsl.w	r3, r2, r3
 8002002:	43db      	mvns	r3, r3
 8002004:	69ba      	ldr	r2, [r7, #24]
 8002006:	4013      	ands	r3, r2
 8002008:	61bb      	str	r3, [r7, #24]
        temp |= ((uint32_t)(GPIO_GET_INDEX(GPIOx)) << (4U * (position & 0x03U)));
 800200a:	687b      	ldr	r3, [r7, #4]
 800200c:	4a58      	ldr	r2, [pc, #352]	; (8002170 <HAL_GPIO_Init+0x32c>)
 800200e:	4293      	cmp	r3, r2
 8002010:	d037      	beq.n	8002082 <HAL_GPIO_Init+0x23e>
 8002012:	687b      	ldr	r3, [r7, #4]
 8002014:	4a57      	ldr	r2, [pc, #348]	; (8002174 <HAL_GPIO_Init+0x330>)
 8002016:	4293      	cmp	r3, r2
 8002018:	d031      	beq.n	800207e <HAL_GPIO_Init+0x23a>
 800201a:	687b      	ldr	r3, [r7, #4]
 800201c:	4a56      	ldr	r2, [pc, #344]	; (8002178 <HAL_GPIO_Init+0x334>)
 800201e:	4293      	cmp	r3, r2
 8002020:	d02b      	beq.n	800207a <HAL_GPIO_Init+0x236>
 8002022:	687b      	ldr	r3, [r7, #4]
 8002024:	4a55      	ldr	r2, [pc, #340]	; (800217c <HAL_GPIO_Init+0x338>)
 8002026:	4293      	cmp	r3, r2
 8002028:	d025      	beq.n	8002076 <HAL_GPIO_Init+0x232>
 800202a:	687b      	ldr	r3, [r7, #4]
 800202c:	4a54      	ldr	r2, [pc, #336]	; (8002180 <HAL_GPIO_Init+0x33c>)
 800202e:	4293      	cmp	r3, r2
 8002030:	d01f      	beq.n	8002072 <HAL_GPIO_Init+0x22e>
 8002032:	687b      	ldr	r3, [r7, #4]
 8002034:	4a53      	ldr	r2, [pc, #332]	; (8002184 <HAL_GPIO_Init+0x340>)
 8002036:	4293      	cmp	r3, r2
 8002038:	d019      	beq.n	800206e <HAL_GPIO_Init+0x22a>
 800203a:	687b      	ldr	r3, [r7, #4]
 800203c:	4a52      	ldr	r2, [pc, #328]	; (8002188 <HAL_GPIO_Init+0x344>)
 800203e:	4293      	cmp	r3, r2
 8002040:	d013      	beq.n	800206a <HAL_GPIO_Init+0x226>
 8002042:	687b      	ldr	r3, [r7, #4]
 8002044:	4a51      	ldr	r2, [pc, #324]	; (800218c <HAL_GPIO_Init+0x348>)
 8002046:	4293      	cmp	r3, r2
 8002048:	d00d      	beq.n	8002066 <HAL_GPIO_Init+0x222>
 800204a:	687b      	ldr	r3, [r7, #4]
 800204c:	4a50      	ldr	r2, [pc, #320]	; (8002190 <HAL_GPIO_Init+0x34c>)
 800204e:	4293      	cmp	r3, r2
 8002050:	d007      	beq.n	8002062 <HAL_GPIO_Init+0x21e>
 8002052:	687b      	ldr	r3, [r7, #4]
 8002054:	4a4f      	ldr	r2, [pc, #316]	; (8002194 <HAL_GPIO_Init+0x350>)
 8002056:	4293      	cmp	r3, r2
 8002058:	d101      	bne.n	800205e <HAL_GPIO_Init+0x21a>
 800205a:	2309      	movs	r3, #9
 800205c:	e012      	b.n	8002084 <HAL_GPIO_Init+0x240>
 800205e:	230a      	movs	r3, #10
 8002060:	e010      	b.n	8002084 <HAL_GPIO_Init+0x240>
 8002062:	2308      	movs	r3, #8
 8002064:	e00e      	b.n	8002084 <HAL_GPIO_Init+0x240>
 8002066:	2307      	movs	r3, #7
 8002068:	e00c      	b.n	8002084 <HAL_GPIO_Init+0x240>
 800206a:	2306      	movs	r3, #6
 800206c:	e00a      	b.n	8002084 <HAL_GPIO_Init+0x240>
 800206e:	2305      	movs	r3, #5
 8002070:	e008      	b.n	8002084 <HAL_GPIO_Init+0x240>
 8002072:	2304      	movs	r3, #4
 8002074:	e006      	b.n	8002084 <HAL_GPIO_Init+0x240>
 8002076:	2303      	movs	r3, #3
 8002078:	e004      	b.n	8002084 <HAL_GPIO_Init+0x240>
 800207a:	2302      	movs	r3, #2
 800207c:	e002      	b.n	8002084 <HAL_GPIO_Init+0x240>
 800207e:	2301      	movs	r3, #1
 8002080:	e000      	b.n	8002084 <HAL_GPIO_Init+0x240>
 8002082:	2300      	movs	r3, #0
 8002084:	69fa      	ldr	r2, [r7, #28]
 8002086:	f002 0203 	and.w	r2, r2, #3
 800208a:	0092      	lsls	r2, r2, #2
 800208c:	4093      	lsls	r3, r2
 800208e:	69ba      	ldr	r2, [r7, #24]
 8002090:	4313      	orrs	r3, r2
 8002092:	61bb      	str	r3, [r7, #24]
        SYSCFG->EXTICR[position >> 2U] = temp;
 8002094:	4935      	ldr	r1, [pc, #212]	; (800216c <HAL_GPIO_Init+0x328>)
 8002096:	69fb      	ldr	r3, [r7, #28]
 8002098:	089b      	lsrs	r3, r3, #2
 800209a:	3302      	adds	r3, #2
 800209c:	69ba      	ldr	r2, [r7, #24]
 800209e:	f841 2023 	str.w	r2, [r1, r3, lsl #2]

        /* Clear Rising Falling edge configuration */
        temp = EXTI->RTSR;
 80020a2:	4b3d      	ldr	r3, [pc, #244]	; (8002198 <HAL_GPIO_Init+0x354>)
 80020a4:	689b      	ldr	r3, [r3, #8]
 80020a6:	61bb      	str	r3, [r7, #24]
        temp &= ~((uint32_t)iocurrent);
 80020a8:	693b      	ldr	r3, [r7, #16]
 80020aa:	43db      	mvns	r3, r3
 80020ac:	69ba      	ldr	r2, [r7, #24]
 80020ae:	4013      	ands	r3, r2
 80020b0:	61bb      	str	r3, [r7, #24]
        if((GPIO_Init->Mode & TRIGGER_RISING) != 0x00U)
 80020b2:	683b      	ldr	r3, [r7, #0]
 80020b4:	685b      	ldr	r3, [r3, #4]
 80020b6:	f403 1380 	and.w	r3, r3, #1048576	; 0x100000
 80020ba:	2b00      	cmp	r3, #0
 80020bc:	d003      	beq.n	80020c6 <HAL_GPIO_Init+0x282>
        {
          temp |= iocurrent;
 80020be:	69ba      	ldr	r2, [r7, #24]
 80020c0:	693b      	ldr	r3, [r7, #16]
 80020c2:	4313      	orrs	r3, r2
 80020c4:	61bb      	str	r3, [r7, #24]
        }
        EXTI->RTSR = temp;
 80020c6:	4a34      	ldr	r2, [pc, #208]	; (8002198 <HAL_GPIO_Init+0x354>)
 80020c8:	69bb      	ldr	r3, [r7, #24]
 80020ca:	6093      	str	r3, [r2, #8]

        temp = EXTI->FTSR;
 80020cc:	4b32      	ldr	r3, [pc, #200]	; (8002198 <HAL_GPIO_Init+0x354>)
 80020ce:	68db      	ldr	r3, [r3, #12]
 80020d0:	61bb      	str	r3, [r7, #24]
        temp &= ~((uint32_t)iocurrent);
 80020d2:	693b      	ldr	r3, [r7, #16]
 80020d4:	43db      	mvns	r3, r3
 80020d6:	69ba      	ldr	r2, [r7, #24]
 80020d8:	4013      	ands	r3, r2
 80020da:	61bb      	str	r3, [r7, #24]
        if((GPIO_Init->Mode & TRIGGER_FALLING) != 0x00U)
 80020dc:	683b      	ldr	r3, [r7, #0]
 80020de:	685b      	ldr	r3, [r3, #4]
 80020e0:	f403 1300 	and.w	r3, r3, #2097152	; 0x200000
 80020e4:	2b00      	cmp	r3, #0
 80020e6:	d003      	beq.n	80020f0 <HAL_GPIO_Init+0x2ac>
        {
          temp |= iocurrent;
 80020e8:	69ba      	ldr	r2, [r7, #24]
 80020ea:	693b      	ldr	r3, [r7, #16]
 80020ec:	4313      	orrs	r3, r2
 80020ee:	61bb      	str	r3, [r7, #24]
        }
        EXTI->FTSR = temp;
 80020f0:	4a29      	ldr	r2, [pc, #164]	; (8002198 <HAL_GPIO_Init+0x354>)
 80020f2:	69bb      	ldr	r3, [r7, #24]
 80020f4:	60d3      	str	r3, [r2, #12]

        temp = EXTI->EMR;
 80020f6:	4b28      	ldr	r3, [pc, #160]	; (8002198 <HAL_GPIO_Init+0x354>)
 80020f8:	685b      	ldr	r3, [r3, #4]
 80020fa:	61bb      	str	r3, [r7, #24]
        temp &= ~((uint32_t)iocurrent);
 80020fc:	693b      	ldr	r3, [r7, #16]
 80020fe:	43db      	mvns	r3, r3
 8002100:	69ba      	ldr	r2, [r7, #24]
 8002102:	4013      	ands	r3, r2
 8002104:	61bb      	str	r3, [r7, #24]
        if((GPIO_Init->Mode & EXTI_EVT) != 0x00U)
 8002106:	683b      	ldr	r3, [r7, #0]
 8002108:	685b      	ldr	r3, [r3, #4]
 800210a:	f403 3300 	and.w	r3, r3, #131072	; 0x20000
 800210e:	2b00      	cmp	r3, #0
 8002110:	d003      	beq.n	800211a <HAL_GPIO_Init+0x2d6>
        {
          temp |= iocurrent;
 8002112:	69ba      	ldr	r2, [r7, #24]
 8002114:	693b      	ldr	r3, [r7, #16]
 8002116:	4313      	orrs	r3, r2
 8002118:	61bb      	str	r3, [r7, #24]
        }
        EXTI->EMR = temp;
 800211a:	4a1f      	ldr	r2, [pc, #124]	; (8002198 <HAL_GPIO_Init+0x354>)
 800211c:	69bb      	ldr	r3, [r7, #24]
 800211e:	6053      	str	r3, [r2, #4]

        /* Clear EXTI line configuration */
        temp = EXTI->IMR;
 8002120:	4b1d      	ldr	r3, [pc, #116]	; (8002198 <HAL_GPIO_Init+0x354>)
 8002122:	681b      	ldr	r3, [r3, #0]
 8002124:	61bb      	str	r3, [r7, #24]
        temp &= ~((uint32_t)iocurrent);
 8002126:	693b      	ldr	r3, [r7, #16]
 8002128:	43db      	mvns	r3, r3
 800212a:	69ba      	ldr	r2, [r7, #24]
 800212c:	4013      	ands	r3, r2
 800212e:	61bb      	str	r3, [r7, #24]
        if((GPIO_Init->Mode & EXTI_IT) != 0x00U)
 8002130:	683b      	ldr	r3, [r7, #0]
 8002132:	685b      	ldr	r3, [r3, #4]
 8002134:	f403 3380 	and.w	r3, r3, #65536	; 0x10000
 8002138:	2b00      	cmp	r3, #0
 800213a:	d003      	beq.n	8002144 <HAL_GPIO_Init+0x300>
        {
          temp |= iocurrent;
 800213c:	69ba      	ldr	r2, [r7, #24]
 800213e:	693b      	ldr	r3, [r7, #16]
 8002140:	4313      	orrs	r3, r2
 8002142:	61bb      	str	r3, [r7, #24]
        }
        EXTI->IMR = temp;
 8002144:	4a14      	ldr	r2, [pc, #80]	; (8002198 <HAL_GPIO_Init+0x354>)
 8002146:	69bb      	ldr	r3, [r7, #24]
 8002148:	6013      	str	r3, [r2, #0]
  for(position = 0U; position < GPIO_NUMBER; position++)
 800214a:	69fb      	ldr	r3, [r7, #28]
 800214c:	3301      	adds	r3, #1
 800214e:	61fb      	str	r3, [r7, #28]
 8002150:	69fb      	ldr	r3, [r7, #28]
 8002152:	2b0f      	cmp	r3, #15
 8002154:	f67f ae84 	bls.w	8001e60 <HAL_GPIO_Init+0x1c>
      }
    }
  }
}
 8002158:	bf00      	nop
 800215a:	bf00      	nop
 800215c:	3724      	adds	r7, #36	; 0x24
 800215e:	46bd      	mov	sp, r7
 8002160:	f85d 7b04 	ldr.w	r7, [sp], #4
 8002164:	4770      	bx	lr
 8002166:	bf00      	nop
 8002168:	40023800 	.word	0x40023800
 800216c:	40013800 	.word	0x40013800
 8002170:	40020000 	.word	0x40020000
 8002174:	40020400 	.word	0x40020400
 8002178:	40020800 	.word	0x40020800
 800217c:	40020c00 	.word	0x40020c00
 8002180:	40021000 	.word	0x40021000
 8002184:	40021400 	.word	0x40021400
 8002188:	40021800 	.word	0x40021800
 800218c:	40021c00 	.word	0x40021c00
 8002190:	40022000 	.word	0x40022000
 8002194:	40022400 	.word	0x40022400
 8002198:	40013c00 	.word	0x40013c00

0800219c <HAL_GPIO_WritePin>:
  *            @arg GPIO_PIN_RESET: to clear the port pin
  *            @arg GPIO_PIN_SET: to set the port pin
  * @retval None
  */
void HAL_GPIO_WritePin(GPIO_TypeDef* GPIOx, uint16_t GPIO_Pin, GPIO_PinState PinState)
{
 800219c:	b480      	push	{r7}
 800219e:	b083      	sub	sp, #12
 80021a0:	af00      	add	r7, sp, #0
 80021a2:	6078      	str	r0, [r7, #4]
 80021a4:	460b      	mov	r3, r1
 80021a6:	807b      	strh	r3, [r7, #2]
 80021a8:	4613      	mov	r3, r2
 80021aa:	707b      	strb	r3, [r7, #1]
  /* Check the parameters */
  assert_param(IS_GPIO_PIN(GPIO_Pin));
  assert_param(IS_GPIO_PIN_ACTION(PinState));

  if(PinState != GPIO_PIN_RESET)
 80021ac:	787b      	ldrb	r3, [r7, #1]
 80021ae:	2b00      	cmp	r3, #0
 80021b0:	d003      	beq.n	80021ba <HAL_GPIO_WritePin+0x1e>
  {
    GPIOx->BSRR = GPIO_Pin;
 80021b2:	887a      	ldrh	r2, [r7, #2]
 80021b4:	687b      	ldr	r3, [r7, #4]
 80021b6:	619a      	str	r2, [r3, #24]
  }
  else
  {
    GPIOx->BSRR = (uint32_t)GPIO_Pin << 16U;
  }
}
 80021b8:	e003      	b.n	80021c2 <HAL_GPIO_WritePin+0x26>
    GPIOx->BSRR = (uint32_t)GPIO_Pin << 16U;
 80021ba:	887b      	ldrh	r3, [r7, #2]
 80021bc:	041a      	lsls	r2, r3, #16
 80021be:	687b      	ldr	r3, [r7, #4]
 80021c0:	619a      	str	r2, [r3, #24]
}
 80021c2:	bf00      	nop
 80021c4:	370c      	adds	r7, #12
 80021c6:	46bd      	mov	sp, r7
 80021c8:	f85d 7b04 	ldr.w	r7, [sp], #4
 80021cc:	4770      	bx	lr
	...

080021d0 <HAL_RCC_OscConfig>:
  *         supported by this API. User should request a transition to HSE Off
  *         first and then HSE On or HSE Bypass.
  * @retval HAL status
  */
__weak HAL_StatusTypeDef HAL_RCC_OscConfig(RCC_OscInitTypeDef  *RCC_OscInitStruct)
{
 80021d0:	b580      	push	{r7, lr}
 80021d2:	b086      	sub	sp, #24
 80021d4:	af00      	add	r7, sp, #0
 80021d6:	6078      	str	r0, [r7, #4]
  uint32_t tickstart, pll_config;

  /* Check Null pointer */
  if(RCC_OscInitStruct == NULL)
 80021d8:	687b      	ldr	r3, [r7, #4]
 80021da:	2b00      	cmp	r3, #0
 80021dc:	d101      	bne.n	80021e2 <HAL_RCC_OscConfig+0x12>
  {
    return HAL_ERROR;
 80021de:	2301      	movs	r3, #1
 80021e0:	e267      	b.n	80026b2 <HAL_RCC_OscConfig+0x4e2>
  }

  /* Check the parameters */
  assert_param(IS_RCC_OSCILLATORTYPE(RCC_OscInitStruct->OscillatorType));
  /*------------------------------- HSE Configuration ------------------------*/
  if(((RCC_OscInitStruct->OscillatorType) & RCC_OSCILLATORTYPE_HSE) == RCC_OSCILLATORTYPE_HSE)
 80021e2:	687b      	ldr	r3, [r7, #4]
 80021e4:	681b      	ldr	r3, [r3, #0]
 80021e6:	f003 0301 	and.w	r3, r3, #1
 80021ea:	2b00      	cmp	r3, #0
 80021ec:	d075      	beq.n	80022da <HAL_RCC_OscConfig+0x10a>
  {
    /* Check the parameters */
    assert_param(IS_RCC_HSE(RCC_OscInitStruct->HSEState));
    /* When the HSE is used as system clock or clock source for PLL in these cases HSE will not disabled */
    if((__HAL_RCC_GET_SYSCLK_SOURCE() == RCC_CFGR_SWS_HSE) ||\
 80021ee:	4b88      	ldr	r3, [pc, #544]	; (8002410 <HAL_RCC_OscConfig+0x240>)
 80021f0:	689b      	ldr	r3, [r3, #8]
 80021f2:	f003 030c 	and.w	r3, r3, #12
 80021f6:	2b04      	cmp	r3, #4
 80021f8:	d00c      	beq.n	8002214 <HAL_RCC_OscConfig+0x44>
      ((__HAL_RCC_GET_SYSCLK_SOURCE() == RCC_CFGR_SWS_PLL) && ((RCC->PLLCFGR & RCC_PLLCFGR_PLLSRC) == RCC_PLLCFGR_PLLSRC_HSE)))
 80021fa:	4b85      	ldr	r3, [pc, #532]	; (8002410 <HAL_RCC_OscConfig+0x240>)
 80021fc:	689b      	ldr	r3, [r3, #8]
 80021fe:	f003 030c 	and.w	r3, r3, #12
    if((__HAL_RCC_GET_SYSCLK_SOURCE() == RCC_CFGR_SWS_HSE) ||\
 8002202:	2b08      	cmp	r3, #8
 8002204:	d112      	bne.n	800222c <HAL_RCC_OscConfig+0x5c>
      ((__HAL_RCC_GET_SYSCLK_SOURCE() == RCC_CFGR_SWS_PLL) && ((RCC->PLLCFGR & RCC_PLLCFGR_PLLSRC) == RCC_PLLCFGR_PLLSRC_HSE)))
 8002206:	4b82      	ldr	r3, [pc, #520]	; (8002410 <HAL_RCC_OscConfig+0x240>)
 8002208:	685b      	ldr	r3, [r3, #4]
 800220a:	f403 0380 	and.w	r3, r3, #4194304	; 0x400000
 800220e:	f5b3 0f80 	cmp.w	r3, #4194304	; 0x400000
 8002212:	d10b      	bne.n	800222c <HAL_RCC_OscConfig+0x5c>
    {
      if((__HAL_RCC_GET_FLAG(RCC_FLAG_HSERDY) != RESET) && (RCC_OscInitStruct->HSEState == RCC_HSE_OFF))
 8002214:	4b7e      	ldr	r3, [pc, #504]	; (8002410 <HAL_RCC_OscConfig+0x240>)
 8002216:	681b      	ldr	r3, [r3, #0]
 8002218:	f403 3300 	and.w	r3, r3, #131072	; 0x20000
 800221c:	2b00      	cmp	r3, #0
 800221e:	d05b      	beq.n	80022d8 <HAL_RCC_OscConfig+0x108>
 8002220:	687b      	ldr	r3, [r7, #4]
 8002222:	685b      	ldr	r3, [r3, #4]
 8002224:	2b00      	cmp	r3, #0
 8002226:	d157      	bne.n	80022d8 <HAL_RCC_OscConfig+0x108>
      {
        return HAL_ERROR;
 8002228:	2301      	movs	r3, #1
 800222a:	e242      	b.n	80026b2 <HAL_RCC_OscConfig+0x4e2>
      }
    }
    else
    {
      /* Set the new HSE configuration ---------------------------------------*/
      __HAL_RCC_HSE_CONFIG(RCC_OscInitStruct->HSEState);
 800222c:	687b      	ldr	r3, [r7, #4]
 800222e:	685b      	ldr	r3, [r3, #4]
 8002230:	f5b3 3f80 	cmp.w	r3, #65536	; 0x10000
 8002234:	d106      	bne.n	8002244 <HAL_RCC_OscConfig+0x74>
 8002236:	4b76      	ldr	r3, [pc, #472]	; (8002410 <HAL_RCC_OscConfig+0x240>)
 8002238:	681b      	ldr	r3, [r3, #0]
 800223a:	4a75      	ldr	r2, [pc, #468]	; (8002410 <HAL_RCC_OscConfig+0x240>)
 800223c:	f443 3380 	orr.w	r3, r3, #65536	; 0x10000
 8002240:	6013      	str	r3, [r2, #0]
 8002242:	e01d      	b.n	8002280 <HAL_RCC_OscConfig+0xb0>
 8002244:	687b      	ldr	r3, [r7, #4]
 8002246:	685b      	ldr	r3, [r3, #4]
 8002248:	f5b3 2fa0 	cmp.w	r3, #327680	; 0x50000
 800224c:	d10c      	bne.n	8002268 <HAL_RCC_OscConfig+0x98>
 800224e:	4b70      	ldr	r3, [pc, #448]	; (8002410 <HAL_RCC_OscConfig+0x240>)
 8002250:	681b      	ldr	r3, [r3, #0]
 8002252:	4a6f      	ldr	r2, [pc, #444]	; (8002410 <HAL_RCC_OscConfig+0x240>)
 8002254:	f443 2380 	orr.w	r3, r3, #262144	; 0x40000
 8002258:	6013      	str	r3, [r2, #0]
 800225a:	4b6d      	ldr	r3, [pc, #436]	; (8002410 <HAL_RCC_OscConfig+0x240>)
 800225c:	681b      	ldr	r3, [r3, #0]
 800225e:	4a6c      	ldr	r2, [pc, #432]	; (8002410 <HAL_RCC_OscConfig+0x240>)
 8002260:	f443 3380 	orr.w	r3, r3, #65536	; 0x10000
 8002264:	6013      	str	r3, [r2, #0]
 8002266:	e00b      	b.n	8002280 <HAL_RCC_OscConfig+0xb0>
 8002268:	4b69      	ldr	r3, [pc, #420]	; (8002410 <HAL_RCC_OscConfig+0x240>)
 800226a:	681b      	ldr	r3, [r3, #0]
 800226c:	4a68      	ldr	r2, [pc, #416]	; (8002410 <HAL_RCC_OscConfig+0x240>)
 800226e:	f423 3380 	bic.w	r3, r3, #65536	; 0x10000
 8002272:	6013      	str	r3, [r2, #0]
 8002274:	4b66      	ldr	r3, [pc, #408]	; (8002410 <HAL_RCC_OscConfig+0x240>)
 8002276:	681b      	ldr	r3, [r3, #0]
 8002278:	4a65      	ldr	r2, [pc, #404]	; (8002410 <HAL_RCC_OscConfig+0x240>)
 800227a:	f423 2380 	bic.w	r3, r3, #262144	; 0x40000
 800227e:	6013      	str	r3, [r2, #0]

      /* Check the HSE State */
      if((RCC_OscInitStruct->HSEState) != RCC_HSE_OFF)
 8002280:	687b      	ldr	r3, [r7, #4]
 8002282:	685b      	ldr	r3, [r3, #4]
 8002284:	2b00      	cmp	r3, #0
 8002286:	d013      	beq.n	80022b0 <HAL_RCC_OscConfig+0xe0>
      {
        /* Get Start Tick */
        tickstart = HAL_GetTick();
 8002288:	f7ff fcc6 	bl	8001c18 <HAL_GetTick>
 800228c:	6138      	str	r0, [r7, #16]

        /* Wait till HSE is ready */
        while(__HAL_RCC_GET_FLAG(RCC_FLAG_HSERDY) == RESET)
 800228e:	e008      	b.n	80022a2 <HAL_RCC_OscConfig+0xd2>
        {
          if((HAL_GetTick() - tickstart ) > HSE_TIMEOUT_VALUE)
 8002290:	f7ff fcc2 	bl	8001c18 <HAL_GetTick>
 8002294:	4602      	mov	r2, r0
 8002296:	693b      	ldr	r3, [r7, #16]
 8002298:	1ad3      	subs	r3, r2, r3
 800229a:	2b64      	cmp	r3, #100	; 0x64
 800229c:	d901      	bls.n	80022a2 <HAL_RCC_OscConfig+0xd2>
          {
            return HAL_TIMEOUT;
 800229e:	2303      	movs	r3, #3
 80022a0:	e207      	b.n	80026b2 <HAL_RCC_OscConfig+0x4e2>
        while(__HAL_RCC_GET_FLAG(RCC_FLAG_HSERDY) == RESET)
 80022a2:	4b5b      	ldr	r3, [pc, #364]	; (8002410 <HAL_RCC_OscConfig+0x240>)
 80022a4:	681b      	ldr	r3, [r3, #0]
 80022a6:	f403 3300 	and.w	r3, r3, #131072	; 0x20000
 80022aa:	2b00      	cmp	r3, #0
 80022ac:	d0f0      	beq.n	8002290 <HAL_RCC_OscConfig+0xc0>
 80022ae:	e014      	b.n	80022da <HAL_RCC_OscConfig+0x10a>
        }
      }
      else
      {
        /* Get Start Tick */
        tickstart = HAL_GetTick();
 80022b0:	f7ff fcb2 	bl	8001c18 <HAL_GetTick>
 80022b4:	6138      	str	r0, [r7, #16]

        /* Wait till HSE is bypassed or disabled */
        while(__HAL_RCC_GET_FLAG(RCC_FLAG_HSERDY) != RESET)
 80022b6:	e008      	b.n	80022ca <HAL_RCC_OscConfig+0xfa>
        {
          if((HAL_GetTick() - tickstart ) > HSE_TIMEOUT_VALUE)
 80022b8:	f7ff fcae 	bl	8001c18 <HAL_GetTick>
 80022bc:	4602      	mov	r2, r0
 80022be:	693b      	ldr	r3, [r7, #16]
 80022c0:	1ad3      	subs	r3, r2, r3
 80022c2:	2b64      	cmp	r3, #100	; 0x64
 80022c4:	d901      	bls.n	80022ca <HAL_RCC_OscConfig+0xfa>
          {
            return HAL_TIMEOUT;
 80022c6:	2303      	movs	r3, #3
 80022c8:	e1f3      	b.n	80026b2 <HAL_RCC_OscConfig+0x4e2>
        while(__HAL_RCC_GET_FLAG(RCC_FLAG_HSERDY) != RESET)
 80022ca:	4b51      	ldr	r3, [pc, #324]	; (8002410 <HAL_RCC_OscConfig+0x240>)
 80022cc:	681b      	ldr	r3, [r3, #0]
 80022ce:	f403 3300 	and.w	r3, r3, #131072	; 0x20000
 80022d2:	2b00      	cmp	r3, #0
 80022d4:	d1f0      	bne.n	80022b8 <HAL_RCC_OscConfig+0xe8>
 80022d6:	e000      	b.n	80022da <HAL_RCC_OscConfig+0x10a>
      if((__HAL_RCC_GET_FLAG(RCC_FLAG_HSERDY) != RESET) && (RCC_OscInitStruct->HSEState == RCC_HSE_OFF))
 80022d8:	bf00      	nop
        }
      }
    }
  }
  /*----------------------------- HSI Configuration --------------------------*/
  if(((RCC_OscInitStruct->OscillatorType) & RCC_OSCILLATORTYPE_HSI) == RCC_OSCILLATORTYPE_HSI)
 80022da:	687b      	ldr	r3, [r7, #4]
 80022dc:	681b      	ldr	r3, [r3, #0]
 80022de:	f003 0302 	and.w	r3, r3, #2
 80022e2:	2b00      	cmp	r3, #0
 80022e4:	d063      	beq.n	80023ae <HAL_RCC_OscConfig+0x1de>
    /* Check the parameters */
    assert_param(IS_RCC_HSI(RCC_OscInitStruct->HSIState));
    assert_param(IS_RCC_CALIBRATION_VALUE(RCC_OscInitStruct->HSICalibrationValue));

    /* Check if HSI is used as system clock or as PLL source when PLL is selected as system clock */
    if((__HAL_RCC_GET_SYSCLK_SOURCE() == RCC_CFGR_SWS_HSI) ||\
 80022e6:	4b4a      	ldr	r3, [pc, #296]	; (8002410 <HAL_RCC_OscConfig+0x240>)
 80022e8:	689b      	ldr	r3, [r3, #8]
 80022ea:	f003 030c 	and.w	r3, r3, #12
 80022ee:	2b00      	cmp	r3, #0
 80022f0:	d00b      	beq.n	800230a <HAL_RCC_OscConfig+0x13a>
      ((__HAL_RCC_GET_SYSCLK_SOURCE() == RCC_CFGR_SWS_PLL) && ((RCC->PLLCFGR & RCC_PLLCFGR_PLLSRC) == RCC_PLLCFGR_PLLSRC_HSI)))
 80022f2:	4b47      	ldr	r3, [pc, #284]	; (8002410 <HAL_RCC_OscConfig+0x240>)
 80022f4:	689b      	ldr	r3, [r3, #8]
 80022f6:	f003 030c 	and.w	r3, r3, #12
    if((__HAL_RCC_GET_SYSCLK_SOURCE() == RCC_CFGR_SWS_HSI) ||\
 80022fa:	2b08      	cmp	r3, #8
 80022fc:	d11c      	bne.n	8002338 <HAL_RCC_OscConfig+0x168>
      ((__HAL_RCC_GET_SYSCLK_SOURCE() == RCC_CFGR_SWS_PLL) && ((RCC->PLLCFGR & RCC_PLLCFGR_PLLSRC) == RCC_PLLCFGR_PLLSRC_HSI)))
 80022fe:	4b44      	ldr	r3, [pc, #272]	; (8002410 <HAL_RCC_OscConfig+0x240>)
 8002300:	685b      	ldr	r3, [r3, #4]
 8002302:	f403 0380 	and.w	r3, r3, #4194304	; 0x400000
 8002306:	2b00      	cmp	r3, #0
 8002308:	d116      	bne.n	8002338 <HAL_RCC_OscConfig+0x168>
    {
      /* When HSI is used as system clock it will not disabled */
      if((__HAL_RCC_GET_FLAG(RCC_FLAG_HSIRDY) != RESET) && (RCC_OscInitStruct->HSIState != RCC_HSI_ON))
 800230a:	4b41      	ldr	r3, [pc, #260]	; (8002410 <HAL_RCC_OscConfig+0x240>)
 800230c:	681b      	ldr	r3, [r3, #0]
 800230e:	f003 0302 	and.w	r3, r3, #2
 8002312:	2b00      	cmp	r3, #0
 8002314:	d005      	beq.n	8002322 <HAL_RCC_OscConfig+0x152>
 8002316:	687b      	ldr	r3, [r7, #4]
 8002318:	68db      	ldr	r3, [r3, #12]
 800231a:	2b01      	cmp	r3, #1
 800231c:	d001      	beq.n	8002322 <HAL_RCC_OscConfig+0x152>
      {
        return HAL_ERROR;
 800231e:	2301      	movs	r3, #1
 8002320:	e1c7      	b.n	80026b2 <HAL_RCC_OscConfig+0x4e2>
      }
      /* Otherwise, just the calibration is allowed */
      else
      {
        /* Adjusts the Internal High Speed oscillator (HSI) calibration value.*/
        __HAL_RCC_HSI_CALIBRATIONVALUE_ADJUST(RCC_OscInitStruct->HSICalibrationValue);
 8002322:	4b3b      	ldr	r3, [pc, #236]	; (8002410 <HAL_RCC_OscConfig+0x240>)
 8002324:	681b      	ldr	r3, [r3, #0]
 8002326:	f023 02f8 	bic.w	r2, r3, #248	; 0xf8
 800232a:	687b      	ldr	r3, [r7, #4]
 800232c:	691b      	ldr	r3, [r3, #16]
 800232e:	00db      	lsls	r3, r3, #3
 8002330:	4937      	ldr	r1, [pc, #220]	; (8002410 <HAL_RCC_OscConfig+0x240>)
 8002332:	4313      	orrs	r3, r2
 8002334:	600b      	str	r3, [r1, #0]
      if((__HAL_RCC_GET_FLAG(RCC_FLAG_HSIRDY) != RESET) && (RCC_OscInitStruct->HSIState != RCC_HSI_ON))
 8002336:	e03a      	b.n	80023ae <HAL_RCC_OscConfig+0x1de>
      }
    }
    else
    {
      /* Check the HSI State */
      if((RCC_OscInitStruct->HSIState)!= RCC_HSI_OFF)
 8002338:	687b      	ldr	r3, [r7, #4]
 800233a:	68db      	ldr	r3, [r3, #12]
 800233c:	2b00      	cmp	r3, #0
 800233e:	d020      	beq.n	8002382 <HAL_RCC_OscConfig+0x1b2>
      {
        /* Enable the Internal High Speed oscillator (HSI). */
        __HAL_RCC_HSI_ENABLE();
 8002340:	4b34      	ldr	r3, [pc, #208]	; (8002414 <HAL_RCC_OscConfig+0x244>)
 8002342:	2201      	movs	r2, #1
 8002344:	601a      	str	r2, [r3, #0]

        /* Get Start Tick*/
        tickstart = HAL_GetTick();
 8002346:	f7ff fc67 	bl	8001c18 <HAL_GetTick>
 800234a:	6138      	str	r0, [r7, #16]

        /* Wait till HSI is ready */
        while(__HAL_RCC_GET_FLAG(RCC_FLAG_HSIRDY) == RESET)
 800234c:	e008      	b.n	8002360 <HAL_RCC_OscConfig+0x190>
        {
          if((HAL_GetTick() - tickstart ) > HSI_TIMEOUT_VALUE)
 800234e:	f7ff fc63 	bl	8001c18 <HAL_GetTick>
 8002352:	4602      	mov	r2, r0
 8002354:	693b      	ldr	r3, [r7, #16]
 8002356:	1ad3      	subs	r3, r2, r3
 8002358:	2b02      	cmp	r3, #2
 800235a:	d901      	bls.n	8002360 <HAL_RCC_OscConfig+0x190>
          {
            return HAL_TIMEOUT;
 800235c:	2303      	movs	r3, #3
 800235e:	e1a8      	b.n	80026b2 <HAL_RCC_OscConfig+0x4e2>
        while(__HAL_RCC_GET_FLAG(RCC_FLAG_HSIRDY) == RESET)
 8002360:	4b2b      	ldr	r3, [pc, #172]	; (8002410 <HAL_RCC_OscConfig+0x240>)
 8002362:	681b      	ldr	r3, [r3, #0]
 8002364:	f003 0302 	and.w	r3, r3, #2
 8002368:	2b00      	cmp	r3, #0
 800236a:	d0f0      	beq.n	800234e <HAL_RCC_OscConfig+0x17e>
          }
        }

        /* Adjusts the Internal High Speed oscillator (HSI) calibration value. */
        __HAL_RCC_HSI_CALIBRATIONVALUE_ADJUST(RCC_OscInitStruct->HSICalibrationValue);
 800236c:	4b28      	ldr	r3, [pc, #160]	; (8002410 <HAL_RCC_OscConfig+0x240>)
 800236e:	681b      	ldr	r3, [r3, #0]
 8002370:	f023 02f8 	bic.w	r2, r3, #248	; 0xf8
 8002374:	687b      	ldr	r3, [r7, #4]
 8002376:	691b      	ldr	r3, [r3, #16]
 8002378:	00db      	lsls	r3, r3, #3
 800237a:	4925      	ldr	r1, [pc, #148]	; (8002410 <HAL_RCC_OscConfig+0x240>)
 800237c:	4313      	orrs	r3, r2
 800237e:	600b      	str	r3, [r1, #0]
 8002380:	e015      	b.n	80023ae <HAL_RCC_OscConfig+0x1de>
      }
      else
      {
        /* Disable the Internal High Speed oscillator (HSI). */
        __HAL_RCC_HSI_DISABLE();
 8002382:	4b24      	ldr	r3, [pc, #144]	; (8002414 <HAL_RCC_OscConfig+0x244>)
 8002384:	2200      	movs	r2, #0
 8002386:	601a      	str	r2, [r3, #0]

        /* Get Start Tick*/
        tickstart = HAL_GetTick();
 8002388:	f7ff fc46 	bl	8001c18 <HAL_GetTick>
 800238c:	6138      	str	r0, [r7, #16]

        /* Wait till HSI is ready */
        while(__HAL_RCC_GET_FLAG(RCC_FLAG_HSIRDY) != RESET)
 800238e:	e008      	b.n	80023a2 <HAL_RCC_OscConfig+0x1d2>
        {
          if((HAL_GetTick() - tickstart ) > HSI_TIMEOUT_VALUE)
 8002390:	f7ff fc42 	bl	8001c18 <HAL_GetTick>
 8002394:	4602      	mov	r2, r0
 8002396:	693b      	ldr	r3, [r7, #16]
 8002398:	1ad3      	subs	r3, r2, r3
 800239a:	2b02      	cmp	r3, #2
 800239c:	d901      	bls.n	80023a2 <HAL_RCC_OscConfig+0x1d2>
          {
            return HAL_TIMEOUT;
 800239e:	2303      	movs	r3, #3
 80023a0:	e187      	b.n	80026b2 <HAL_RCC_OscConfig+0x4e2>
        while(__HAL_RCC_GET_FLAG(RCC_FLAG_HSIRDY) != RESET)
 80023a2:	4b1b      	ldr	r3, [pc, #108]	; (8002410 <HAL_RCC_OscConfig+0x240>)
 80023a4:	681b      	ldr	r3, [r3, #0]
 80023a6:	f003 0302 	and.w	r3, r3, #2
 80023aa:	2b00      	cmp	r3, #0
 80023ac:	d1f0      	bne.n	8002390 <HAL_RCC_OscConfig+0x1c0>
        }
      }
    }
  }
  /*------------------------------ LSI Configuration -------------------------*/
  if(((RCC_OscInitStruct->OscillatorType) & RCC_OSCILLATORTYPE_LSI) == RCC_OSCILLATORTYPE_LSI)
 80023ae:	687b      	ldr	r3, [r7, #4]
 80023b0:	681b      	ldr	r3, [r3, #0]
 80023b2:	f003 0308 	and.w	r3, r3, #8
 80023b6:	2b00      	cmp	r3, #0
 80023b8:	d036      	beq.n	8002428 <HAL_RCC_OscConfig+0x258>
  {
    /* Check the parameters */
    assert_param(IS_RCC_LSI(RCC_OscInitStruct->LSIState));

    /* Check the LSI State */
    if((RCC_OscInitStruct->LSIState)!= RCC_LSI_OFF)
 80023ba:	687b      	ldr	r3, [r7, #4]
 80023bc:	695b      	ldr	r3, [r3, #20]
 80023be:	2b00      	cmp	r3, #0
 80023c0:	d016      	beq.n	80023f0 <HAL_RCC_OscConfig+0x220>
    {
      /* Enable the Internal Low Speed oscillator (LSI). */
      __HAL_RCC_LSI_ENABLE();
 80023c2:	4b15      	ldr	r3, [pc, #84]	; (8002418 <HAL_RCC_OscConfig+0x248>)
 80023c4:	2201      	movs	r2, #1
 80023c6:	601a      	str	r2, [r3, #0]

      /* Get Start Tick*/
      tickstart = HAL_GetTick();
 80023c8:	f7ff fc26 	bl	8001c18 <HAL_GetTick>
 80023cc:	6138      	str	r0, [r7, #16]

      /* Wait till LSI is ready */
      while(__HAL_RCC_GET_FLAG(RCC_FLAG_LSIRDY) == RESET)
 80023ce:	e008      	b.n	80023e2 <HAL_RCC_OscConfig+0x212>
      {
        if((HAL_GetTick() - tickstart ) > LSI_TIMEOUT_VALUE)
 80023d0:	f7ff fc22 	bl	8001c18 <HAL_GetTick>
 80023d4:	4602      	mov	r2, r0
 80023d6:	693b      	ldr	r3, [r7, #16]
 80023d8:	1ad3      	subs	r3, r2, r3
 80023da:	2b02      	cmp	r3, #2
 80023dc:	d901      	bls.n	80023e2 <HAL_RCC_OscConfig+0x212>
        {
          return HAL_TIMEOUT;
 80023de:	2303      	movs	r3, #3
 80023e0:	e167      	b.n	80026b2 <HAL_RCC_OscConfig+0x4e2>
      while(__HAL_RCC_GET_FLAG(RCC_FLAG_LSIRDY) == RESET)
 80023e2:	4b0b      	ldr	r3, [pc, #44]	; (8002410 <HAL_RCC_OscConfig+0x240>)
 80023e4:	6f5b      	ldr	r3, [r3, #116]	; 0x74
 80023e6:	f003 0302 	and.w	r3, r3, #2
 80023ea:	2b00      	cmp	r3, #0
 80023ec:	d0f0      	beq.n	80023d0 <HAL_RCC_OscConfig+0x200>
 80023ee:	e01b      	b.n	8002428 <HAL_RCC_OscConfig+0x258>
      }
    }
    else
    {
      /* Disable the Internal Low Speed oscillator (LSI). */
      __HAL_RCC_LSI_DISABLE();
 80023f0:	4b09      	ldr	r3, [pc, #36]	; (8002418 <HAL_RCC_OscConfig+0x248>)
 80023f2:	2200      	movs	r2, #0
 80023f4:	601a      	str	r2, [r3, #0]

      /* Get Start Tick */
      tickstart = HAL_GetTick();
 80023f6:	f7ff fc0f 	bl	8001c18 <HAL_GetTick>
 80023fa:	6138      	str	r0, [r7, #16]

      /* Wait till LSI is ready */
      while(__HAL_RCC_GET_FLAG(RCC_FLAG_LSIRDY) != RESET)
 80023fc:	e00e      	b.n	800241c <HAL_RCC_OscConfig+0x24c>
      {
        if((HAL_GetTick() - tickstart ) > LSI_TIMEOUT_VALUE)
 80023fe:	f7ff fc0b 	bl	8001c18 <HAL_GetTick>
 8002402:	4602      	mov	r2, r0
 8002404:	693b      	ldr	r3, [r7, #16]
 8002406:	1ad3      	subs	r3, r2, r3
 8002408:	2b02      	cmp	r3, #2
 800240a:	d907      	bls.n	800241c <HAL_RCC_OscConfig+0x24c>
        {
          return HAL_TIMEOUT;
 800240c:	2303      	movs	r3, #3
 800240e:	e150      	b.n	80026b2 <HAL_RCC_OscConfig+0x4e2>
 8002410:	40023800 	.word	0x40023800
 8002414:	42470000 	.word	0x42470000
 8002418:	42470e80 	.word	0x42470e80
      while(__HAL_RCC_GET_FLAG(RCC_FLAG_LSIRDY) != RESET)
 800241c:	4b88      	ldr	r3, [pc, #544]	; (8002640 <HAL_RCC_OscConfig+0x470>)
 800241e:	6f5b      	ldr	r3, [r3, #116]	; 0x74
 8002420:	f003 0302 	and.w	r3, r3, #2
 8002424:	2b00      	cmp	r3, #0
 8002426:	d1ea      	bne.n	80023fe <HAL_RCC_OscConfig+0x22e>
        }
      }
    }
  }
  /*------------------------------ LSE Configuration -------------------------*/
  if(((RCC_OscInitStruct->OscillatorType) & RCC_OSCILLATORTYPE_LSE) == RCC_OSCILLATORTYPE_LSE)
 8002428:	687b      	ldr	r3, [r7, #4]
 800242a:	681b      	ldr	r3, [r3, #0]
 800242c:	f003 0304 	and.w	r3, r3, #4
 8002430:	2b00      	cmp	r3, #0
 8002432:	f000 8097 	beq.w	8002564 <HAL_RCC_OscConfig+0x394>
  {
    FlagStatus       pwrclkchanged = RESET;
 8002436:	2300      	movs	r3, #0
 8002438:	75fb      	strb	r3, [r7, #23]
    /* Check the parameters */
    assert_param(IS_RCC_LSE(RCC_OscInitStruct->LSEState));

    /* Update LSE configuration in Backup Domain control register    */
    /* Requires to enable write access to Backup Domain of necessary */
    if(__HAL_RCC_PWR_IS_CLK_DISABLED())
 800243a:	4b81      	ldr	r3, [pc, #516]	; (8002640 <HAL_RCC_OscConfig+0x470>)
 800243c:	6c1b      	ldr	r3, [r3, #64]	; 0x40
 800243e:	f003 5380 	and.w	r3, r3, #268435456	; 0x10000000
 8002442:	2b00      	cmp	r3, #0
 8002444:	d10f      	bne.n	8002466 <HAL_RCC_OscConfig+0x296>
    {
      __HAL_RCC_PWR_CLK_ENABLE();
 8002446:	2300      	movs	r3, #0
 8002448:	60bb      	str	r3, [r7, #8]
 800244a:	4b7d      	ldr	r3, [pc, #500]	; (8002640 <HAL_RCC_OscConfig+0x470>)
 800244c:	6c1b      	ldr	r3, [r3, #64]	; 0x40
 800244e:	4a7c      	ldr	r2, [pc, #496]	; (8002640 <HAL_RCC_OscConfig+0x470>)
 8002450:	f043 5380 	orr.w	r3, r3, #268435456	; 0x10000000
 8002454:	6413      	str	r3, [r2, #64]	; 0x40
 8002456:	4b7a      	ldr	r3, [pc, #488]	; (8002640 <HAL_RCC_OscConfig+0x470>)
 8002458:	6c1b      	ldr	r3, [r3, #64]	; 0x40
 800245a:	f003 5380 	and.w	r3, r3, #268435456	; 0x10000000
 800245e:	60bb      	str	r3, [r7, #8]
 8002460:	68bb      	ldr	r3, [r7, #8]
      pwrclkchanged = SET;
 8002462:	2301      	movs	r3, #1
 8002464:	75fb      	strb	r3, [r7, #23]
    }

    if(HAL_IS_BIT_CLR(PWR->CR, PWR_CR_DBP))
 8002466:	4b77      	ldr	r3, [pc, #476]	; (8002644 <HAL_RCC_OscConfig+0x474>)
 8002468:	681b      	ldr	r3, [r3, #0]
 800246a:	f403 7380 	and.w	r3, r3, #256	; 0x100
 800246e:	2b00      	cmp	r3, #0
 8002470:	d118      	bne.n	80024a4 <HAL_RCC_OscConfig+0x2d4>
    {
      /* Enable write access to Backup domain */
      SET_BIT(PWR->CR, PWR_CR_DBP);
 8002472:	4b74      	ldr	r3, [pc, #464]	; (8002644 <HAL_RCC_OscConfig+0x474>)
 8002474:	681b      	ldr	r3, [r3, #0]
 8002476:	4a73      	ldr	r2, [pc, #460]	; (8002644 <HAL_RCC_OscConfig+0x474>)
 8002478:	f443 7380 	orr.w	r3, r3, #256	; 0x100
 800247c:	6013      	str	r3, [r2, #0]

      /* Wait for Backup domain Write protection disable */
      tickstart = HAL_GetTick();
 800247e:	f7ff fbcb 	bl	8001c18 <HAL_GetTick>
 8002482:	6138      	str	r0, [r7, #16]

      while(HAL_IS_BIT_CLR(PWR->CR, PWR_CR_DBP))
 8002484:	e008      	b.n	8002498 <HAL_RCC_OscConfig+0x2c8>
      {
        if((HAL_GetTick() - tickstart) > RCC_DBP_TIMEOUT_VALUE)
 8002486:	f7ff fbc7 	bl	8001c18 <HAL_GetTick>
 800248a:	4602      	mov	r2, r0
 800248c:	693b      	ldr	r3, [r7, #16]
 800248e:	1ad3      	subs	r3, r2, r3
 8002490:	2b02      	cmp	r3, #2
 8002492:	d901      	bls.n	8002498 <HAL_RCC_OscConfig+0x2c8>
        {
          return HAL_TIMEOUT;
 8002494:	2303      	movs	r3, #3
 8002496:	e10c      	b.n	80026b2 <HAL_RCC_OscConfig+0x4e2>
      while(HAL_IS_BIT_CLR(PWR->CR, PWR_CR_DBP))
 8002498:	4b6a      	ldr	r3, [pc, #424]	; (8002644 <HAL_RCC_OscConfig+0x474>)
 800249a:	681b      	ldr	r3, [r3, #0]
 800249c:	f403 7380 	and.w	r3, r3, #256	; 0x100
 80024a0:	2b00      	cmp	r3, #0
 80024a2:	d0f0      	beq.n	8002486 <HAL_RCC_OscConfig+0x2b6>
        }
      }
    }

    /* Set the new LSE configuration -----------------------------------------*/
    __HAL_RCC_LSE_CONFIG(RCC_OscInitStruct->LSEState);
 80024a4:	687b      	ldr	r3, [r7, #4]
 80024a6:	689b      	ldr	r3, [r3, #8]
 80024a8:	2b01      	cmp	r3, #1
 80024aa:	d106      	bne.n	80024ba <HAL_RCC_OscConfig+0x2ea>
 80024ac:	4b64      	ldr	r3, [pc, #400]	; (8002640 <HAL_RCC_OscConfig+0x470>)
 80024ae:	6f1b      	ldr	r3, [r3, #112]	; 0x70
 80024b0:	4a63      	ldr	r2, [pc, #396]	; (8002640 <HAL_RCC_OscConfig+0x470>)
 80024b2:	f043 0301 	orr.w	r3, r3, #1
 80024b6:	6713      	str	r3, [r2, #112]	; 0x70
 80024b8:	e01c      	b.n	80024f4 <HAL_RCC_OscConfig+0x324>
 80024ba:	687b      	ldr	r3, [r7, #4]
 80024bc:	689b      	ldr	r3, [r3, #8]
 80024be:	2b05      	cmp	r3, #5
 80024c0:	d10c      	bne.n	80024dc <HAL_RCC_OscConfig+0x30c>
 80024c2:	4b5f      	ldr	r3, [pc, #380]	; (8002640 <HAL_RCC_OscConfig+0x470>)
 80024c4:	6f1b      	ldr	r3, [r3, #112]	; 0x70
 80024c6:	4a5e      	ldr	r2, [pc, #376]	; (8002640 <HAL_RCC_OscConfig+0x470>)
 80024c8:	f043 0304 	orr.w	r3, r3, #4
 80024cc:	6713      	str	r3, [r2, #112]	; 0x70
 80024ce:	4b5c      	ldr	r3, [pc, #368]	; (8002640 <HAL_RCC_OscConfig+0x470>)
 80024d0:	6f1b      	ldr	r3, [r3, #112]	; 0x70
 80024d2:	4a5b      	ldr	r2, [pc, #364]	; (8002640 <HAL_RCC_OscConfig+0x470>)
 80024d4:	f043 0301 	orr.w	r3, r3, #1
 80024d8:	6713      	str	r3, [r2, #112]	; 0x70
 80024da:	e00b      	b.n	80024f4 <HAL_RCC_OscConfig+0x324>
 80024dc:	4b58      	ldr	r3, [pc, #352]	; (8002640 <HAL_RCC_OscConfig+0x470>)
 80024de:	6f1b      	ldr	r3, [r3, #112]	; 0x70
 80024e0:	4a57      	ldr	r2, [pc, #348]	; (8002640 <HAL_RCC_OscConfig+0x470>)
 80024e2:	f023 0301 	bic.w	r3, r3, #1
 80024e6:	6713      	str	r3, [r2, #112]	; 0x70
 80024e8:	4b55      	ldr	r3, [pc, #340]	; (8002640 <HAL_RCC_OscConfig+0x470>)
 80024ea:	6f1b      	ldr	r3, [r3, #112]	; 0x70
 80024ec:	4a54      	ldr	r2, [pc, #336]	; (8002640 <HAL_RCC_OscConfig+0x470>)
 80024ee:	f023 0304 	bic.w	r3, r3, #4
 80024f2:	6713      	str	r3, [r2, #112]	; 0x70
    /* Check the LSE State */
    if((RCC_OscInitStruct->LSEState) != RCC_LSE_OFF)
 80024f4:	687b      	ldr	r3, [r7, #4]
 80024f6:	689b      	ldr	r3, [r3, #8]
 80024f8:	2b00      	cmp	r3, #0
 80024fa:	d015      	beq.n	8002528 <HAL_RCC_OscConfig+0x358>
    {
      /* Get Start Tick*/
      tickstart = HAL_GetTick();
 80024fc:	f7ff fb8c 	bl	8001c18 <HAL_GetTick>
 8002500:	6138      	str	r0, [r7, #16]

      /* Wait till LSE is ready */
      while(__HAL_RCC_GET_FLAG(RCC_FLAG_LSERDY) == RESET)
 8002502:	e00a      	b.n	800251a <HAL_RCC_OscConfig+0x34a>
      {
        if((HAL_GetTick() - tickstart ) > RCC_LSE_TIMEOUT_VALUE)
 8002504:	f7ff fb88 	bl	8001c18 <HAL_GetTick>
 8002508:	4602      	mov	r2, r0
 800250a:	693b      	ldr	r3, [r7, #16]
 800250c:	1ad3      	subs	r3, r2, r3
 800250e:	f241 3288 	movw	r2, #5000	; 0x1388
 8002512:	4293      	cmp	r3, r2
 8002514:	d901      	bls.n	800251a <HAL_RCC_OscConfig+0x34a>
        {
          return HAL_TIMEOUT;
 8002516:	2303      	movs	r3, #3
 8002518:	e0cb      	b.n	80026b2 <HAL_RCC_OscConfig+0x4e2>
      while(__HAL_RCC_GET_FLAG(RCC_FLAG_LSERDY) == RESET)
 800251a:	4b49      	ldr	r3, [pc, #292]	; (8002640 <HAL_RCC_OscConfig+0x470>)
 800251c:	6f1b      	ldr	r3, [r3, #112]	; 0x70
 800251e:	f003 0302 	and.w	r3, r3, #2
 8002522:	2b00      	cmp	r3, #0
 8002524:	d0ee      	beq.n	8002504 <HAL_RCC_OscConfig+0x334>
 8002526:	e014      	b.n	8002552 <HAL_RCC_OscConfig+0x382>
      }
    }
    else
    {
      /* Get Start Tick */
      tickstart = HAL_GetTick();
 8002528:	f7ff fb76 	bl	8001c18 <HAL_GetTick>
 800252c:	6138      	str	r0, [r7, #16]

      /* Wait till LSE is ready */
      while(__HAL_RCC_GET_FLAG(RCC_FLAG_LSERDY) != RESET)
 800252e:	e00a      	b.n	8002546 <HAL_RCC_OscConfig+0x376>
      {
        if((HAL_GetTick() - tickstart ) > RCC_LSE_TIMEOUT_VALUE)
 8002530:	f7ff fb72 	bl	8001c18 <HAL_GetTick>
 8002534:	4602      	mov	r2, r0
 8002536:	693b      	ldr	r3, [r7, #16]
 8002538:	1ad3      	subs	r3, r2, r3
 800253a:	f241 3288 	movw	r2, #5000	; 0x1388
 800253e:	4293      	cmp	r3, r2
 8002540:	d901      	bls.n	8002546 <HAL_RCC_OscConfig+0x376>
        {
          return HAL_TIMEOUT;
 8002542:	2303      	movs	r3, #3
 8002544:	e0b5      	b.n	80026b2 <HAL_RCC_OscConfig+0x4e2>
      while(__HAL_RCC_GET_FLAG(RCC_FLAG_LSERDY) != RESET)
 8002546:	4b3e      	ldr	r3, [pc, #248]	; (8002640 <HAL_RCC_OscConfig+0x470>)
 8002548:	6f1b      	ldr	r3, [r3, #112]	; 0x70
 800254a:	f003 0302 	and.w	r3, r3, #2
 800254e:	2b00      	cmp	r3, #0
 8002550:	d1ee      	bne.n	8002530 <HAL_RCC_OscConfig+0x360>
        }
      }
    }

    /* Restore clock configuration if changed */
    if(pwrclkchanged == SET)
 8002552:	7dfb      	ldrb	r3, [r7, #23]
 8002554:	2b01      	cmp	r3, #1
 8002556:	d105      	bne.n	8002564 <HAL_RCC_OscConfig+0x394>
    {
      __HAL_RCC_PWR_CLK_DISABLE();
 8002558:	4b39      	ldr	r3, [pc, #228]	; (8002640 <HAL_RCC_OscConfig+0x470>)
 800255a:	6c1b      	ldr	r3, [r3, #64]	; 0x40
 800255c:	4a38      	ldr	r2, [pc, #224]	; (8002640 <HAL_RCC_OscConfig+0x470>)
 800255e:	f023 5380 	bic.w	r3, r3, #268435456	; 0x10000000
 8002562:	6413      	str	r3, [r2, #64]	; 0x40
    }
  }
  /*-------------------------------- PLL Configuration -----------------------*/
  /* Check the parameters */
  assert_param(IS_RCC_PLL(RCC_OscInitStruct->PLL.PLLState));
  if ((RCC_OscInitStruct->PLL.PLLState) != RCC_PLL_NONE)
 8002564:	687b      	ldr	r3, [r7, #4]
 8002566:	699b      	ldr	r3, [r3, #24]
 8002568:	2b00      	cmp	r3, #0
 800256a:	f000 80a1 	beq.w	80026b0 <HAL_RCC_OscConfig+0x4e0>
  {
    /* Check if the PLL is used as system clock or not */
    if(__HAL_RCC_GET_SYSCLK_SOURCE() != RCC_CFGR_SWS_PLL)
 800256e:	4b34      	ldr	r3, [pc, #208]	; (8002640 <HAL_RCC_OscConfig+0x470>)
 8002570:	689b      	ldr	r3, [r3, #8]
 8002572:	f003 030c 	and.w	r3, r3, #12
 8002576:	2b08      	cmp	r3, #8
 8002578:	d05c      	beq.n	8002634 <HAL_RCC_OscConfig+0x464>
    {
      if((RCC_OscInitStruct->PLL.PLLState) == RCC_PLL_ON)
 800257a:	687b      	ldr	r3, [r7, #4]
 800257c:	699b      	ldr	r3, [r3, #24]
 800257e:	2b02      	cmp	r3, #2
 8002580:	d141      	bne.n	8002606 <HAL_RCC_OscConfig+0x436>
        assert_param(IS_RCC_PLLN_VALUE(RCC_OscInitStruct->PLL.PLLN));
        assert_param(IS_RCC_PLLP_VALUE(RCC_OscInitStruct->PLL.PLLP));
        assert_param(IS_RCC_PLLQ_VALUE(RCC_OscInitStruct->PLL.PLLQ));

        /* Disable the main PLL. */
        __HAL_RCC_PLL_DISABLE();
 8002582:	4b31      	ldr	r3, [pc, #196]	; (8002648 <HAL_RCC_OscConfig+0x478>)
 8002584:	2200      	movs	r2, #0
 8002586:	601a      	str	r2, [r3, #0]

        /* Get Start Tick */
        tickstart = HAL_GetTick();
 8002588:	f7ff fb46 	bl	8001c18 <HAL_GetTick>
 800258c:	6138      	str	r0, [r7, #16]

        /* Wait till PLL is ready */
        while(__HAL_RCC_GET_FLAG(RCC_FLAG_PLLRDY) != RESET)
 800258e:	e008      	b.n	80025a2 <HAL_RCC_OscConfig+0x3d2>
        {
          if((HAL_GetTick() - tickstart ) > PLL_TIMEOUT_VALUE)
 8002590:	f7ff fb42 	bl	8001c18 <HAL_GetTick>
 8002594:	4602      	mov	r2, r0
 8002596:	693b      	ldr	r3, [r7, #16]
 8002598:	1ad3      	subs	r3, r2, r3
 800259a:	2b02      	cmp	r3, #2
 800259c:	d901      	bls.n	80025a2 <HAL_RCC_OscConfig+0x3d2>
          {
            return HAL_TIMEOUT;
 800259e:	2303      	movs	r3, #3
 80025a0:	e087      	b.n	80026b2 <HAL_RCC_OscConfig+0x4e2>
        while(__HAL_RCC_GET_FLAG(RCC_FLAG_PLLRDY) != RESET)
 80025a2:	4b27      	ldr	r3, [pc, #156]	; (8002640 <HAL_RCC_OscConfig+0x470>)
 80025a4:	681b      	ldr	r3, [r3, #0]
 80025a6:	f003 7300 	and.w	r3, r3, #33554432	; 0x2000000
 80025aa:	2b00      	cmp	r3, #0
 80025ac:	d1f0      	bne.n	8002590 <HAL_RCC_OscConfig+0x3c0>
          }
        }

        /* Configure the main PLL clock source, multiplication and division factors. */
        WRITE_REG(RCC->PLLCFGR, (RCC_OscInitStruct->PLL.PLLSource                                            | \
 80025ae:	687b      	ldr	r3, [r7, #4]
 80025b0:	69da      	ldr	r2, [r3, #28]
 80025b2:	687b      	ldr	r3, [r7, #4]
 80025b4:	6a1b      	ldr	r3, [r3, #32]
 80025b6:	431a      	orrs	r2, r3
 80025b8:	687b      	ldr	r3, [r7, #4]
 80025ba:	6a5b      	ldr	r3, [r3, #36]	; 0x24
 80025bc:	019b      	lsls	r3, r3, #6
 80025be:	431a      	orrs	r2, r3
 80025c0:	687b      	ldr	r3, [r7, #4]
 80025c2:	6a9b      	ldr	r3, [r3, #40]	; 0x28
 80025c4:	085b      	lsrs	r3, r3, #1
 80025c6:	3b01      	subs	r3, #1
 80025c8:	041b      	lsls	r3, r3, #16
 80025ca:	431a      	orrs	r2, r3
 80025cc:	687b      	ldr	r3, [r7, #4]
 80025ce:	6adb      	ldr	r3, [r3, #44]	; 0x2c
 80025d0:	061b      	lsls	r3, r3, #24
 80025d2:	491b      	ldr	r1, [pc, #108]	; (8002640 <HAL_RCC_OscConfig+0x470>)
 80025d4:	4313      	orrs	r3, r2
 80025d6:	604b      	str	r3, [r1, #4]
                                 RCC_OscInitStruct->PLL.PLLM                                                 | \
                                 (RCC_OscInitStruct->PLL.PLLN << RCC_PLLCFGR_PLLN_Pos)             | \
                                 (((RCC_OscInitStruct->PLL.PLLP >> 1U) - 1U) << RCC_PLLCFGR_PLLP_Pos) | \
                                 (RCC_OscInitStruct->PLL.PLLQ << RCC_PLLCFGR_PLLQ_Pos)));
        /* Enable the main PLL. */
        __HAL_RCC_PLL_ENABLE();
 80025d8:	4b1b      	ldr	r3, [pc, #108]	; (8002648 <HAL_RCC_OscConfig+0x478>)
 80025da:	2201      	movs	r2, #1
 80025dc:	601a      	str	r2, [r3, #0]

        /* Get Start Tick */
        tickstart = HAL_GetTick();
 80025de:	f7ff fb1b 	bl	8001c18 <HAL_GetTick>
 80025e2:	6138      	str	r0, [r7, #16]

        /* Wait till PLL is ready */
        while(__HAL_RCC_GET_FLAG(RCC_FLAG_PLLRDY) == RESET)
 80025e4:	e008      	b.n	80025f8 <HAL_RCC_OscConfig+0x428>
        {
          if((HAL_GetTick() - tickstart ) > PLL_TIMEOUT_VALUE)
 80025e6:	f7ff fb17 	bl	8001c18 <HAL_GetTick>
 80025ea:	4602      	mov	r2, r0
 80025ec:	693b      	ldr	r3, [r7, #16]
 80025ee:	1ad3      	subs	r3, r2, r3
 80025f0:	2b02      	cmp	r3, #2
 80025f2:	d901      	bls.n	80025f8 <HAL_RCC_OscConfig+0x428>
          {
            return HAL_TIMEOUT;
 80025f4:	2303      	movs	r3, #3
 80025f6:	e05c      	b.n	80026b2 <HAL_RCC_OscConfig+0x4e2>
        while(__HAL_RCC_GET_FLAG(RCC_FLAG_PLLRDY) == RESET)
 80025f8:	4b11      	ldr	r3, [pc, #68]	; (8002640 <HAL_RCC_OscConfig+0x470>)
 80025fa:	681b      	ldr	r3, [r3, #0]
 80025fc:	f003 7300 	and.w	r3, r3, #33554432	; 0x2000000
 8002600:	2b00      	cmp	r3, #0
 8002602:	d0f0      	beq.n	80025e6 <HAL_RCC_OscConfig+0x416>
 8002604:	e054      	b.n	80026b0 <HAL_RCC_OscConfig+0x4e0>
        }
      }
      else
      {
        /* Disable the main PLL. */
        __HAL_RCC_PLL_DISABLE();
 8002606:	4b10      	ldr	r3, [pc, #64]	; (8002648 <HAL_RCC_OscConfig+0x478>)
 8002608:	2200      	movs	r2, #0
 800260a:	601a      	str	r2, [r3, #0]

        /* Get Start Tick */
        tickstart = HAL_GetTick();
 800260c:	f7ff fb04 	bl	8001c18 <HAL_GetTick>
 8002610:	6138      	str	r0, [r7, #16]

        /* Wait till PLL is ready */
        while(__HAL_RCC_GET_FLAG(RCC_FLAG_PLLRDY) != RESET)
 8002612:	e008      	b.n	8002626 <HAL_RCC_OscConfig+0x456>
        {
          if((HAL_GetTick() - tickstart ) > PLL_TIMEOUT_VALUE)
 8002614:	f7ff fb00 	bl	8001c18 <HAL_GetTick>
 8002618:	4602      	mov	r2, r0
 800261a:	693b      	ldr	r3, [r7, #16]
 800261c:	1ad3      	subs	r3, r2, r3
 800261e:	2b02      	cmp	r3, #2
 8002620:	d901      	bls.n	8002626 <HAL_RCC_OscConfig+0x456>
          {
            return HAL_TIMEOUT;
 8002622:	2303      	movs	r3, #3
 8002624:	e045      	b.n	80026b2 <HAL_RCC_OscConfig+0x4e2>
        while(__HAL_RCC_GET_FLAG(RCC_FLAG_PLLRDY) != RESET)
 8002626:	4b06      	ldr	r3, [pc, #24]	; (8002640 <HAL_RCC_OscConfig+0x470>)
 8002628:	681b      	ldr	r3, [r3, #0]
 800262a:	f003 7300 	and.w	r3, r3, #33554432	; 0x2000000
 800262e:	2b00      	cmp	r3, #0
 8002630:	d1f0      	bne.n	8002614 <HAL_RCC_OscConfig+0x444>
 8002632:	e03d      	b.n	80026b0 <HAL_RCC_OscConfig+0x4e0>
      }
    }
    else
    {
      /* Check if there is a request to disable the PLL used as System clock source */
      if((RCC_OscInitStruct->PLL.PLLState) == RCC_PLL_OFF)
 8002634:	687b      	ldr	r3, [r7, #4]
 8002636:	699b      	ldr	r3, [r3, #24]
 8002638:	2b01      	cmp	r3, #1
 800263a:	d107      	bne.n	800264c <HAL_RCC_OscConfig+0x47c>
      {
        return HAL_ERROR;
 800263c:	2301      	movs	r3, #1
 800263e:	e038      	b.n	80026b2 <HAL_RCC_OscConfig+0x4e2>
 8002640:	40023800 	.word	0x40023800
 8002644:	40007000 	.word	0x40007000
 8002648:	42470060 	.word	0x42470060
      }
      else
      {
        /* Do not return HAL_ERROR if request repeats the current configuration */
        pll_config = RCC->PLLCFGR;
 800264c:	4b1b      	ldr	r3, [pc, #108]	; (80026bc <HAL_RCC_OscConfig+0x4ec>)
 800264e:	685b      	ldr	r3, [r3, #4]
 8002650:	60fb      	str	r3, [r7, #12]
            (READ_BIT(pll_config, RCC_PLLCFGR_PLLN) != (RCC_OscInitStruct->PLL.PLLN) << RCC_PLLCFGR_PLLN_Pos) ||
            (READ_BIT(pll_config, RCC_PLLCFGR_PLLP) != (((RCC_OscInitStruct->PLL.PLLP >> 1U) - 1U)) << RCC_PLLCFGR_PLLP_Pos) ||
            (READ_BIT(pll_config, RCC_PLLCFGR_PLLQ) != (RCC_OscInitStruct->PLL.PLLQ << RCC_PLLCFGR_PLLQ_Pos)) ||
            (READ_BIT(pll_config, RCC_PLLCFGR_PLLR) != (RCC_OscInitStruct->PLL.PLLR << RCC_PLLCFGR_PLLR_Pos)))
#else
        if (((RCC_OscInitStruct->PLL.PLLState) == RCC_PLL_OFF) ||
 8002652:	687b      	ldr	r3, [r7, #4]
 8002654:	699b      	ldr	r3, [r3, #24]
 8002656:	2b01      	cmp	r3, #1
 8002658:	d028      	beq.n	80026ac <HAL_RCC_OscConfig+0x4dc>
            (READ_BIT(pll_config, RCC_PLLCFGR_PLLSRC) != RCC_OscInitStruct->PLL.PLLSource) ||
 800265a:	68fb      	ldr	r3, [r7, #12]
 800265c:	f403 0280 	and.w	r2, r3, #4194304	; 0x400000
 8002660:	687b      	ldr	r3, [r7, #4]
 8002662:	69db      	ldr	r3, [r3, #28]
        if (((RCC_OscInitStruct->PLL.PLLState) == RCC_PLL_OFF) ||
 8002664:	429a      	cmp	r2, r3
 8002666:	d121      	bne.n	80026ac <HAL_RCC_OscConfig+0x4dc>
            (READ_BIT(pll_config, RCC_PLLCFGR_PLLM) != (RCC_OscInitStruct->PLL.PLLM) << RCC_PLLCFGR_PLLM_Pos) ||
 8002668:	68fb      	ldr	r3, [r7, #12]
 800266a:	f003 023f 	and.w	r2, r3, #63	; 0x3f
 800266e:	687b      	ldr	r3, [r7, #4]
 8002670:	6a1b      	ldr	r3, [r3, #32]
            (READ_BIT(pll_config, RCC_PLLCFGR_PLLSRC) != RCC_OscInitStruct->PLL.PLLSource) ||
 8002672:	429a      	cmp	r2, r3
 8002674:	d11a      	bne.n	80026ac <HAL_RCC_OscConfig+0x4dc>
            (READ_BIT(pll_config, RCC_PLLCFGR_PLLN) != (RCC_OscInitStruct->PLL.PLLN) << RCC_PLLCFGR_PLLN_Pos) ||
 8002676:	68fa      	ldr	r2, [r7, #12]
 8002678:	f647 73c0 	movw	r3, #32704	; 0x7fc0
 800267c:	4013      	ands	r3, r2
 800267e:	687a      	ldr	r2, [r7, #4]
 8002680:	6a52      	ldr	r2, [r2, #36]	; 0x24
 8002682:	0192      	lsls	r2, r2, #6
            (READ_BIT(pll_config, RCC_PLLCFGR_PLLM) != (RCC_OscInitStruct->PLL.PLLM) << RCC_PLLCFGR_PLLM_Pos) ||
 8002684:	4293      	cmp	r3, r2
 8002686:	d111      	bne.n	80026ac <HAL_RCC_OscConfig+0x4dc>
            (READ_BIT(pll_config, RCC_PLLCFGR_PLLP) != (((RCC_OscInitStruct->PLL.PLLP >> 1U) - 1U)) << RCC_PLLCFGR_PLLP_Pos) ||
 8002688:	68fb      	ldr	r3, [r7, #12]
